:020000040000FA
:1000000000F80202B5700000F13400006D420000FB
:1000100000000000000000000000000000000000E0
:1000200000000000204F0100684F0100F134000083
:100030000000000000000000F13400002D770000F7
:10004000E9320000F1340000F1340000D570000006
:10005000754A0000A96B000081340000753500006E
:100060005918000095170000F1340000F534000025
:10007000494A0000958C0000557000008170000016
:10008000F1340000F1340000F1340000817A000006
:10009000A17A0000F1340000F1340000F1340000D6
:1000A000397F0000437F0000EB320000696F0000E1
:1000B000F1340000116C000000000000000000009E
:1000C0000348854600F016FF0048004779CA000043
:1000D00000F8020230B50B46014600202022012420
:1000E00009E00D46D5409D4205D31D469540491B6C
:1000F0002546954040191546521E002DF1DC30BDB5
:1001000070B500242546002801DA01244042002968
:1001100001DA01254942FFF7DDFFAC4200D0404241
:10012000002C00D0494270BDF8B5002425460029B6
:1001300004DA0E46012400214042B141002B04DACA
:100140001E46002352420125B34100F0D1FC8C46EB
:1001500017461E46AC4203D0002540428D41AC46B6
:10016000002C02D0002657429E4161463A46334653
:1001700001B0F0BD03460B439B0703D009E008C95B
:10018000121F08C0042AFAD203E00B780370401C47
:10019000491C521EF9D27047D2B201E00270401CD5
:1001A000491EFBD270470022F6E710B513460A46F7
:1001B00004461946FFF7F0FF204610BDCAB2401EA4
:1001C0004178401C8A4202D00029F9D100207047B2
:1001D000421C0178401C0029FBD1801A704730B5C1
:1001E00004460020034600E05B1C934203D2E05C1F
:1001F000CD5C401BF8D030BD30B50546002003462D
:1002000000E05B1C934205D2EC5CC85C201A01D173
:10021000002CF6D130BD00000FB400B58DB00990B0
:100220000B9010A900200091C0430A9000200C9070
:1002300006480690064807906A4609A80F9900F0FC
:10024000C1FC0DB008BC04B018470000E50B00006D
:10025000050C0000FFB5002083B0009050680190AD
:1002600091691446002697680498884705460C99BA
:100270000698084305D009E0A169761C04988847D0
:100280000546216A284688470028F5D1681C03D016
:100290000198C00704D017E00020C04307B0F0BDAC
:1002A0002068011D2160006800900DE00198C007E2
:1002B00004D1009805700098401C0090A169761C3C
:1002C0007F1E049888470546002F1CDD681C1AD045
:1002D000069800280FD0E817C00E401941118A0077
:1002E00006994009511840012A1A096801209040D6
:1002F0000142DBD107E00C980028D7D1216A2846BB
:1003000088470028D2D0E169049888470C980028D3
:1003100007D1002E05DD0198C00702D10098002109
:100320000170A068B84204DD0C98002804D0002FAA
:1003300002D00120C043B1E73046AFE770B50646B2
:1003400011F052F9046805460A220021304600F0F7
:10035000C5FC2C6070BDF8B502464A40D40F42007F
:100360004B0052085B089A4202D2024608461146E8
:100370004A0023D0C30D4A00DDB2120EAD1A202D63
:1003800035DA49020126490AF6058A19002C00D0FF
:10039000524220214F1B1146B9402A411018C20D6C
:1003A0009A4221D0002C17D0012D08DCDA05801AE2
:1003B000D20F8019D207DBB200F0D0FCF8BDDA050D
:1003C000801A012340001B06C01880185A4280186A
:1003D000CA0F1043490007E04908C2071143DA0574
:1003E000801A80194008801800F0B0FCF8BD610048
:1003F0000122511A001BF7E70122D2075140AAE758
:100400000122D2075040A6E7024670B54A40D30FFA
:10041000DB0740002DD04A002AD0010E140E000246
:1004200012020919400A520A8418E501044654438D
:10043000000A120A2E045043A4194219200CC54385
:10044000AA18120C0125AD03521C521912047F394F
:10045000240400D0521C104301D44000491EC2B2F3
:100460000C06C0092018401C4008802A02D003E076
:10047000002070BD40084000002900DA0020184329
:1004800070BD70B502464A40D50F40004A00ED07E6
:1004900040085208002814D0002A12D0C40DD30DF1
:1004A00041020120C0055202490A520AE41A091801
:1004B00012187D34914201D3641C00E04900002CE5
:1004C00001DA002070BD0023914201D3891A034351
:1004D000400849000028F7D100290AD0914202D1F2
:1004E0000121C90705E0914201D2012101E001216A
:1004F000C943E005C018401900F028FC70BD000099
:10050000F0B507460846584087B0C00F0490480031
:100510000E46590040084908BC1A884105D23846A1
:1005200031461E4617460B46024658004008104307
:100530004CD0300D039040055900400D490D0590F9
:10054000401A0290402872DA18030121000B0905B5
:100550000843019004980092002805D00199524266
:100560000020884100920190029840210A1A0199C6
:10057000009800F0EDFA05460C466B4607CB00F0FC
:1005800008FBC0197141039A0E0D0023D71756407E
:100590001A467A40164344D0049A002A2DD0029A73
:1005A000012A039A15DC1205C01A9141012636056D
:1005B000001C7141D20F059ED20700930192029652
:1005C0002A46234600F010FC07B0F0BD38463146FD
:1005D000FAE71605224A0F46B218C01AB7410121A0
:1005E0000905001C4F4100187F4111461818794138
:1005F000E20F10436D19644113E0E2076D081543E3
:100600006408C2071443039A01261205C01A9141D7
:100610003605001C7141CE07400830434908C01818
:1006200051412A46234600F0D2FBCDE7FFE704986C
:1006300001224000C117121A00238B410498314651
:10064000C417381AA141EEE730B40124E40763402F
:1006500030BC55E730B40124E407614030BC4FE7BB
:100660000000E0FFF0B51FB488B00B990998002492
:1006700048400999C00F490049080991C0070B99E2
:100680000090490049080B9109990898A64608432B
:100690001CD00B990A98084318D0099801244000EF
:1006A000420D4800410D099824050003000B20432A
:1006B00009900B980003000B20430B9050181C4925
:1006C0004018002201901446104605E00020014623
:1006D0000DB0F0BD032801DA034600E003239C4679
:1006E000C11A0AAE0AE05F0008ADED5B4F00F75B90
:1006F0007D430027AA187C41491C5B1E6145F2DD41
:10070000410004AB5A522104120C0A43240C401C31
:100710000828DFDB01980290009970460191009053
:10072000059B049A0799069800F05EFBD0E700004D
:100730000DFCFFFFF0B50C465C4085B0E40FE4070C
:1007400003944C0000266408590094464908024668
:100750000296224321D062460A431ED06200570D02
:100760004A000E032303550D012402462C4924059B
:10077000781B1B0B360B4018234326436146009021
:100780001C46501AB44103D30098401C009002E06C
:10079000921800985B41002803DA0020014605B05A
:1007A000F0BD0020012109050746864611E0644698
:1007B0001D46141BB54106D36546521BB341744612
:1007C00007430C43A646CD07400849082843921822
:1007D0005B4105460D43EAD11046184313D06046ED
:1007E000194650407140084306D06046101AB34184
:1007F00006D20122002306E000220123DB0702E0EB
:100800000122D2435310009874460105381C6141FF
:10081000029C039D0019694100F0D9FABFE700006E
:10082000FD0300000122D207002800DB101A002976
:1008300000DB511A814201D8012070470020704727
:100840000122D207002800DB101A002900DB511A10
:10085000814201D201207047002070470122D20757
:10086000002800DB101A002900DB511A814201D355
:1008700001207047002070470122D207002800DBCA
:10088000101A002900DB511A814201D9012070475A
:10089000002070470122D207002800DB101A00292F
:1008A00000DB511A814201D10120704700207047BE
:1008B00010B5002904DB0C460121C9074042A141C3
:1008C000002B04DB1C460123DB075242A341801AA4
:1008D000994101D3012010BD002010BD10B50029A1
:1008E00004DB0C460121C9074042A141002B04DB77
:1008F0001C460123DB075242A341101A8B4101D34E
:10090000012010BD002010BDC217C10F504010B50E
:100910004018CA079623002100F020FA10BD10B538
:1009200000229623114600F019FA10BD0EB5C21729
:10093000C10F5040CA0740180021054B0293019295
:1009400000910A460B4600F04FFA03B000BD0000CC
:10095000330400000EB505490291002100910A46BA
:100960000B46019100F040FA03B000BD33040000D3
:100970003EB5CA17CB0F002450405140C01861410A
:10098000DA07054B0293019200942246234600F0B9
:100990002BFA03B030BD000033040000C20F410049
:1009A00040020123400ADB05D207090EC0187F2947
:1009B00001DA00207047962903DC9623591AC840B3
:1009C00001E096398840002AF4D040427047410047
:1009D00040020122400AD205090E80187F2901DA5F
:1009E00000207047962903DC9622511AC8407047B0
:1009F000963988407047000070B5CD0F4A00090352
:100A00000123090B1B0519430B4BED070024520D65
:100A10009A4201DA002070BD074B34339A4203DC5E
:100A20009A1A00F0A5F802E00449511888402C43B6
:100A3000F1D0404270BD0000FF030000CDFBFFFF7E
:100A400070B5CD0F4A0009030123090B1B0519439B
:100A50000D4BED070024520D9A4202DA00200146A8
:100A600070BD094B34339A4203DC9A1A00F080F8C7
:100A700003E0064BD21800F06BF82C43F0D00022B4
:100A800040428A41114670BDFF030000CDFBFFFFCD
:100A9000C20FD207400040080BD0C10D0723DB0175
:100AA000C91840020905400A1143C2084007114312
:100AB0007047002001467047CB0FDB07490010B597
:100AC000490802460A4307D00A0D07240903E40136
:100AD000090B121B002A01DC002010BDC900440FC5
:100AE0000C43C100E018D205801800F02FF910BDAA
:100AF000F0B51FB40646002082B00546402401919F
:100B000000901BE0019922460F46304600F030F875
:100B1000049A059B801A994110D310461946224623
:100B200000F016F8361A8F41019722460120002165
:100B3000009F00F00DF838184D4100902046641ECB
:100B40000028DFDC019B00982946324607B0F0BD43
:100B500010B5202A04DB0146203A9140002010BD48
:100B6000914020239C1A0346E3401943904010BD56
:100B700010B5202A04DB0846203AD040002110BDE1
:100B80000B46D340D0402024A21A91400843194676
:100B900010BD10B5202A06DBCB170846203A1041BD
:100BA000C1170B4306E00B461341D0402024A21A84
:100BB00091400843194610BD02681378511801602E
:100BC0001846704710B5D16004495161044911625B
:100BD00000211161114600F0ADF910BDB90B000004
:100BE000210F00004268002A08D001680B78491CD8
:100BF000002B03D0521E06C0184670470121C16069
:100C0000881E70474268002A0BD0C3680168002B19
:100C100007D183688B4204D0491E521C06C00020B5
:100C200070470020C04370470FB400B589B00A4632
:100C30000DA9009100230C99002ACB60234B069349
:100C4000234B079301D0042300E00023214A0292A2
:100C5000214A0892019302466B46002000F095FB62
:100C600009B008BC04B01847F0B585B007460020AD
:100C7000C04301901E46002015460C46009102918B
:100C800004903B466A46314604A8FFF7CDFF04991D
:100C900002466018002D05D0002901D0034600E06F
:100CA00023462B6000290ED0002A02DD00998142E4
:100CB00009D0001B019000943B466A4631460294DD
:100CC00004A8FFF7B1FF05B0F0BD0000E50B000080
:100CD000050C0000FFFFFF7F210F0000F7B5009C0F
:100CE0000F4600262578641C002D05D000F014F96D
:100CF0000068405DC007F5D12B2D02D02D2D18D0F6
:100D0000641E39462046029A00F06AFC002F04D087
:100D10003968A14201D10099396071050224002986
:100D20000BDA4042002803DD10F05EFC0460A007EF
:100D3000FEBD012080020643E3E70028F8DA10F048
:100D400053FC04600048FEBDFFFFFF7F002904DA6A
:100D5000401C490001D140084000704770B4002495
:100D6000050C05D11024000402D1002921D0112442
:100D7000050E01D100020834050F01D10001241D28
:100D8000850F01D18000A41C002801DB4000641CF9
:100D9000002908D020252E1B0D46F540A14000D08B
:100DA00001212943084301061B1B000ADB1D02D554
:100DB000002070BC7047DB05181880180029F8DA8D
:100DC000401C4900F5D170BC40084000704710B588
:100DD000002B08DA0024401C614192185B411A4341
:100DE00001D14008400010BDF0B51FB482B00546E7
:100DF0000C0003D0084610F0DFFB02E010F0DCFB33
:100E000020300246009021462846FFF7A1FE049BB1
:100E1000059A04460F4618431143084314D0184658
:100E200010431BD0009840210A1A18460599FFF775
:100E30009FFE05460E46009A05990498FFF788FE26
:100E4000084305D0012004E02046394607B0F0BD34
:100E50000020C11705430E432C43374300990E98D9
:100E60006305401A7905E40A00220C43FD0A0A30A2
:100E700002D500200146E9E70105101969410C9CE3
:100E80000D9D00196941FFF7A2FFDFE74A00090342
:100E90000123090B1B0519430A4B10B5520D9A4249
:100EA00002DA0020014610BD064B34339A4203DCBF
:100EB0009A1AFFF75DFE10BD034BD218FFF748FEEC
:100EC00010BD0000FF030000CDFBFFFF10B500299F
:100ED00004DB0124E40740428C412146002B04DB63
:100EE0001C460123DB075242A341994200D19042A4
:100EF00010BD0000064C0125064E05E0E36807CC56
:100F00002B430C3C98471034B442F7D3FFF7DCF87E
:100F1000604901008049010000487047841F0100BA
:100F200010B50446FFF7F8FF0068005DC007C00F6A
:100F300010BD0000F3B58DB000200A9001200B9089
:100F4000002608460C300C46099062690121099878
:100F50009047051E2ED0252D2DD0216A88470028C8
:100F600018D06269012109989047216A88470028B2
:100F7000F7D1411E62690998904700E0761CA1698B
:100F80000D988847216A88470028F7D1E1690D98B4
:100F90008847DAE7A1690D9888470746A84201D13A
:100FA000761CD2E7E1690D9888477F1C02D10A9828
:100FB000002877D049E1002762693D463946099803
:100FC00090472A280CD16269012109989047012590
:100FD00006E00A214F433F18303FEBD41020054371
:100FE0006269012109989047014630390A2903D2E4
:100FF0009B498F42DEDCECE7E90600D4994F6C2870
:101000000AD04C2810D0682824D06A282ED0742802
:101010000CD07A280AD00DE0626901210998904726
:101020006C2823D004211CE02020054362690121A3
:1010300009989047A760656065284FD026DC58283E
:1010400039D01ADC452849D012DC252834D0412873
:10105000B0D143E06269012109989047682802D025
:1010600008210D43E6E70120C002DEE70220DCE7AD
:10107000462833D047282CD130E05B2870D0612837
:101080002CD063286CD0642823D161E06F284FD026
:1010900009DC662822D0672820D0692826D06E284F
:1010A00017D12EE0CDE070284DD073286FD0752871
:1010B0004ED078280DD154E0A1690D988847054697
:1010C000252800D16CE7E1690D9888476D1C00D197
:1010D0006DE7BAE00A224CE00A2252E001202346E2
:1010E0006A46C0430D9900F050F9A3E0284640211C
:1010F00008436060A807234601D5002239E000229A
:101100003FE0E80700D020E72068011D216000686B
:10111000290501D5067018E7290701D5068014E7CF
:10112000A90703D5F117066041600EE706600CE7DA
:101130002846402108436060A807234601D50822BD
:1011400017E008221DE0484928460840606016E084
:101150002846402108436060A8072346BCD5B9E76C
:1011600015E02846402108436060A80707D52346BC
:1011700010220120C0430D99C046C0465AE02346C4
:1011800010220120C0430D99C046C04652E0002104
:101190000C910B460091632802D05B2807D043E0F6
:1011A000E80601D40120A060012000903CE06269C3
:1011B0000121099890475E2805D101200C90014635
:1011C0006269099890472169002906D10B4601AA56
:1011D0008F00491CD3510829FADB002835D021693A
:1011E00000290ED1C117C90E09184A11930001AA8E
:1011F0009A1849094901411A01201368884003439C
:10120000136062690121099890475D28E5D10C9827
:10121000002808D0002001AB81005A58401CD2435E
:101220005A500828F8DB01AB01202246C0430D9933
:10123000FFF710F800280ADA401C06D10B980028A6
:1012400003D00020C0430FB0F0BD0A98FBE7E907C8
:1012500002D10A99491C0A91361800200B9074E6B5
:10126000CCCCCC0CFFFFFF7FF1F7FFFFFFB5087878
:1012700089B01546FF2805D0491C2D2804D000222E
:10128000002407E000240BE00122F9E70A235C4375
:101290000419491C0878FF28F8D1002A00D06442BC
:1012A000002004902A7801462D2A01D02B2A0FD144
:1012B0006D1C2D2A02D00022049209E00122FBE7D6
:1012C00000260A2233466D1C00F0DDF93818714102
:1012D0002F78FF2FF4D10C9AA218069202460A43E7
:1012E00004D0FF23069A9133DA4205DA00210998E7
:1012F0000A4606C00DB0F0BD0024B74AB54D2646DB
:10130000079200F00DFA029006980391002801DA86
:10131000474200E0074639050020AF4A001C514112
:101320000191009012E0F80707D022462B46304684
:101330000799FFF797F90646079122462B46104674
:101340001946FFF78FF904460D467F10002FEAD1AA
:101350000698019B0028009A0399029806DAFFF785
:10136000E9F93246079BFFF7E5F905E0FFF77AF95F
:101370003246079BFFF776F9049A002A02D0012231
:10138000D2075140099A03C2B4E7FFB591B00020DB
:1013900009900025ED432E209E685C681F46019051
:1013A000B9696D1C129888470090396A88470028EF
:1013B000F6D10098401C0AD00D20C0018443002EB5
:1013C00012DD00982B2809D02D280DD103E0002034
:1013D000C04315B0F0BD012080020443B9696D1C03
:1013E00012988847761E009003A9600501D52D202C
:1013F00000E02B206A461073491C0CA80F91029044
:101400000AE0B9696D1C12988847009001204002DB
:1014100004431398761E0560002E02DD00983028E4
:10142000EFD001990098884245D18020044308E01C
:101430000998401E09900120400204431399681C3A
:101440000860B9696D1C761E129888470090302894
:10145000EED030E00199884205D1200603D48020E7
:101460000443761E1DE0009810F08CF9002825D06A
:10147000012149020C43009807AA0F990332303822
:10148000761E914208D208700F98401C0F902006DB
:1014900007D50998401E03E0200602D40998401C95
:1014A0000990A00502D51399681C0860B9696D1CE4
:1014B000129888470090002ECCDC59E0002E57DDB2
:1014C0000098652801D0452852D1A00550D50320A9
:1014D00000028443B9696D1C761E129888470090FB
:1014E000002E0CDD2B2804D02D2808D1FF20013040
:1014F0000443B9696D1C12988847761E0090E00578
:1015000001D52D2100E02B21029801700298401C8A
:101510000290019025E00120400204430EA90298A8
:101520000131761E88420ED20098029930380006AA
:10153000000E087003D10299019881420AD90298DD
:10154000401C029006E0E00501D5244801E0234854
:1015500040420990B9696D1C129888470090139811
:101560000560002E04DD009810F00CF90028D2D19F
:10157000F969129888470F99FF200870029903AA09
:10158000087000200A900B900CA90AA8099BFFF78D
:101590006DFEA00502D40120C0431AE724200442B6
:1015A00009D0E00713D138680B9A0A99031D3B60F4
:1015B000006806C00BE00B990A98FFF77DFA014618
:1015C000E00704D13868021D3A60006801602846CF
:1015D000FFE60000000014400000F03FF1D8FFFFDC
:1015E000F7B582B0029C00272078641C154601974D
:1015F000302802D0002D15D015E020780127641C7A
:10160000782804D0582802D0002D09D00BE0002DF6
:1016100001D0102D07D1002710252078641C02E08E
:10162000082500E00A250026009610E00099012711
:1016300069430818020C294680B2714300908E1845
:101640003804864201D3012001902078641C294689
:1016500000F056F80028E9DA0398002805D0002F9A
:1016600001D0641E00E0029C04600198002806D0AE
:101670000FF0BAFF02210160C81E05B0F0BD00994D
:1016800030040843F9E7F0B51FB486B0002000909D
:10169000019002900698069980B204900798090C70
:1016A00002040014114307900027089D0998069131
:1016B0003E463C4603900398A9B20204000C0390F6
:1016C00004982D0C1543484300212246FFF740FAA9
:1016D000C719714110340E46402CECDB3846029A93
:1016E000FFF736FA009A019B801800905941029842
:1016F0000191103002904028CCDB00980BB0F0BD77
:101700003A2800D23038202302469A43412A01D396
:1017100010463738884201D30020C043704700008C
:101720000EB5054A02920022009213460192FFF77D
:101730005BFB03B000BD00003304000070B58C18E3
:101740000578401C6B075B0F01D10378401C2A1100
:1017500006D10278401C03E006780E70401C491C3C
:101760005B1EF9D12B0705D40023521E0DD40B703C
:10177000491CFAE70378401CCB1A921C03E01D7841
:101780000D70491C5B1C521EF9D5A142D8D3002014
:1017900070BD000010B52148016A8A0715D44A07B8
:1017A00015D4C90732D01E498A89002A15D0531E84
:1017B0008B8182688C6904C48C610A691B040DD01A
:1017C000002A22D10121016010BD022100E0042184
:1017D000C16113488021416110BD0A69012A09D104
:1017E000026801239A430260C361FF206830993088
:1017F0000C4A106001204861CA69002A05D0886936
:1018000009898B00C01A904710BD10BDFF226832B5
:10181000054806A109A30DF049FBC04608D00140C8
:10182000A095010280E200E0D82E01004144435F10
:1018300049525148616E646C65720000556E65785E
:101840007065637465642041444320696E746572F9
:10185000727570740D0A000070B582B00023019398
:10186000444801688A6A4C6813252540132D02D12B
:10187000CB689B07DB0F4361930772D453070AD4ED
:10188000D30711D1130724D5048F838E1C1B102C72
:101890000EDD102310E0042088620220032142A202
:1018A0000EF060FB02B070BD0120886202B070BD16
:1018B000048F1B1B1C0610D0DBB20024058FC66AE8
:1018C00075192D5D0D74641CA342F7D1048FE318C4
:1018D0000387D20607D400212FE04B6A0824A343D4
:1018E0004B62D206F7D5CB68C28E448F141B5B04C3
:1018F000DB0EA34201D3438FD31ADAB2002A16D0EB
:10190000097D438F046BE1540199012A10D0012312
:101910001C46890145582D7D41184E8F9B19096B36
:10192000CD54641CE3B201999A42F2D800E0002140
:101930008B01C3185C8FA2185A878A0181184B8FBC
:10194000CC8EA3420BD301230B618058002242624C
:10195000CA6B002A03D03A31098801A8904702B027
:1019600070BD02208862044804A1084A08A30DF053
:101970009DFAC04684900102F12E01004145535F5B
:1019800049525148616E646C65720000CE020000DD
:1019900041455320696E707574206F766572666C70
:1019A0006F770D0A00000000414553206F75747079
:1019B000757420756E646572666C6F770D0A000031
:1019C000F0B581B001243F2900D993E00346806837
:1019D000456B2D688E0001A7BE59B7461B1B000042
:1019E000371B0000131B0000131B0000F51A00003A
:1019F000F51A0000F51A0000F51A0000F51A0000AB
:101A0000F51A0000F51A0000F51A0000F51A00009A
:101A1000F51A0000491B0000651B0000F51A0000C4
:101A2000F51A0000F51A0000F51A0000F51A00007A
:101A3000F51A0000F51A0000F51A0000F51A00006A
:101A4000F51A0000F51A0000F51A0000F51A00005A
:101A5000F51A0000F51A0000F51A0000F51A00004A
:101A6000F51A0000F51A0000F51A0000F51A00003A
:101A7000F51A0000F51A0000F51A0000F51A00002A
:101A8000F51A0000F51A0000F51A0000F51A00001A
:101A9000F51A0000F51A0000F51A0000F51A00000A
:101AA000F51A0000F51A0000F51A0000F51A0000FA
:101AB000F51A0000DD1A0000DD1A0000DD1A000032
:101AC000DD1A0000DD1A0000DD1A0000DD1A00003A
:101AD000DD1A0000DD1A0000DD1A0000434800692D
:101AE0000024022809D001280DD0002802D103CA01
:101AF00004F0A6FF204601B0F0BD03CA04F092FF37
:101B0000204601B0F0BD03CA04F0B0FF204601B08A
:101B1000F0BD022931D0022430E0344D00242C6184
:101B20006C619849354A01F05FFE6869401C686144
:101B3000204601B0F0BD01F091FE284602F0FEF80B
:101B40000024204601B0F0BD284909690C234B430D
:101B50002749CA58C918496801F046FE00242046A2
:101B600001B0F0BD0024204604F038FF0128C1D1A7
:101B70001E483030204900241CE001241B490F6915
:101B80000C26314679431A4A51188968214208D0F7
:101B900000247D1C15490D614C61042D10D315499D
:101BA00006E012494869401C4861032812D32949BC
:101BB00000241846224602F071F8204601B0F0BD1C
:101BC0006E430B498A598919496801F00DFE204678
:101BD00001B0F0BD0E20009000240A2228462146C4
:101BE00002F04CF8204601B0F0BDC0463899010221
:101BF000881F01008826010068260100563A01006E
:101C0000B0B504290FD804468068C04679440979E4
:101C100049008F44020A0E1C1700104910A201F05F
:101C2000E3FD0020B0BD0120B0BD01F017FE002093
:101C3000B0BD00250321284604F0E0FE06492046F9
:101C40002A4602E003490022204602F027F800203D
:101C5000B0BDC04678260100F826010088130000B8
:101C6000415445300D0A0000B0B582B001240A2964
:101C700010D883687944097949008F440E290505F5
:101C80000B0B0B0B0B0B1A00194909680024224699
:101C900002F004F8204602B0B0BD50681449086054
:101CA000144915A2184601F09FFD0024204602B0F9
:101CB000B0BD0024019403CA09A201AB02F00CF9E3
:101CC0000228E7D1019804F0EDFE204602B0B0BD35
:101CD000184601F0C3FD0024204602B0B0BDC04646
:101CE0002B4353513A2025642C252A0D0A0000006D
:101CF000E09A01028813000041542B4353510D0A0E
:101D000000000000B0B582B00546002404F0C4FE17
:101D100001280DD108498C60E86B426853684B601C
:101D2000009401926A4601F0B9FF204602B0B0BDAE
:101D3000E443204602B0B0BDC8930102B0B50546E9
:101D4000881E02280AD3A868012913D0002915D1BA
:101D50000C490DA201F048FD0020B0BD0220014653
:101D600004F04CFE064900242846224601F096FF66
:101D70002046B0BD01F072FD0020B0BD0120B0BD15
:101D8000482601008813000041542B4346554E3D20
:101D9000300D0A0080B5E0B00320C10168460FF0A5
:101DA000F3FB06480078002804D003206A46014669
:101DB0000EF0D8F8002060B080BDC0469F990102A7
:101DC000F0B597B008201490642013902548109027
:101DD00002200E904B20C0011690234D284614304F
:101DE000129001270F97B802119003200EA906F058
:101DF000A3F90026F443002802D0204617B0F0BD16
:101E00000C35284601F0A8FF0028F6D180200C9060
:101E100016490B910A9016480990164808901648E2
:101E200007901648069039200590154804901548EB
:101E300003900D95144D03A9284601F03FFD00289D
:101E4000DBD1009501970F4C104911A2124B20468F
:101E500001F0D8FE1149204601F008FF3446204623
:101E600017B0F0BD60C001022C97010260C40102EE
:101E7000E0C40102192F0000792F0000E92E0000B4
:101E8000082801006899010270C90102E8250100D3
:101E9000414952373830450008270100951D0000A0
:101EA00010B50348002404700EF0E8FF204610BD72
:101EB000F89E010280B501F04BF9002080BD0000C2
:101EC000F0B58DB00E4600270C970B970A9709972F
:101ED0000897079706970597029080680490406BD3
:101EE0000068019004F074FD04465BA10522039292
:101EF000FEF782F95A4D00281ED05AA1052220462D
:101F0000FEF77AF9002817D058A105222046FEF7DF
:101F100073F900280FD059A105222046FEF76CF96D
:101F2000002809D057A105222046FEF765F90028B0
:101F300007D156A500E04FA505A820212A4602F0AA
:101F40009DF801203F2E00D936E0C0467E44367908
:101F50007600B7443340474A57313131313131315E
:101F6000313165303131313131313131313131312E
:101F70003131313131313131313131313131313151
:101F8000313131313131313131311F1F1F1F1F1FAD
:101F90001F1F1F1FBE48416A04290CD1039A4262C9
:101FA00087620C2050433D490A580818416805AB28
:101FB000049801F019FC38460DB0F0BDB44C002077
:101FC0006062A062CD49364A049801F00DFCA06A17
:101FD000401CA062EFE7049801F040FC019801F07A
:101FE000ADFEE8E7AA48406A05E0A949486A01222F
:101FF0000243032A1CD1A649421C4A628F62062A68
:10200000CFD30BE0A2494A6A012013460343052BB4
:10201000D2D1501C48628F62062803D31E490DE0BE
:102020009B48406A0C2141431C4842584018BDE778
:10203000886A401C8862032805D31649002202984A
:1020400001F02CFEB7E70E20009000210A22019833
:10205000029B01F013FEAEE7343630303000000052
:102060007E3A0100343630303200000034363030F1
:1020700031000000554E494E455400003436303092
:1020800036000000343630303300000043544E45F3
:1020900054000000E825010038260100B81F0100A7
:1020A000FE39010070B5022956D30F2907D1784CAB
:1020B000217A012905D1002222728F494AE00120AC
:1020C00070BD866801F06EFE002004F08FFC0128D0
:1020D00003D10020032104F091FC0025284604F0E0
:1020E0007DFC012804D130346A490022204631E0C9
:1020F000304600F0EFFD00282ED03046FFF702FEFC
:10210000002829D004F084FC012807D15F498D60A4
:10211000F06B4268E26252684A601AE0022004F002
:102120005DFC012808D159498D61F06B4268E2627B
:1021300052684A6110310CE0022004F057FC01287B
:102140000AD152498D62F06B4268E26252684A627B
:1021500020312A4601F0A2FD002070BD10B582B0EA
:1021600003460120272931D87944097949008F4451
:102170002C132D2D162D2D2D2D2D2D2D2D2D2D2CC2
:102180002D2D2D2D2D2D2D2D2D2D1C2D2D2D2D2D90
:102190002D2D2D2D2D2D2D2905F02EF815E0DF49A3
:1021A0000022184601F07AFD0FE00020019003CADA
:1021B00008A201AB01F090FE012806D1019805F0BC
:1021C00035F902E0024801210172002002B010BD81
:1021D000389901022B51495552433A2022636C6FC2
:1021E000736564222C25640D0A000000B0B5022935
:1021F0004AD30F2914D18568002004F0F7FB012889
:1022000003D10020032104F0F9FB0024204604F050
:10221000E5FB012806D1D94830301E49002231E0C3
:102220000120B0BD2846FFF76DFD00282CD004F03A
:10223000EFFB012808D115498C60E86B4268CF4B51
:10224000DA6252684A601CE0022004F0C7FB0128F1
:1022500009D10E498C61E86B4268C84BDA6252685A
:102260004A6110310DE0022004F0C0FB01280BD1BF
:1022700006498C62E86B4268C04BDA6252684A6277
:102280002031224601F00AFD0020B0BD509001022D
:10229000389901026826010080B5022905D3042976
:1022A00005D19E49002201F0F9FC002080BD0120EB
:1022B00080BDC046B0B50546881E02280AD3A8686E
:1022C000012913D0002915D10C490DA201F08CFA77
:1022D0000020B0BD0220032104F090FB0649002439
:1022E0002846224601F0DAFC2046B0BD01F0B6FADD
:1022F0000020B0BD0120B0BD882601008813000079
:1023000041542B4346554E3D310D0A0010B50F295F
:102310000BD001291DD000291DD1FFF7C1FD0020E0
:10232000022104F06BFB002010BD0446002004F0E5
:1023300055FB012803D10020022104F05FFB00209F
:1023400004F054FB012804D104490022204601F086
:10235000A5FC002010BD012010BDC046782601005C
:10236000F0B581B00124322928D805468768786BFA
:102370000668C0467944097949008F442F3F1919EE
:10238000191F1F1F1F1F1F1F1F1F221F1F1F1F1F60
:102390001F1F1F1F1F1F1F1F1F1F1F1F1F1F1F1F4D
:1023A0001F1F1F1F1F1F1F1F1F1F1F1F1F1F260055
:1023B0001E4900242846224601F070FC204601B048
:1023C000F0BD1B48017800291FD018490024284679
:1023D000224601F063FC204601B0F0BD0024FC62FF
:1023E0003969384688470028FAD011480470FC62E1
:1023F000FFF756FD0E20009001220EE0304601F05E
:102400009DFC0024204601B0F0BD01210170FFF7C2
:1024100051FD0E20009000240522304621462B4617
:1024200001F02CFC204601B0F0BDC046082601009A
:10243000E49A010210B586B0034601203B2900D979
:1024400056E0C0467944097949008F4450505151B3
:10245000335151515151515151515151515151518A
:10246000515151515151515151515151515151515C
:10247000515151515151515151515151515151514C
:1024800051391D1D1D1D1D1D0020059003CA02AAE6
:10249000009218A205AB01F01FFD022827D1039A74
:1024A000029817A1FDF7A8FE002820D1059804F096
:1024B000BDFF1CE0B5490022184601F0EFFB16E015
:1024C000002002900590049003CA05AA019204AA74
:1024D00000920DA202AB01F0FFFC032807D1049A81
:1024E0000599029805F06AF8029804F0E3FF0020CD
:1024F00006B010BD25642C2025700D0A00000000D8
:10250000434C4F53454400002B52454345495645E3
:102510002C25642C25643A0D0A25650058260100F7
:10252000012901D80020704701207047B0B5054649
:10253000881E03280BD2104604F072FA0F48C16AB5
:1025400000242846224601F0A9FB2046B0BDAC6815
:1025500001290BD000290ED104F03CFA03460849AA
:1025600008A2204601F040F90020B0BD204601F04D
:1025700075F90020B0BD0120B0BDC04638990102F8
:102580008813000025730D0A0000000070B582B0AA
:1025900001240F293DD803468568686B0668C0464C
:1025A0007944097949008F4407141E343434342F98
:1025B000373434343434434E664800240470846124
:1025C000C461012101716649664A284601F00CF98F
:1025D0001FE0284601F042F9304601F0AFFB00242D
:1025E000204602B070BD5B4800240471826904215A
:1025F00011430278002A2ED0052958D1016A491CBE
:10260000016259D2624961E0524B187800240028D7
:1026100031D0204602B070BD4E4B1878012816D13B
:1026200003CA183351A201F057FC002002B070BD5C
:10263000484800248461012101710078484900283C
:1026400012D1484A11E0434E307900281BD00024B3
:10265000204602B070BD052932D10024012101704D
:102660008461C46101713E493F4A284601F0BCF8CB
:10267000204602B070BD03CA183340A201F02CFC02
:10268000204602B070BD002004F0B0F9012803D14B
:102690000020032104F0B2F90024204604F09EF942
:1026A000012816D130362D49002430464BE0002158
:1026B0000162C169491CC1610E20009000241CE028
:1026C000C169491CC161652915D3304900241846E8
:1026D00039E02846FFF716FB00289AD004F098F955
:1026E000012812D11C4900248C60E86B4268F26218
:1026F00052684A6027E00E200090022230462146B0
:1027000001F0BCFA204602B070BD022004F066F968
:10271000012809D1104900248C61E86B4268F262FB
:1027200052684A6110310EE0022004F05FF901287E
:1027300000D06EE7084900248C62E86B4268F262C0
:1027400052684A622031224601F0A8FA204602B0BF
:1027500070BDC04638990102509001026826010000
:10276000881300001A3A0100253A01002B43475212
:1027700045473A20252A2C25640000002B4352456A
:10278000473A20252A2C2564000000005826010025
:1027900018260100B0B584B001243B2900D937E0E8
:1027A000134605468068C0467944097949008F443C
:1027B0004B5532322F2F2F2F2F2F2F2F2F2F2F2FE1
:1027C0002F2F2F2F2F2F2F2F2F2F2F2F2F2F2F2F19
:1027D0002F2F2F2F2F2F2F2F2F2F2F2F2F2F2F2F09
:1027E0002F2F2F2F2F2F1D1D1D1D1D1D0024039466
:1027F00003CB01AA00921C4A03AB01F06DFB022837
:1028000006D1029A019819A1FDF7F6FC00280FD015
:10281000204604B0B0BD1848006804F007FE174910
:1028200000242846224601F039FA204604B0B0BD03
:102830001148006804F0FAFD10490022284601F012
:102840002DFA204604B0B0BD0B490B601E210CA22E
:1028500000F0CAFF0024204604B0B0BD00F0FEFF27
:102860000024204604B0B0BD7E3B0100434C4F53D2
:1028700045204F4B00000000E89A01022826010085
:1028800041542B434950434C4F53453D25640D0A59
:1028900000000000F0B589B0044601203B2900D9B2
:1028A000AAE01646A7687A6B1568C046794409798C
:1028B00049008F44536AA071A1A1A1A1A1A1A1A126
:1028C000A1A18AA1A1A1A1A1A1A1A1A1A1A1A1A10F
:1028D000A1A1A1A1A1A1A1A1A1A1A1A1A1A1A1A1E8
:1028E000A1A1A1A1A1A1A1A1A1A11D1D1D1D1D1DF0
:1028F0000027089703CE06AA0092414A08AB01F0D0
:10290000EBFA022877D13F4805680898854272D1D2
:10291000079A069E3CA130460592FDF76DFC002803
:1029200047D03DA13046059AFDF766FC002840D00F
:102930003CA13046059AFDF75FFC0028314E5AD184
:10294000284604F08DFD7068401C706003283CD35D
:1029500003207060306804F00BFD36E02948066003
:10296000304604F059FD05902648006804F028FD23
:1029700004902448006804F02FFD0499019102900E
:102980000598012827D02EA026E0384600F066FFE3
:10299000284601F0D3F92EE01A4D286804F060FDB6
:1029A0006868401C686003280FD300226A602249CF
:1029B0000DE0144E7760284604F068FD306804F09E
:1029C000A3FE002801D01B4900E00C49002220464C
:1029D00001F064F90FE019A000901A491AA23846D4
:1029E000334600F001FF0E2000900021B42228465B
:1029F000234601F043F9002009B0F0BD282601006C
:102A00007E3B0100A4970102414C524541445920AC
:102A1000434F4E4E45435400434F4E4E4543542082
:102A20004F4B0000434F4E4E454354204641494CC6
:102A300000000000C8260100E825010054435000B2
:102A4000554450008813000041542B4349505354BF
:102A50004152543D25642C222573222C22257322B9
:102A60002C25750D0A000000B0B582B014468A1EF0
:102A7000022A12D38568012917D000291CD12046CB
:102A800004F090FC00901E210EA22846234600F080
:102A9000ABFE0024204602B0B0BD09490024224606
:102AA00001F0FCF8204602B0B0BD284600F0D6FE8A
:102AB0000024204602B0B0BD0124204602B0B0BDC3
:102AC000D826010041545E4845415254434F4E467A
:102AD00049473D312C25642C25750D0A0000000066
:102AE000F0B583B014468A1E022A1CD385680129DA
:102AF00021D0002926D1164F3C60204604F044FC2A
:102B0000FDF766FB0646386804F03EFC710800914C
:102B100001901E210FA22846234600F065FE0024E6
:102B2000204603B0F0BD09490024224601F0B6F862
:102B3000204603B0F0BD284600F090FE0024204659
:102B400003B0F0BD0124204603B0F0BD28260100EB
:102B5000EC9A010241545E48454152544245415469
:102B60004845583D25642C25752C25730D0A000019
:102B7000F0B585B0044601203B2900D988E0A5685E
:102B80007944097949008F444257825E8383838365
:102B90008383838383838383638383838383838325
:102BA00083838383838383838383838383838383F5
:102BB00083838383838383838383838383831D1DB1
:102BC0001D1D1D1D0020049003CA02AA0092314A57
:102BD00004AB01F081F9022859D12F488568049887
:102BE000854254D1039E029F2CA138463246FDF700
:102BF00003FB00283DD02BA138463246FDF7FCFAF6
:102C0000002844D1284604F011FC29493BE0224C1D
:102C1000A260104604F0ECFB002838D001F0C5FAA1
:102C2000E060002833D0A36840680090234924A2C4
:102C3000284600F0D9FD2AE017480021C160284647
:102C400000F00CFE23E01448806804F0EFFB19E06C
:102C500000F074FE012804D10F48C16803C900F0D8
:102C600075FF0D48C0680CC81349284600F0FCFDEC
:102C70000DE0284604F0BCFB0028074907D0C968CE
:102C800001F069FA0B490022204601F007F8002004
:102C900005B0F0BD7E3B0100A497010253454E44B0
:102CA000204F4B0053454E44204641494C00000004
:102CB0005826010028260100204E0000881300003D
:102CC00041542B43495053454E443D25642C2575B2
:102CD0000D0A0000F0B583B0074601F063F8002646
:102CE000304604F08FFB032835460BD104212846DB
:102CF00004F0FAFCF86B51492A4600F0CFFF304649
:102D000003B0F0BD02970024204604F07BFB0428AA
:102D1000254609D10298C06B49492A4600F0BEFFFA
:102D20002646304603B0F0BD0027384604F06AFB63
:102D300005283D4609D10298C06B40492A4600F05B
:102D4000ADFF3E46304603B0F0BD01970125284651
:102D500004F058FB0328029FC8D00125284604F040
:102D600051FB0428D6D00125284604F04BFB05284A
:102D7000019FE0D00225284604F044FB0328029F6F
:102D8000B4D00225284604F03DFB0428C2D0022519
:102D9000284604F037FB0528019FCCD0254C20683D
:102DA000401C0321FDF7ACF90D46084604F02AFB50
:102DB0000628029F08D1284604F01AFB002803D0F9
:102DC00001F0F3F900282AD1681C0321FDF798F9D6
:102DD0000D46084604F016FB062808D1284604F0E4
:102DE00007FB002803D001F0E0F9002817D1681C88
:102DF0000321FDF785F90D46084604F003FB002189
:102E0000CE43062800D07AE7284604F0F1FA0028DD
:102E100000D174E701F0C9F9002800D16FE72560FF
:102E2000F86B05492A4600F039FF0026304603B00A
:102E3000F0BDC046F09A0102E8260100A826010074
:102E4000B8260100B0B582B001220F293ED8034652
:102E50008068446B2468C0467944097949008F44EE
:102E6000071F2527343535353535353535350A15C0
:102E70002749002204E02649CA68092A20D8521CA2
:102E8000CA601649164A00F0AFFC1EE0002003F0AD
:102E9000A5FD012819D11E4830300E49002212E04C
:102EA00000F0DCFC204600F049FF0EE00D4908E090
:102EB0000E20009000210122204600F0DFFE04E0F9
:102EC00005490022184600F0E9FE0022104602B033
:102ED000B0BDC046682601004826010088130000E6
:102EE000313A0100F825010080B5032005F00CF906
:102EF00080BD00000648416B0020002905D0054A2E
:102F0000914203D049680029FAD1704701207047E7
:102F10003899010238260100B0B514460D4608461E
:102F2000114600F0C0FF01281ED1285D00281BD1EA
:102F3000002C0FD06019401E00780A280AD17B4867
:102F40000078002810D003200A4A01462B460DF0D5
:102F500009F809E075480078002805D00320054AE3
:102F600001462B460CF0FEFF03202946224605F0C1
:102F7000B7F9B0BDC7390100F0B585B0054604A862
:102F800000240470E743002D12D0EA68002A0FD015
:102F9000686A00280CD0A86A002809D0401EE96A97
:102FA000814200D38EE004A928469047002803D030
:102FB0003C46204605B0F0BD564EE86A411CE96229
:102FC000696A049A0A54E86A696A002202920A54F9
:102FD000E86A092806D1696A09224D48FDF7FFF819
:102FE00000283ED03078411E022908D800F0DAFED1
:102FF000B168401A4849884264D8464E30780A2859
:1030000020D0012823D16E6A3A213046FDF7D6F848
:10301000002847D0019002980390E96A03AB30463C
:103020003EA200F059FF02284CD10398002849D055
:103030000A21384A117001990818696A401AC01C9F
:1030400050602FE07068E96A81422BD13AE004A811
:1030500000780A280FD00D2814D101202863E86ACF
:103060001AE00120307000F09DFEB0603078411E03
:103070000229BBD9C3E7296B012904D102202863A7
:10308000E86A03E0296BE86A022905D1022817D112
:103090000298E862286305E0012803D1686A007895
:1030A0003E280FD0A86AE96A401E81420AD2EA6827
:1030B00004A9284690470028164E00D17DE777E7FF
:1030C00002982863E96A686A00F0EDFE012819D1C8
:1030D000E86A00280CD06B6AC018401E00780A28E5
:1030E00006D11248007800280CD0032010A206E078
:1030F0000E480078002805D06B6A032010A2014614
:103100000CF030FF03480470204605B0F0BDC04607
:103110000A3301002C970102DC0500002B524543C5
:10312000454956452C252A2C25643A009F990102D1
:103130005B415420526563765D20257300000000DA
:103140005B415420526563765D2025730D0A0000B3
:1031500010B5064C2078002108F0BCFC044806F0AD
:1031600061FD2078012108F0B5FC10BDB696010282
:1031700060E31600B0B50F2001F0DEFB194D68705A
:10318000287033282AD120243721204601F020FC42
:103190002120032101F01CFC2220402101F018FC19
:1031A0002320082101F014FC3020AA2101F010FC9A
:1031B000A24802210187322001F00AFC33200121BC
:1031C00001F006FC5F21204601F002FC0F2001F017
:1031D000B3FB28700A2006F025FDB0BD97480021FA
:1031E000C187B0BD04960102F0B581B0364C2121F3
:1031F00000916172354909886170354F7A89627131
:10320000FD6AFD61334B1B782370090AA170110A16
:10321000A171B978814207D10AF098FE6421FCF7C8
:1032200059FFB981B978FD6A2B4848432B494018AA
:103230000A21FCF74FFF45193D630AF01DFE4019B6
:103240000BF076FA06460D462548007D0BF0FCF89B
:10325000244909882222A15482B2D20B801802B2DA
:10326000D0175210B2186841130E009D6355130C0D
:1032700020256355BB6DA3761D0AE5761D0C2577C9
:103280001B0E637723462233090A5970A2773A65E9
:1032900078653A667866100AE0770AF057FE386279
:1032A0003B6B2821012220460EF0F4F80AF04EFE76
:1032B000B86109F017F80028FBD1042008F0CAFB18
:1032C000002001B0F0BDC0461ED40102C499010225
:1032D000D09801029E990102800A1B0040C20C0096
:1032E00038900102AA99010270477047F0B587B083
:1032F0004F480068FDF71AFB04460D464D48406AEA
:10330000FDF7C6FB02460B4620462946FDF712FA9A
:1033100002460B46002448492046FDF795F90490E3
:10332000039106204549085EFDF700FB01900091DE
:103330000120069040020290414F05E04F4908519C
:103340007F1C241D642C70D0387805283D48F5D1A9
:1033500005973D4801593D4E31613D480359B360E1
:103360003C480059B0613C4A1259326200275D1A4C
:1033700035637369F1689941069B00DB3B46002B7E
:1033800001D0029BC918314E7163F369716A101A3A
:103390009941069A00DB3A46002A01D0029A891820
:1033A000FDF7E6FA02460B4604980399FDF75AF931
:1033B000FDF746FB254A9062D162401BC10F4018C1
:1033C000401010601546FDF7B1FA244A244BFDF772
:1033D00049F9A863E963234A234BFDF743F93A46C9
:1033E000224BFDF73FF93A46214BFDF789F8054698
:1033F0000E4616480564416428463A461D4BFDF7C3
:1034000057FA0028059F9BD10022284631461A4BC7
:10341000FDF764FA002893D128463146019A009BB3
:10342000FDF76EF8FDF7E8FA88E707B0F0BDC04693
:10343000F8960102E42001000000F03F4AA90102D1
:1034400008980102FFFF0100AC9F010218960102DB
:1034500010A001020CE0010270E00102699006690F
:103460009006903F52257997532ED33F0000594044
:1034700000003E4000408FC0006AF84038D2010290
:10348000B0B582B0194C2068056801A90020087009
:1034900007E090470198401C01A90870C0B20828B5
:1034A00022D2012211048140294209D022685160B0
:1034B00080002018826A002AECD001A80121E8E7E8
:1034C000130283402B4201D0022104E082402A42B1
:1034D000E0D00321134622685360800020188268E0
:1034E000002AD7D001A8D4E702B0B0BDD49201021F
:1034F000FEE7000010B509480168CA69202313439C
:10350000CB610269032A08D1012293050C689C4310
:103510000C605102C26E0A43C26610BD489301029C
:1035200081B010B581B00393002807D0C16A00298B
:1035300004D003AB0093C46A0021A04701B010BCC3
:1035400001BC01B00047000080B502460848006891
:10355000002807D091B2120C03889A4203D0406928
:103560000028F9D180BD002200F0F4FA80BDC046E9
:103570006CC90102F0B581B05C4C2068856BE8072E
:1035800007D0E168002904D0002088472068012185
:103590008163A80707D52169002904D00120884745
:1035A000206802218163680707D56169002904D07A
:1035B00002208847206804218163280707D5A16974
:1035C000002904D003208847206808218163E80689
:1035D00007D5E169002904D004208847206810211C
:1035E0008163A80607D5216A002904D005208847F1
:1035F000206820218163680607D5616A002904D00C
:1036000006208847206840218163280607D5A16AE3
:10361000002904D007208847206880218163012683
:10362000E80507D5E16A002904D037020820884759
:1036300020688763A80507D5216B002904D077028D
:103640000920884720688763680507D5616B0029D2
:1036500004D0B7020A20884720688763280507D569
:10366000A16B002904D0F7020B20884720688763EC
:10367000E80407D5E16B002904D037030C20884704
:1036800020688763A80407D5216C002904D077033C
:103690000D20884720688763680407D5616C00297E
:1036A00004D0B7030E20884720688763280407D515
:1036B000A16C002904D0F7030F2088472068876396
:1036C000E80307D5E16C002904D0370410208847AF
:1036D00020688763A80307D5216D002904D07504ED
:1036E000112088472068856301B0F0BDD89301029E
:1036F00002480068411E88417047C046B8990102DF
:10370000F0B58DB0002862D00446406800285ED035
:10371000A06840285BD8E56A002D58D007462046AF
:1037200040300026039003E0019E4AE0039848E001
:10373000402101220691FCF72FFDAE4202963ED2B7
:1037400000203146019009900398069B3E46002ECA
:10375000EAD0606A0491405C07900998401C05908B
:103760000021042708916518EA5C012A17D10A96FE
:103770006268D3191B1F1B68099E9E5D07988642CD
:1037800008D1059D5B5D002B0A9E22D00898401C45
:10379000089003E0403500222A70A668069B08378F
:1037A000491CB142DFD308980028BFD00499491CB6
:1037B000E06A8142059809900398C8D301E0039814
:1037C0003E463746E56A029E761CAE42B0D30DB047
:1037D000F0BD616A0B91E16A0C91D1590BAA2046A8
:1037E00000F09CF80DB0F0BD81B0B0B583B00D46CF
:1037F0000446079307AB02938069E1690DF0C4FEAC
:10380000206265480078002803D1216AA06900F091
:103810009FF96369A169226A204698470146A06B17
:10382000002905D069460C600021224B0A460CE0B5
:1038300000F084FA7D2081002846FCF74BFC02460C
:10384000A06B69460C6000211B4B00F0D3FA0020EE
:1038500003B0B0BC02BC01B00847C04680B5806B65
:1038600000F06CFA002080BD70B582B00D460446B1
:10387000466911461A46B0470146A06B002907D099
:1038800069460C6000210B4B0A4600F0B3FA0EE0CB
:1038900000F054FA7D2081002846FCF71BFC02460C
:1038A000A06B69460C600021034B00F0A3FA0020D6
:1038B00002B070BDA1390000B739000070B50D46E7
:1038C0000446802100F0C0FA2868E0636868606000
:1038D000A868A060E868E0602869206168696061A4
:1038E000A869A061E86900262662E061286A606232
:1038F000686A2663E662A062A86A60632046383080
:1039000000F02AFA002802D0F643304670BD214864
:10391000016821600460304670BDC04670B5144631
:103920000D460646881E032802D8B06B00F006FA42
:10393000F06B2946224600F00DF970BD164801785B
:10394000012048407047C04670B512480468002CFA
:103950001FD0114E11A5216920468847002815D196
:10396000307800280DD1E16A606A00F09CFA0146C7
:10397000606A012903D0E16A00F0E8F8284600F007
:10398000E3F82046FFF7BCFE0020E0622468002C2C
:10399000E1D170BD68C9010260C901020D0A0000D1
:1039A00010B50446806B00F0C9F9E06B05210022D8
:1039B00000F0D0F810BD10B50446806B00F0BEF9E1
:1039C000E06B0421002200F0C5F810BDF0B581B015
:1039D00000910646C7680468A01C3946FCF77AFBCC
:1039E00000257068814201D1ED430BE0601C39462F
:1039F000FCF770FB316032695143B06808180099D8
:103A0000FCF7B8FB284601B0F0BDB0B50124002595
:103A10000560446008300EC0B0BD70B50E46044667
:103A2000C1680068401CFCF755FB002560688142B6
:103A300002D1ED43284670BD22695043A168411868
:103A40003046FCF797FBE1686068401CFCF742FBDE
:103A50006160284670BDB0B5002400280DD0054631
:103A600000688842FDD3401A286068684018E968F9
:103A7000FCF730FB69602046B0BDE4432046B0BD92
:103A8000B0B5002400280ED0054600684018286014
:103A9000EA689042FDD8A86840181146FCF71AFB66
:103AA000A9602046B0BDE4432046B0BDF0B583B068
:103AB000164602460027F843002E22D01C46002B53
:103AC0001FD00D46D168136899421AD9CB1AAB4260
:103AD00017D39268019252198A423A4607D9019A3D
:103AE0008A1A0292029A52199342029A09D30292B6
:103AF00001981018FCF7EEFA316002984019206026
:103B0000384603B0F0BD4068704780687047024691
:103B10000020002A04D0106050609060D16070478F
:103B2000C0437047002803D00168484248417047AD
:103B300001207047002805D00168C068411A48423A
:103B400048417047012070470020704700207047AF
:103B500000207047F0B583B014460D4606464088F5
:103B6000012818D1306900280CD0A90040580178EC
:103B70002D2910D0F368716809686A461160506099
:103B800010A205E0F36870680068694621C115A2BB
:103B90003046FFF7C5FC7768FB6830462946224669
:103BA0009847012808D00AE0C368304629462246D3
:103BB00098477F68012802D178680028F4D103B0C3
:103BC000F0BDC04646534D3A252D3873205354411D
:103BD00054453A252D323873204556454E543A25E2
:103BE000730D0A0046534D3A252D38732053544126
:103BF00054453A252D323873204556454E543A25C2
:103C0000750D0A00F0B581B0002828D01E460C467C
:103C10000546079B0698009000206862A862E8624B
:103C2000104909886B8029800F4B1F686C60009BCE
:103C3000AB602B460C33C4C3A861E8612862481C02
:103C40000849088008480560002C08D06C600021F5
:103C500028460A46FFF77EFFA468002CF6D101B083
:103C6000F0BDC046F0CC01026CC901020246002042
:103C7000002A01D0D1627047C043704710B582B0AE
:103C800004AC24881B881B041B196C462360024B60
:103C900000F0B0F802B010BD49350000F0B597B0A3
:103CA0001646029105464268002A30D001966A60A5
:103CB00001210024284616462246FFF74BFF3046D6
:103CC000029FBE4232D003A85021FCF76CFA324664
:103CD0007268002F0CD003AF029811C74068083FEC
:103CE000824209D0394608313C4600280F46F4D1BB
:103CF000002A019EDBD10AE0019E3868686000213D
:103D000028463246FFF726FF7F68002FF5D102983C
:103D10008468002C08D06C60002128463246FFF7EA
:103D200019FFA468002CF6D117B0F0BD0021284679
:103D3000019E3246FFF70EFFE9E700000146002032
:103D40001F2901D9C043704718224A43344901232F
:103D50008B5089188860704710B50021CC4300282B
:103D60000BD00A4A1368002B09D01832491C2029AD
:103D7000F8D306D106A0FFF7E7FE204610BD0123C9
:103D8000136001600024204610BDC046F0C9010246
:103D900074696D65722049442069732066756C6C86
:103DA0000D0A0000264800687047C04670B5202400
:103DB0001B4D234E2868022817D13068A968EA688D
:103DC000401A904211D96969002907D02879002842
:103DD00007D0022028603068A86004E00120286035
:103DE00003E001202860286988471835641EE1D166
:103DF00070BDC046F0B5044600201F2C01D9C04359
:103E0000F0BD059D18266643054C0227A751A4194D
:103E100021710B4909682646083626C66361F0BD44
:103E2000F0C9010206480168491C01600548416863
:103E300002680023521C02604B4143607047C04639
:103E4000A4AD0102A8AD010280B5FCF7ACF980BDBC
:103E5000B0B50278002A24D0441C0021084601E0B5
:103E6000573A08E023460001D5B2302D0C4611D355
:103E7000392D02D8303A14460CE0412D0C4609D3B6
:103E8000462D01D8373AF6E71446613CE4B2062CD9
:103E9000E6D30024E2B280185C1C1A78002AE1D133
:103EA000B0BD0020B0BD10B50246012000290DD0E4
:103EB0000023D45C202C02D37F2C04D307E00D2CEC
:103EC00001D00A2C05D15B1C8B42F2D310BD00201F
:103ED00010BD002010BD000081B0F0B584B0099382
:103EE00000230393002800D1C2E0002A00D1BFE0E4
:103EF00009AB03931678002E00D1A8E05623DB43CC
:103F0000009300231D46002900D1A2E0252E3FD1B9
:103F1000971C52781446643C0023142C43D8C046A6
:103F20007C4424796400A7440A99A3A3A3A3A3A370
:103F3000A3A3A3A34CA3A3A3A3A3A3A35F0002973C
:103F4000039A131D0393126801920122002317465E
:103F50001E460478FF0703D02D2C01D1164607E03A
:103F60002746303F092F09D80A275F433B19303BCA
:103F7000491E401C00270029EBD13946029A019CBA
:103F8000002C03D0012E00D15B4223606B1C06E0A5
:103F90000378B3425BD1491E521C401C2B46167855
:103FA000002EAFD164E02A2A62D13A780378934296
:103FB00004D0491E401C0029F8D100216B1C3A4650
:103FC000EDE7039A131D03933E7812680023C45C47
:103FD000B44233D0491E5B1C0029F8D13C46C718B7
:103FE0000021002A2ED12EE00297039A131D03937D
:103FF00012680023009E0778302F18D33A2F02D280
:10400000344627340BE0612F03D3672F344606D3A1
:104010000DE03C46413C052C09D8344620341B01B8
:104020001B19DB19491E401C0029E4D10021029C08
:10403000002A00D013606B1C2246B0E73C46C7182C
:10404000002A00D009C26B1C22463846A7E700238D
:104050000EE0252E0BD15178652908D103990A1D50
:1040600003920968002900D008606B1C00E02B4611
:10407000184604B0F0BC02BC01B0084781B010B5CE
:1040800081B00C46039303AB00930DF07DFAA04280
:1040900000D3601E01B010BC02BC01B0084770B56F
:1040A00004460020002A1BD0002C19D0002B17D06A
:1040B00014600120022B13D32578002D10D0641C2E
:1040C00001208D4205D1651E00262E7085005451B9
:1040D000401C984204D2661C2578002D3446F0D14D
:1040E00070BDB0B504467821FCF768F8002805D10A
:1040F00058212046FCF762F8002828D04278002A90
:1041000023D0841C0021084623460001D5B2302D5F
:104110000C4613D3392D01D8303A0EE0412D0C4610
:104120000CD3462D01D8373A07E01446613CE4B27F
:10413000062C01D3002401E0573A1446E2B280185D
:104140005C1C1A78002ADFD1B0BD0020B0BD20462B
:10415000FCF7F4F8B0BD70B504460026F043002C1F
:104160000DD00D4600290AD0204610300121FFF75E
:1041700072FCA96820342046FFF76DFC304670BD04
:1041800070B504460026F043002C0DD00D460029E2
:104190000AD0204610300121FFF772FCA9682034B4
:1041A0002046FFF76DFC304670BD70B50024002836
:1041B00014D00546064610363046FFF7B3FC0128FA
:1041C0000CD028462030FFF7ADFC012806D02C6823
:1041D0003046FFF798FC0C2141436418204670BD1F
:1041E000F0B583B000250295019500281FD00C463C
:1041F0000646074610373846FFF79CFC002816D1C4
:104200003046203002AA01AB2146FFF74FFC0028C0
:104210000DD135683846FFF778FC0C214143B06872
:10422000029A101868506D186C600198A8602846B2
:1042300003B0F0BD70B505460C20584300249042F1
:1042400011D2121A461829606860AE60EA602846EA
:1042500010301946FFF75BFCE96820352846FFF768
:1042600056FC204670BDE443204670BD04217046D4
:10427000084204D0EFF30983EFF3088203E0EFF381
:104280000883EFF309829BB004A8F0C044464D4672
:1042900056465F4608A8F0C01846F0C86846F0C009
:1042A00018690C90202018440D9058690E90986958
:1042B0000F90D8691090EFF310801190EFF31480F5
:1042C0001290094908681390084908681490084931
:1042D0000868159007490868169017931892704659
:1042E000199068460AF0FCFF04ED00E00CED00E0D8
:1042F00010ED00E014ED00E0F0B581B003260024DD
:104300003046214607F02AFC04252846214607F0BE
:1043100025FC0127304639463A4607F0B3FB3046C4
:104320002146324607F042FC284639463A4607F015
:10433000A9FB02212846224607F038FC01B0F0BD57
:10434000F0B589B008900425284607F083FB0A27BA
:10435000384605F067FC284607F08CFB032420460E
:1043600007F080FB07900526304605F05BFC2846E9
:1043700007F070FB384605F055FC284607F07AFB3D
:10438000204607F06FFB0690304605F04BFC2846B0
:1043900007F060FB384605F045FC284607F06AFB4D
:1043A000204607F05FFB0590304605F03BFC2846B1
:1043B00007F050FB384605F035FC284607F05AFB5D
:1043C000204607F04FFB0490304605F02BFC2846B2
:1043D00007F040FB384605F025FC284607F04AFB6D
:1043E000204607F03FFB0390304605F01BFC2846B3
:1043F00007F030FB3846019705F014FC284607F01B
:1044000039FB204607F02EFB0290304605F00AFCEF
:10441000284607F01FFB384605F004FC284607F045
:1044200029FB204607F01EFB0746304605F0FAFB45
:10443000284607F00FFB019805F0F4FB284607F02B
:1044400019FB204607F00EFB0446304605F0EAFB58
:10445000284607F0FFFA0699481E81410A46079947
:10446000481E8141480080188000059A511E8A41EB
:1044700051004018049A511E8A4180188000039A06
:10448000511E8A4151004018029A511E8A418018DB
:104490008000791E8F4179004018611E8C410619F9
:1044A0000898002803D0032007F0D4FA02E0032084
:1044B00007F0E0FA0A24204605F0B4FB042528465C
:1044C00007F0D8FA204605F0ADFB284607F0C2FAFF
:1044D000F0B209B0F0BD70B50446042007F0BAFA96
:1044E00060B2002803D4032007F0B4FA02E00320EE
:1044F00007F0C0FA0A25284605F094FB042630464A
:1045000007F0B8FA284605F08DFB304607F0A2FA0E
:10451000284605F087FB600603D4032007F09AFACB
:1045200002E0032007F0A6FA0A25284605F07AFBE8
:104530000426304607F09EFA284605F073FB304605
:1045400007F088FA284605F06DFBA00603D4032087
:1045500007F080FA02E0032007F08CFA0A252846CB
:1045600005F060FB0426304607F084FA284605F083
:1045700059FB304607F06EFA284605F053FBE0067B
:1045800003D4032007F066FA02E0032007F072FA72
:104590000A25284605F046FB0426304607F06AFA4D
:1045A000284605F03FFB304607F054FA284605F050
:1045B00039FB200703D4032007F04CFA02E0032064
:1045C00007F058FA0A25284605F02CFB0426304649
:1045D00007F050FA284605F025FB304607F03AFA76
:1045E000284605F01FFB600703D4032007F032FACA
:1045F00002E0032007F03EFA0A25284605F012FBE8
:104600000426304607F036FA284605F00BFB304604
:1046100007F020FA284605F005FBA00703D4032085
:1046200007F018FA02E0032007F024FA0A252846CA
:1046300005F0F8FA0426304607F01CFA284605F083
:10464000F1FA304607F006FA284605F0EBFAE007E3
:1046500003D1032007F0FEF902E0032007F00AFA75
:104660000A24204605F0DEFA0425284607F002FA5F
:10467000204605F0D7FA284607F0ECF9204605F069
:10468000D1FA70BDF0B581B0032600250124304673
:104690002946224607F0F6F9304607F0EBF90626E0
:1046A000304605F0BFFA042007F0E4F9304605F083
:1046B000B9FA032007F0D6F900281BD0681CFA2DA0
:1046C0000546F6D30425284607F0C4F903263046EC
:1046D00007F0C0F90A27384605F0A4FA284607F083
:1046E000C9F9304607F0C6F9384605F09BFA20466E
:1046F00001B0F0BD032001210A4607F0C3F90420F0
:1047000007F0A8F90024204601B0F0BDB0B504467A
:10471000C00703D1032007F09DF902E0032007F052
:10472000A9F90825284607F0A5F9284607F092F9C7
:10473000A00703D4032007F08DF902E0032007F05F
:1047400099F90825284607F095F9284607F082F9D7
:10475000600703D4032007F07DF902E0032007F08F
:1047600089F90825284607F085F9284607F072F9E7
:10477000200703D4032007F06DF902E0032007F0BF
:1047800079F90825284607F075F9284607F062F9F7
:10479000E00603D4032007F05DF902E0032007F0F0
:1047A00069F90825284607F065F9284607F052F907
:1047B000A00603D4032007F04DF902E0032007F020
:1047C00059F90825284607F055F9284607F042F917
:1047D000600603D4032007F03DF902E0032007F050
:1047E00049F90825284607F045F9284607F032F927
:1047F00060B2002803D4032007F02CF902E0032064
:1048000007F038F90824204607F034F9204607F06D
:1048100021F90724204607F02DF9204607F01AF960
:10482000B0BDF0B581B0032700243846214607F01B
:1048300085F93846214607F091F901253846294681
:10484000224607F01FF9052638462946324607F06A
:10485000ADF908273846214607F080F93846294641
:10486000224607F00FF938462946324607F09EF9EE
:1048700007273846214607F071F93846294622466F
:1048800007F000F938462946324607F08FF901B0A3
:10489000F0BD000080B50B2007F0E4F812490A785B
:1048A000002804D0002A12D003F050FB80BD012A5A
:1048B000FAD1002008700F49C8830C4908700C48D1
:1048C000012101700BF08AFC03F040FB80BD07481A
:1048D000012202700A700648002101700BF09EFC54
:1048E00003F034FB80BDC0461C9001021890010209
:1048F000199001024AA9010202484069811E4842FA
:10490000484170477096010280B5FDF759FA0028BA
:1049100001D00020C04380BD80B5FEF7EBFA80BD1A
:1049200010B504480F2100242246FFF713F9204652
:1049300010BDC04668990102F0B581B00746032456
:10494000204607F097F80425284607F093F82046FC
:1049500007F080F80A26304605F064F9284607F08B
:1049600079F83220FFF7B7FDFFF78CFEF8B2FFF7BA
:10497000B2FDFFF787FE204607F07CF8284607F0D7
:1049800079F8204607F066F8304605F04BF92846DE
:1049900007F060F83320FFF79EFDFFF773FE00205D
:1049A000FFF7CEFC0746284607F054F8204607F0EC
:1049B00051F8304605F036F9284607F05BF82046F6
:1049C00007F058F8304605F02DF9384601B0F0BD33
:1049D000F0B581B0009107460324204607F04AF85D
:1049E0000426304607F046F8204607F033F80A253B
:1049F000284605F017F9304607F02CF83220FFF76B
:104A00006AFDFFF73FFEF8B2FFF765FDFFF73AFEDC
:104A10000098FFF760FDFFF735FE304607F01AF803
:104A2000204607F017F8284605F0FCF8304607F056
:104A300021F8204607F01EF8284605F0F3F828462E
:104A400005F0F0F801B0F0BD80B507480121017014
:104A5000064802680A43026005480268002A02D03C
:104A600000200146904780BDF6CC01021C1000508A
:104A7000F8CC0102F0B599B0F548017BC67A427BCB
:104A80000E92F44C221F1368F34A12680692427881
:104A90000C9202790592C76A04931F4001200F907F
:104AA0007A0200D5BCE03A0200D5BFE0FA0102D597
:104AB0000F9802062260502508968A191826BB0115
:104AC00002D50F98430623604123079569430A9650
:104AD000354655431426FC0210D50F980405384678
:104AE0003746DC4E3460DA4CA469B464D84CE469CF
:104AF0007464DA4C241D34603E46074690000B90E7
:104B0000D8040D90681809900E9B73430F98820388
:104B1000B902D04D22D50F9841052960CC480E9698
:104B20001646024681692965C169696509990D982A
:104B300001430898000108180B994018C018C8498B
:104B4000098892794A4380180A301C4605F04AFBCE
:104B5000234632460E9EC04988672A600F98C404D7
:104B6000380300D52C60F80302D50F9800042860A4
:104B70000F984104B80300D52960380400D4E4E15B
:104B8000039402910E9308920D980B990C180A98B1
:104B90000C9941430C910F98C0030B90286008F0CA
:104BA00067F9002801D005F0FFFA0C98005B410B73
:104BB00043D1099800190E99401805990901401828
:104BC0000E90E74D287B079B4343E97A0A010D9C31
:104BD0002243D21841188B00D2180A9B4B43D1189C
:104BE0006A7B564389190E9E2A791018DF4A12886B
:104BF0004243881816903068C000800D10A9C88202
:104C0000002511957079C0077ED110A80F99818277
:104C1000069C00940020E8A2049B0BF0A3F978E026
:104C20000F98820522603A0200D43FE70F98C20530
:104C30002260FA0100D53BE73DE707214903084020
:104C4000032149038842089A00D07EE1069707F0C5
:104C500071FD0020169009901590C14CE07A217BDF
:104C600008180A99414380000D9A10434118627B4D
:104C70000E9672438A186178A379079E7343D718FA
:104C8000FA683F26324063789A420C976ED10596B7
:104C90000A9A4A4380580F210A0702400398401E8F
:104CA000C04B1B68DB090340981810900F98C00296
:104CB0000B90B868800767D42C46283C0AF0C8F8E7
:104CC00005462068000609D5C3208401786A40079C
:104CD00004D40AF0BDF8401BA042F7D905980002A1
:104CE000B96849080140B34803688268B868C40CD1
:104CF00020202040DB0700D095E0002310221D4635
:104D00001C460E9E0B9FB1E010A88582B0681190E2
:104D1000069C701D924B1979E20707D1491C197145
:104D2000D97A1A798A4202D31D7100E0D9700178CC
:104D30004278120251188278120489180322914392
:104D4000017035715878401C5870D87A197B081852
:104D50005978884200D85D70D879401ED871596B57
:104D6000002901D010A888477E4DEDE010A80B99CE
:104D70008182F86830406378009000207CA20F990F
:104D80000BF0F0F80E9E94E0388A874A024010A893
:104D9000C2822022BA5C9307DB0F3C68C3720F9B70
:104DA0001A4082726205D20C0D9B1A431692FA6861
:104DB000130E0372BB69FC697C4D2D682D0C0574C4
:104DC0005204920F427211931394654CA07B0028F9
:104DD00009980E9E0B9F5FD075480068007A0328E3
:104DE000099859D00C98007D08400928099853D19A
:104DF000C32084010AF02CF805460C98406A41074C
:104E00000BD4594909680906890F06D10AF020F820
:104E1000401BA042F1D90C98406A4103089888438E
:104E200010A9888237E0D2070E9E0B9F03D108237A
:104E30000022154619E00C9B9A68029C224211D16F
:104E40009A68520C022494430022134615460DE042
:104E5000FCD1010228A000503CA10050FC1F000022
:104E6000F8D10102042500221346144608431043DA
:104E700018432843204310A9888238420BD10C9B49
:104E8000198A494A0A4010A9CA8219684905C90CF9
:104E90000D9A11431691324C2921615C002908D0EA
:104EA0003037B84205D010A908461130123109F048
:104EB000E1FAE77A2A48047BE519294800790E903F
:104EC00027484078401C2946FBF704F988000D9AD2
:104ED0001043189007996143380110434018204946
:104EE000497B4E4380191C21694340180E990919CA
:104EF0001B4B1E4A12884A4380181790099A0C9936
:104F00008A60987B002800D04A629879401C98718A
:104F1000187B99798142069F00D39A715978491C70
:104F20005970D97A0818597888420E4D00D85A70AD
:104F3000187A401E18722820185C002804D0996B3B
:104F4000002901D010A88847089A174202D00F986C
:104F5000000328601C480449486019B0F0BDC046F1
:104F6000FCD1010228A000503CA10050F8D1010260
:104F700048572045542069647820256420616E6478
:104F80002045542069647820256420696E20525899
:104F90002064657363206D69736D617463680D0AC5
:104FA0000000000038200040FF0300009430004063
:104FB00044940102604000404D4143204556542036
:104FC00025782025780D0A00FFFFFF03F0B5A5B076
:104FD0001E460C9208910024239422A90C8016A945
:104FE0000C8024A909250D80598C0D91FBF772F8CE
:104FF0002A99012900D0DFE03189012900D0DBE0C6
:10500000318C012900D0D7E00D99002900D1D3E0DF
:10501000224607962C990B912B99069180B2059008
:105020000F9415A8058090000E900C990C582E46F0
:105030000025204629461746FBF7F4FB0028119669
:1050400036D12C200A9778430899081817A90A46E0
:1050500068C868C2E8C8E8C2E8C8E8C2079F1198F3
:1050600080B280000E5822AD019523A80090204602
:105070003946059A069B04F0E3FD0F98401C0F90FB
:10508000288800282DD03B8A239913AC039416A8B6
:10509000029014A8019015AE009617A824AA04F057
:1050A000A9FF2588308811900120149E0A9A05E0F6
:1050B00013A8058014952E4628463A460E9F5100A7
:1050C0000B9B119C5C52591808830D84D81986607B
:1050D0000F981885521C0D9882426DD024A805881F
:1050E0009FE7099616A800250580149524A8068830
:1050F000239812902F46109503E06D1CA8B2B04281
:1051000013D8A8B2800017A90C5820461299FBF7B3
:1051100097FB0028F1D1002FEFD115A8058016A824
:105120000127078014941094E7E715A80288B01AA5
:10513000012805D115A80680099F1497119628E02B
:1051400010200799095E0129119221DB551CA8B294
:105150000C18109F0E9B099403E06D1CA8B28442AA
:1051600018DDAAB2B242F8D8800017AA10581090E1
:10517000394634461E46FBF755FB33462646099C06
:105180000028EAD115A80580109F14971195E4E72F
:10519000109F0E9B1C463E4638461299FBF771F94C
:1051A000FBF7FCFB0546052800D3052513A8058061
:1051B00001200A9A274682E725B0F0BDF0B58BB0F2
:1051C0000243159A149C139E2BD0054601A856C085
:1051D000129CD869196A09900A911E469F6B012397
:1051E000009309A807AA0146059306F005FD716C16
:1051F0003846FBF746F90746E06A616BFBF741F971
:10520000002D069613D0044611980199012924D146
:105210000921081A0421069A515E884229D1642581
:10522000B1E000203080207010700BB0F0BDB0886D
:1052300000226425002829D0059269493846FBF7E9
:105240001BFB0028049C039E6FD166493846FBF780
:1052500013FB00281DD05A2567E03C25082800D103
:1052600091E05F492046FBF707FB002819D0502545
:1052700089E00A291DDB1D293BDC59493846FBF72B
:10528000FBFA0022002854D05A253AE03346049C09
:1052900039E055493846FBF7EFFA002821D0502570
:1052A00043E050492046FBF7E7FA00282ED0462578
:1052B00069E03C25012866D049492046FBF7DCFA25
:1052C0000028D4D147492046FBF7D6FA0028EED172
:1052D00045492046FBF7D0FA002854D143492046DF
:1052E0006EE042493846FBF7C7FA00281CD1282552
:1052F0001BE03B493846FBF7BFFA0022002832D0BA
:105300005025049C069B0299039E41E036492046A5
:10531000FBF7B2FA002836D134492046FBF7ACFA45
:1053200000282FD114252EE037250299059A069BD7
:105330002EE005922B493846FBF79EFA002896D1BD
:1053400029493846FBF798FA0028B0D12749384652
:10535000FBF792FA0028049C069B0299039E059A8B
:105360003BD11E2514E005921E493846FBF784FA0E
:1053700000289CD11C493846FBF77EFA00281DD036
:105380003C2500E02325049C069B0299039E059A78
:105390002580327000200870307800280CD1186801
:1053A0001349FBF75BFA002806D12088102803D3A5
:1053B0000F3820800BB0F0BD0BB0F0BD0B49384664
:1053C000FBF75AFA0028049C069B0299039E059A53
:1053D00001D11425DCE72325DAE72D25D8E7C046DF
:1053E000CDCCCC3DCDCC4C3DCDCCCC3C0AD7233C18
:1053F0000000204070B588B00C4606464088002862
:1054000020D0FBF78CFA059005A804A901252A46AF
:1054100006F05CFE3088B188081AFBF775FA039035
:10542000049903A807AA2B4606F010FE5249079DCF
:105430002846FBF721FA002808D0BF20000620608C
:1054400008B070BD0020206008B070BD4B492846F0
:10545000FBF7F6F9002804D03F200006206008B0D2
:1054600070BD47492846FBF707FA002801D0002005
:1054700010E000212846FBF7FFF9002801D00220A8
:1054800008E040492846FBF7F7F9002801D004203E
:1054900000E0062001957F21C905029180003A496C
:1054A000091801A806AA022306F084FD06982060C8
:1054B00008B070BDF0B587B00C46054647680026B9
:1054C00038463146FBF7E6F9002802D0266007B0DF
:1054D000F0BD049704A803A90126324606F0F6FDA4
:1054E000A8682968FAF788FF0290039902A806AA1B
:1054F000334606F0ABFD2049069D2846FBF7BCF974
:10550000002804D0BF200606266007B0F0BD1B4966
:105510002846FBF795F9002804D03F2006062660B0
:1055200007B0F0BD16492846FBF7A6F9002801D0C0
:10553000002010E000212846FBF79EF9002801D04A
:10554000022008E00F492846FBF796F9002801D011
:10555000042000E0062000957F21C905019180000C
:1055600009490918684605AA022306F023FD059E8D
:10557000266007B0F0BDC046CDCC0C3F295C0FBF04
:10558000CDCC4C3ECDCC4CBE4C940102F0B587B096
:105590000C4606467F270088002801D0FD0503E061
:1055A000B08800282ED0334DFBF7B9F903907088EE
:1055B000FBF7B5F9049003A802A90126324606F0CC
:1055C00085FD029904A806AA334606F03FFD2A4944
:1055D000069E3046FBF750F9002802D03F20010616
:1055E00041E026493046FBF72BF9002802D0BF20C6
:1055F000010638E022493046FBF73EF9002805D085
:10560000002024E00020206007B0F0BD1D49304696
:10561000FBF732F9002801D0022018E01A49304681
:10562000FBF72AF9002801D0042010E01749304682
:10563000FBF722F9002801D0062008E01449304683
:10564000FBF71AF9002801D0082000E00A20009694
:10565000F905019180000F490918684605AA02233F
:1056600006F0A8FC05992846FAF7CEFE206007B0A0
:10567000F0BDC046000080BF000038433333733FA5
:105680000000C84200007042000020420000A0411B
:105690000000C0406C940102F0B59DB015460B911E
:1056A0007F210391C9051C9102911B9119A9002426
:1056B0008C80199418941794598C0691198C0F9119
:1056C000DE8B998B0791997805911F882B21CA430E
:1056D0002799914201DB7F0015E04022D24391429D
:1056E00011DC4922D243914202DB7908CF190AE04A
:1056F0005322D2439142EEDA5D22D243914201DB42
:10570000BF0000E0FF000A971396269E597E0029ED
:105710000BD0002132460F46D1709170517011703C
:10572000121D7F1C5C7EA742F6D30C931195259920
:10573000149122990D91159041088C4211D2FD4A85
:105740002346A00084583454270A451C7755250C5D
:10575000871CF555240EC01C34545B1C9CB2A1421E
:10576000EFD82398109001200990009030463146E0
:10577000149A159F3B4606F04DFA0D9800060890C6
:10578000400E139D00D186E068000490002F3FD0AA
:10579000002210461146144606E01C461146159F8D
:1057A000401C82B2BA420ED283B2AB42F8D0920011
:1057B000149B9A5E0FB2BA42034600DC2346BA42FB
:1057C000EBDC0A46E9E7002F25D0002210461146FF
:1057D000129206E012931146159F401C82B2BA4203
:1057E00014D283B2AB42F8D0A5B2AB420CD0920037
:1057F000149B9A5E0FB2BA42034600DC129BBA4277
:10580000139DE7DC0A46E5E7139DE6E7129903E0FE
:105810000024214600E00021129110980183C482E7
:105820008582049FF057FBF76FF87921C9050E9127
:10583000FAF7EAFD1099C86109980743F057FBF79A
:1058400063F80E99FAF7E0FD109F38622004C40B4C
:105850003057FBF759F80E99FAF7D6FD7862601CBD
:105860003056FBF751F80E9C2146FAF7CDFDB86291
:1058700012980004C70BF057FBF746F82146FAF7D9
:10588000C3FD109CE062781C3056FBF73DF80E9982
:10589000FAF7BAFD2063119805800C98407E41000C
:1058A00000278D4228463A46149E1ED30A9880B29D
:1058B0008AB29300F45E84420BDA491C8AB2AA428F
:1058C000F6D9002728463A4681B2691A012910D034
:1058D0001BE0F018119B1980078808040FD05000B6
:1058E00040008019001F0288084681B2691A012908
:1058F0000BD1A800301811990D80078826E00020F0
:10590000024681B2691A0129F3D00A9989B2079B2C
:105910004B43BB421AD306998A4217D805990029EE
:1059200014D0401C82B2891803E0401C82B291421C
:105930000CD983B2AB42F8D89200B35EBCB2A3429A
:10594000F3DDB218119B18801788EEE712970B98B9
:105950000580119800882B1A002B16DD02210F9A62
:105960001143032942D10E93411C421E10B28142C1
:105970000EDA0E98032824DB0C98808C012820D0A6
:1059800019A818A9FFF736FD1FE0002018902BE09A
:105990000026F443374608E0B8B2400019AD2B5258
:1059A0007F1C521C10B28142E3DB13B2A342334688
:1059B000F2DD159B98423346EEDA8000149B1B5AA9
:1059C000EAE719A818A9FFF7E1FD149E139D0F9AA5
:1059D000012A13D0032A11D0022A04D11198008879
:1059E000281A02280ADA0020179034E0022A01D18E
:1059F000022BB8DA00201890012AEBD1681C691E2E
:105A00000FB2B84208DA0C98808C01281DD119A871
:105A100017A9FFF7BBFD1CE00022D343144608E0A2
:105A2000A5B26D0019AF7E53641C491C0FB2B84279
:105A3000E9DB0DB29D421646F2DD159DAF421646DA
:105A4000EEDABD00149E765BEAE719A817A9FFF706
:105A5000D1FC149E139D249F189C17992046FAF799
:105A6000CBFC0F99012900D8204638600D980028FA
:105A700000D1CBE011990888109FB8860888281AB1
:105A8000B880129880B2FAF74AFF7921CC052146F6
:105A9000FAF7BAFC2146FAF7B7FCB863119F3888C9
:105AA000002849D081008919091F0988129C0C1906
:105AB0001599884203D280008019808804191598AE
:105AC0004300534916AA304606F082FA16981099F8
:105AD0004864FAF77CFFA4B2A04201D14D480FE020
:105AE000001BFAF71CFF1C901CA81BA9012206F042
:105AF000EDFA2046FAF713FF01461B98FAF784FCEB
:105B0000109908603988491B4A1C92B2032A02D2B4
:105B10000021159F17E009B20229159F12DB3F21D2
:105B20000906FAF7A9FE002802990CD10998810705
:105B300009E0C046402100400020129C159988428F
:105B4000B9D3BCE73449109801610898800E5DD044
:105B5000002F1CD000221146144610464B1B1DB2CC
:105B6000ED135B196B40139D1BB29200B25E534361
:105B70001818A418491C8AB2BA42EFD3FAF7CFFE1C
:105B800006462046FAF7CBFE002C03D100E00026A3
:105B90000398C0051C901CA81BA901252A4606F0E5
:105BA00095FA1B9C20463146FAF72EFC01461098C8
:105BB0008160002F119422D0002427462646139599
:105BC0001291B8B2FAF7ABFE1299FAF715FC054636
:105BD000A0001499085EFAF797FE01461398C007D3
:105BE00085432846FAF710FC01463046FAF7B3FB26
:105BF00006467F1CBCB215988442E2D300E0002622
:105C000011983146FAF700FC1099C8601DB0F0BD3C
:105C100048A701020000204100004040F0B58FB0CD
:105C20000692F74A09AF70CA70C770CA70C70328D6
:105C3000079320D88800F3A10858F649FAF78BFBA0
:105C40000446F549FAF787FB0D90F4492046FAF728
:105C500082FB0C90F2492046FAF77DFB0B90F1494C
:105C60002046FAF778FB0A90EF492046FAF773FBD3
:105C70000990EE4969E0042822D0062820D888003F
:105C8000EBA10858EE49FAF766FB0446ED49FAF72E
:105C900062FB0D90EC492046FAF75DFB0C90EB4956
:105CA0002046FAF758FB0B90E9492046FAF753FBD8
:105CB0000A90E8492046FAF74EFB0990FD4944E076
:105CC0000838022821D88800FBA10858D149FAF7E2
:105CD00042FB0446FC49FAF73EFB0D90FB49204687
:105CE000FAF739FB0C90FF2081052046FAF733FBC9
:105CF0000B90F7492046FAF72EFB0A90CA49204636
:105D0000FAF729FB0990FE491FE08800F1A1085825
:105D1000F449FAF720FB0446F349FAF71CFB0D900F
:105D2000F2492046FAF717FB0C90F1492046FAF7A2
:105D300012FB0B90EF492046FAF70DFB0A90EE4953
:105D40002046FAF708FB0990EC4900942046FAF740
:105D500002FBEC4909680E90EB480468EB480168C7
:105D60004808EB4F05463D400022002D08922DD0FB
:105D7000CA01120E07D0280CE90D12D14000E649E5
:105D8000085AE6490AE0C903090E0CD0280AE90BB3
:105D900010D14000E049085A8F2189004018E430B2
:105DA0000DE0DC490AE081B27F2905D84800DA49D4
:105DB000085A04E0D94901E08F218900401800B257
:105DC000FAF7A2FDD649FAF71FFB024602920395A5
:105DD00007252606D34B1A68002A089840D0791C5C
:105DE0008A420BD21102090E13D0110C1F46D00D9E
:105DF0001FD14800C849085AC84907E01F46110E7C
:105E0000002A13D44800C449085AC2494018E43053
:105E10001FE011041F46090E0ED0110AD00B12D13B
:105E20004800BD49085A8F218900EFE7BE4808188D
:105E30000FE0B84808180CE091B27F2906D8480056
:105E4000B549085A05E0B548081802E08F218900D5
:105E5000501800B2FAF758FDB149FAF7D5FA3B46A7
:105E60000590159F2C40F50E5B69B04919400898C4
:105E700010D0DA02D20E34D0C80B3E210140A64821
:105E8000405AA6494018E43000B2FAF73DFDA44953
:105E9000FAF7BAFA0490149E6800A5A1085EFAF712
:105EA00033FD0146A00009AA1058FAF754FA01463A
:105EB000B8B20128089F019102D1022C0AD9A74F3C
:105EC000052C24D1189808900C2D20D80B2D16D312
:105ED000A44918E00027022C089718D08120C70594
:105EE00015E01A04120E00D1CAE0080AC90B00D04E
:105EF000CDE040008849085A8F218900C2E7092D6A
:105F000000D2C7E096490898FAF725FA08900120D0
:105F10000021B542034600D30B46052C00D30846AA
:105F20001799169A1A9C199D1843069B012B12D19A
:105F3000079B402B22D1002840D03846FAF70BFAB5
:105F400001460198FAF707FA01460098FAF754FA61
:105F5000059A04998AE0079B402B1FD1002838D06E
:105F60003846FAF7F8F901460198FAF7F4F90146CC
:105F70000098FAF741FA059A049977E0002833D09F
:105F80003846FAF7E8F901460198FAF7E4F90146CC
:105F90000098FAF731FA059A049967E000285BD077
:105FA0003846FAF7D8F901460198FAF7D4F90146CC
:105FB0000098FAF721FA059A049957E002981146D9
:105FC000FAF71AFA0399002900D16748059A04994B
:105FD0004CE002981146FAF70FFA0399002900D114
:105FE0006148059A049941E002981146FAF704FACB
:105FF0000399002900D15C48059A049936E0C0460F
:1060000000200100000068C1000088C166665EC112
:10601000000084C1000084410000B44100004841F8
:10602000000020400000F0C0000084C10000F841E2
:10603000333323C1000050C19A9929C19A9949C1AB
:106040009A9949413333CB4166667641CDCCAC4019
:10605000333393C09A9949C102981146FAF7CCF9A3
:106060000399002900D14048059A049928601046F8
:10607000FAF7C2F90899FAF7BFF920600FB0F0BD3E
:1060800099B27F2911D848002349085AFCE62349D0
:106090004018F9E6C12001060898FAF75CF9089063
:1060A000062D00D933E7002030E78F2189005818EA
:1060B000EAE6C0463333F341000058C19A9961C102
:1060C0009A9969C1000084C10000AC4100003841C8
:1060D000000008C1CDCC80C1CDCC88C133338FC185
:1060E000333397C133339741CDCC8C413333F340B5
:1060F0009A9919C0666646C1333397C1CDCCB44175
:106100000000D4410C000040503000406840004086
:10611000FFFFFF007C0800000C2401005C0500006C
:10612000919AF63C642000409C0B0000FFFF1F008A
:10613000FAFFFCFFFEFF000002000400060008005A
:106140000A000C000E0010001200140016001800C7
:106150001A001C001E00200022002400000080BF46
:106160000000A0C0000040C00000DCC2F0B5FFB0DD
:10617000ECB017460E460D900021E991E891DC91B4
:1061800099919891979196911491139112919AA83F
:10619000F49DF39CF29A002E00D1E6E10B9380303F
:1061A000F09B1180099529602546DBAC218095ACD8
:1061B00021800C952980DA917F24E405B994B89464
:1061C000B794B694B594B494B394B294B194B09493
:1061D000AF94AE94AD94AC94AB94AA94A994A894C3
:1061E000A794A694A594A494A394A294A194A094F3
:1061F0009F949E949D949C949B949A940466446668
:106200008466C466046744678467C467046444643E
:106210008464C464046544658465C465046244623E
:106220008462C462046344638463C463046044603E
:106230008460C460046144618461C461B0090B2559
:106240000B2800D3AE011095012B0B9D00D070E1FF
:106250002B89012B00D06CE1298C00290E9200D1F2
:106260008BE16B8C002B00D1FAE1AA8C3021695CA8
:10627000002900D188E10892109F5F4311963046B3
:1062800039460F93F9F726FF0590FAF73DFB0146D3
:106290002046FAF7F6F88321C905FAF7B5F806465D
:1062A00096A8021D119887420A9200D879E155A854
:1062B00011909AA9069196AF15463A46059C234639
:1062C00005F078FE15A80F9006992A46234605F09A
:1062D00071FE02230D93384631463A4605F0B6FE6C
:1062E000012308930093E8AA10923846394605F036
:1062F00083FCE898DD901198069D29463A4623468E
:1063000005F058FE0F9829460A9A234605F052FEDA
:10631000384631463A460D9B05F098FE089B00939F
:1063200038463946109A05F067FCE898DE901198D7
:106330002C4629463A46059D2B4605F03BFE0F9814
:1063400021460A9A2C462B4605F034FE3846314643
:106350003A460D9B05F07AFE089B00933846394675
:10636000109A05F049FCE898DF901198069D29469F
:106370003A46234605F01EFE0F9829460A9A234600
:10638000254605F017FE384631463A460D9B05F086
:106390005DFE089B009338463946109A05F02CFCA8
:1063A000E898E0901198069C21463A462B4605F065
:1063B00001FE0F9821460A9A2C462B4605F0FAFD5D
:1063C000384631463A460D9B05F040FE089B009347
:1063D00038463946109A05F00FFCE898E19011987C
:1063E000069D29463A46234605F0E4FD0F982946C6
:1063F0000A9A2346254605F0DDFD384631463A46E1
:106400000D9B05F023FE089B009338463946109AF1
:1064100005F0F2FBE898E2901198069C21463A4676
:106420002B4605F0C7FD0F9821460A9A2B4605F02A
:10643000C1FD384631463A460D9B05F007FE089BE4
:10644000009338463946109A05F0D6FBE898E39059
:10645000119821463A462B4605F0ACFD0F9821468F
:106460000A9A2B462C4605F0A5FD384631463A4699
:106470000D9B05F0EBFD089B009338463946109ABA
:1064800005F0BAFBE898E4901198069D29463A4633
:10649000234605F08FFD0F9829460A9A2546234684
:1064A00005F088FD384631463A460D9B05F0CEFD95
:1064B000089B009338463946109A05F09DFBE898F2
:1064C000E5901198069C21463A462B4605F072FD50
:1064D0000F9821460A9A2B4605F06CFD3846314646
:1064E0003A460D9B05F0B2FD089B009338463946AD
:1064F000109A05F081FBE898E690119821463A46FB
:106500002B4605F057FD0F9821460A9A2B4605F0B9
:1065100051FD384631463A460D9B05F097FD089BE4
:10652000009338463946109A05F066FBE898E790E4
:106530007AE010880C9A108099919891DA9E08461A
:106540000F46099DF59CF9F757FF2860DC982760F6
:106550006060A6600C34DDA80EC80EC42EC82EC420
:106560002EC82EC47FB06CB0F0BDFF20108000217B
:10657000296020807FB06CB0F0BD00220123302163
:10658000695C002900D076E6DDAA1ACF1AC23ACF9C
:106590003AC23ACF3AC20B213046F9F79BFD054685
:1065A00042E000200690059D0796089F11900698EE
:1065B00001460D9C0F9A4A43D219109B5A43119BD6
:1065C000D218D200A35889002E4655AD6B503546DF
:1065D000121DA25815AB5A50401C01B28E42E9DC84
:1065E00055A89AAE96AC314622462B4605F0E2FC01
:1065F00015A831460A9A2B4605F0DCFC02232046FA
:106600000799224605F022FD01230093E8AA2046BF
:10661000214605F0F1FA119B9800DDA9E89A0A508D
:106620005B1C0B2B1846C1D1F19EDDA89AA9DCAAF0
:106630000B2305F0BFFC09210E980F9101800B98E8
:10664000C168DC9C2046F9F7DFFE0146A8B2E69F50
:106650000F281BD808280DD30846F9F77CFE14E054
:10666000FF2010800021099A11600C9908807FB0EA
:106670006CB0F0BD042803D381220846D10502E0A6
:10668000412208461106F9F7BFFE01462B20C04300
:1066900086420D9704DB0846F9F75DFE014603E0EC
:1066A0004020C043864244DD0E9A0C9C0B98408AE1
:1066B000002811D00B98038A95A80390DBA80290BC
:1066C000DAA801900094DDA80D4603F093FC29465A
:1066D0002488DA9E099D68E011910F982080002798
:1066E0003D46109705E00E9804887F1CB8B2A04282
:1066F00011D8B8B28000DDA90C5820461199FAF7DC
:106700009FF80028EFD1002DEDD10C9807800125CE
:106710000F971094E7E7DBA805800F9A90B2201A34
:10672000012811D10C9804800D9FDA973E46099DEF
:106730003AE04920C043864200DA8BE0FF22084657
:106740009105F9F761FEA9E710200B990E5E012E65
:1067500000DA90E0551CABB21846A1B2AAB28A4248
:1067600017D805E00E990C88A1B2AAB28A4210D8B7
:106770008000DDA90C58204610991F46FAF752F800
:106780003B46002805D10C9805800B98068A0F958A
:10679000109430B2C1186D1CA8B28142E2DC109E88
:1067A000DA960F9C099D0D9F11993046F9F769FE05
:1067B000FAF7F4F8052800D3052095A90880A0B2BF
:1067C0000E990988814218D9401C611E0CB2A04262
:1067D00018DA12A898A9FEF76DFE0E980188481CD9
:1067E000491E0CB2A04221DA12A899A9FEF762FE56
:1067F00099999898099D0D9FA4E6002198919991E7
:1068000008469FE60022134608E09CB2A40012AF9F
:106810003D515B1C491C0CB2A042DADB8DB20A2D43
:106820001546F2D8A400DDAD2D59EEE7002213463F
:1068300008E09CB2A40012AF3D515B1C491C0CB295
:10684000A042D1DB8DB20A2D1546F2D8A400DDADF1
:106850002D59EEE75320C043864200DB1BE70E466E
:106860000B9881692046F9F7DDFF00280C9C08D1C0
:106870000B98808B07E01446099D0D9F1199109E7F
:1068800093E70B98C08BFAF74AF801463046F9F7C0
:10689000BBFD119021E70000F0B58BB01C460993B9
:1068A0000E46034600200A9040480088224F059774
:1068B0000AA9049103940292109C01940125009569
:1068C0000B21414389B230331C4A3046FFF74EFC5E
:1068D0003868079078680890B86806903348008850
:1068E000334F009501940297324E30363249334A85
:1068F0003346FEF76BFB0698F862079838630898F2
:106900007863099800882E4905912E4904912E49F3
:1069100003910297019000962C4B284629462A465F
:10692000FEF74CFC432001060A98F9F76DFDFAF7D3
:1069300035F80BB0F0BDC04610A70102C8DF010258
:10694000F0B589B00F9F0E9C002815D010980790C5
:1069500016480088164E012500950191029608936D
:10696000144B30331449154AFEF730FB089BF7628D
:1069700007983063746303E00D484763C4620025E1
:1069800018880F4905910F4904910F49039108494F
:106990000291019007483030009001210B4B2846AE
:1069A0000A46FEF70BFC09B0F0BDC046B4AD0102CB
:1069B0008CD4010274A00102FC9E01029CD201024F
:1069C00040A40102B0AD010250AD010258AD010278
:1069D0003048704700487047F4AD010280003749E5
:1069E0000918C86B0022CA637047C046800033494B
:1069F0000918886C00228A647047C04680B52F4A07
:106A0000D369002B01D0126A9847002080BDC04690
:106A10000249087800220A707047C04664C9010222
:106A20000020704780B5182905D803468A1E034800
:106A30001946F9F79FFB002080BDC046B8AD0102A2
:106A4000B0B502460020022901D2C043B0BD8C1E61
:106A50000F2C07D8044D284611462246F9F78AFB29
:106A600000202855B0BDC046D4AD0102B0B50246E5
:106A70000020022901D2C043B0BD8C1E0F2C07D8C4
:106A8000044D284611462246F9F774FB002028558C
:106A9000B0BDC046E4AD01020849087800220A7082
:106AA0007047C046B0B50446044DAA68002A02D01B
:106AB000E968204690472C610020B0BDB4970102E0
:106AC000F0B581B0E14C206A0025002828465ED050
:106AD000324E3278012A11D1DB48808A3049096868
:106AE000012281420ADA0020E0706178002905D095
:106AF000E0706070022002F039F93278D24FB98A22
:106B000027480068884201DC002A0ED1E278531C35
:106B1000E370152A09D36278002A06D1012060703B
:106B200002F024F9B98A1E48006888420DDA2078FC
:106B3000002801D0002020700020A0706062194958
:106B40000870307800280CD118E00121A170626A29
:106B5000531C6362FB8A9842132A04DA30780028B7
:106B60000CD001B0F0BD2078002800D121700020A9
:106B700060620C48017030780028F2D1207800283B
:106B800001D101202070F6480549086001206562A6
:106B9000A0700449087001B0F0BDC046D098010251
:106BA000F8980102B596010280B5124801681F22CB
:106BB0000A40026003200840022812D10E480268F1
:106BC000D30D02D0FF231B06D2180C4B1A600C4ABF
:106BD00012680C4B1A6080680B4A1080000C0B4A3C
:106BE00010801A488268002A02D0826800209047EC
:106BF00080BDC0467420004064400040B0D2010215
:106C000078300040B4D20102D8A0010282D401023F
:106C100080B50D48016889070FD5052101600B4833
:106C2000C178002908D00021C170C168002903D0B3
:106C3000C26841680020904780BD054805A10B4A05
:106C40000BA308F033F9C0462C0400403494010231
:106C5000703D01005048595F54494D45525F4952BB
:106C60005148616E646C6572000000008D0A00007E
:106C7000556E657870656374656420696E746572BD
:106C8000727570740000000070B50446401E012843
:106C900014D80320084011D13F2040030818050BE9
:106CA000281980280AD8164E3178012048402946F4
:106CB00004F0FAF8641E6D1C002CF5D170BDC046BE
:106CC00080B50020014603F037FE002800D080BDCB
:106CD0000B480121017080BD70B516460C46054673
:106CE000FF22F9F759FA05483118054802780120C2
:106CF00050402A46234603F07FFF70BD00E00704A2
:106D000048A9010201200003704701204003704799
:106D1000F0B585B04A484B49016005F0FDFF4A4D8A
:106D2000E98A522249488152AA8A5023C252AC8D24
:106D30004023C452AB88C362AE7A8671AE89468264
:106D40008282C18204938387611E8C41610001624B
:106D5000A98B3B2901D83C21A9830021E983322159
:106D6000695CC171288B3A490880852040006880A1
:106D70006C8C0F20224602407D21C900260B4E4319
:106D8000B6182205170F64225743F6192406270F59
:106D90000A246743F6192F4F3E80AE8C37460740D2
:106DA0002B46350B4D43ED1937053F0F5743ED1972
:106DB0003606360F6643AD19274E3580DD8C2E46DC
:106DC00006402F0B4F43BE192F053F0F5743F619AF
:106DD0002D062D0F65437519204F3D801D8D2840D0
:106DE0002E0B4E4330182905090F51434018290630
:106DF000090F614340181A4E3080032419A220461F
:106E00002146049B09F0AEF80F484088C1B20091BA
:106E1000030A18A22046214609F0A4F80D48038869
:106E20000D48008839883288094D2D8800AE27C664
:106E300019A22046214609F095F805B0F0BDC046DC
:106E400000960102058500004AA9010298990102F5
:106E50007C960102749601027696010278960102F0
:106E60007A960102C9E8B1B849443A202578202E23
:106E70000D0A0000B9CCBCFEB0E6B1BE3A5557428F
:106E80002D3447B3B5D4D8CAD6BBB7205625642E07
:106E900025642E200D0A0000B7FECEF1C6F7B5D846
:106EA000D6B73A2025642E25642E25642E25643A13
:106EB00025642E0D0A000000F0B581B0254E337810
:106EC000002B0CD0244D4035002214462F888742D9
:106ED0000AD0AD1C641C521C9A42F7D301E0002476
:106EE00022469C4203D006E0D4B29C4203D1172B29
:106EF00001D8631C33705300174CE31840255853D6
:106F00000020A0543089002820D0144A90421DD07F
:106F1000B46A1348844219D00846F9F707FD0025E2
:106F2000104B2A46F9F79EFB074600912046F9F7D9
:106F3000FDFC2A460B4BF9F795FB02460B463846FB
:106F40000099F9F7DDFAF9F757FD0146B16201B092
:106F5000F0BDC046D0980102089A0102FF7F0000F0
:106F6000FFFF01000000E03FF0B583B0304800684B
:106F7000C16B0901890F01D003B0F0BDC16BC06BBB
:106F80002C4D05404800400F0826029686400227F7
:106F9000384602F077FD01907043C10B4A1B26482A
:106FA0005043F9F7ADF8044607F0C2FE032123A2CF
:106FB00038461F4F0091234608F0D4FFF88A002876
:106FC00017D0019840012946F9F784F84643182262
:106FD000324001200F2A014600D8002173095B18B6
:106FE0001B4CA3420DD8194DED1A6D050F2A0CD874
:106FF0000CE038680021C160112002F033FD03B0BD
:10700000F0BD5D1C6D050F2A00D956422A0C029D69
:107010002E4009018919A34202D80098000400E01B
:107020004004081880183968086303B0F0BDC046F2
:10703000C4940102FFFF1F0040420F0052434F3330
:10704000324B2070706D2025640D0A00FF07000090
:10705000FE7F0000B0B582B0154908688269D2078A
:107060000CD00122C2610D69002D07D000686C466A
:10707000214607F0F5FB00212046A84702B0B0BD2D
:10708000B0B582B00A490868026C92070ED5026C4E
:10709000012313430364CD68002D07D000686C46BC
:1070A000214607F0DDFB00212046A84702B0B0BD15
:1070B000C4940102064801680322914301600168FB
:1070C00001220A43026000F03DFB07F053FEC04678
:1070D0002800004080B50D490868002810D52248D6
:1070E00002680423032A01D01A4300E01A460A600A
:1070F0001E490A68002A02D041680020904780BDDE
:1071000003A00CA19E2211A307F0D0FE2C10014079
:10711000696E636C7564652F647269766572732F2E
:107120006D6B5F736C6565705F74696D65722E63FE
:1071300000000000534C4545505F54494D45525F97
:1071400049525148616E646C65720000556E6578F5
:1071500070656374656420736C65657020696E7416
:1071600065727275707400000C90010288D401027F
:10717000B0B582B004460078002811D0094D01A9AD
:1071800008702868416A0029FCD101A90122002069
:10719000034609F0A9FC611C607800280C46EED17A
:1071A00002B0B0BDFC94010270B50C784D782D0290
:1071B0002C198D78C9780902491909040919800028
:1071C000094C21509178D47815785278074E335075
:1071D000074B069E1E501202521923025918090429
:1071E0008918044A115070BDAC9F010270E0010281
:1071F0000CE0010210A0010210B5DC4C2168062948
:107200000FD8012002468A4058210A4209D0206046
:107210000020A0602369002B03D0626900200221B6
:107220009847D1482258062A12D801210B4693408C
:10723000582213420CD0215020180021816003698C
:10724000002B05D0AD20C000225801200221984714
:10725000D9482258062A11D801210B4693405822BA
:1072600013420BD021502018002181600369002BAC
:1072700004D003482258022001469847002010BD40
:10728000BC0A0000F0B581B00024022803D9E44311
:10729000204601B0F0BD17460B46094E464309484B
:1072A0008519284618302A2107A2FCF7E7FE42205C
:1072B0002F52032003498851204601B0F0BDC0463B
:1072C0005405000074AE010225730000F0B585B0CE
:1072D000DD4D2C68002C0CD0DA4FDB4CE659002E2B
:1072E0000CD0B54FE659002E0DD00020C04305B09C
:1072F000F0BD01AC0FC400272E4608E001AE0FC65A
:10730000E619012703E001AE0FC6E6190227CD4CAE
:1073100030462146FCF798FD022030607C43291955
:10732000029D4D60CF60039808610498486108464B
:107330004430CC310122560210233246FCF77AFF4A
:10734000E1480019B32189004118012D05D1B83059
:1073500001233246FCF759FB04E074301023324617
:10736000FCF768FF01980760002005B0F0BDC0463B
:1073700001460020022901D9C0437047E04A4A4330
:10738000E04988507047C046022806D8E449414386
:10739000E44840180249401870474B20800070476D
:1073A000D4040000022802D94B2080007047DC4939
:1073B0004143DC4840184D21090140587047C04600
:1073C000032801DB03487047D5494143D54840189D
:1073D000183070477D3B0100022806DCD04941434C
:1073E000D04840184221405A704700207047C0469C
:1073F000032801DB00207047C9494143C9484018B0
:1074000044307047022804DCC5494143C548405810
:10741000704700207047C046022805DCC049414340
:10742000C04840184068704700207047B0B500243D
:10743000E14302280FD8BA4A4243BA4B9D58042D63
:1074400009D0991801220A600B69002B05D04A69FE
:107450000221984721460846B0BD2046B0BDC0462F
:1074600010B50024022801D9E04310BDAC494143C6
:10747000AC4A0723535051180B69002B03D04A69BB
:10748000002421469847204610BDC04610B5002470
:10749000022801D9E04310BDA1494143A14A062376
:1074A000535051180B69002B02D04A6901219847AB
:1074B000204610BD10B50024022801D9E04310BDBC
:1074C00097494143974A51180B69002B02D04A69EA
:1074D00003219847204610BDF0B583B0174600241D
:1074E000E24302281AD8002B18D00D468C4941439C
:1074F0008C48461870680128029312D1002F0AD0D8
:10750000B836002429193046FCF787FA002825D11F
:10751000641CA742F6D1029807600022104603B00F
:10752000F0BD019274363046FCF73FFE002811D0C2
:1075300003464268BA4209D2196828461D46F8F740
:1075400019FE2B4668680299086001943046194676
:10755000FCF701FE019A104603B0F0BD02980460EA
:107560000022104603B0F0BD5405000074AE0102C5
:107570006C480168062909D06949415806290BD091
:107580000D49415806290ED0002070470121816025
:10759000634941580629F3D1064901224250064960
:1075A00041580629F0D1AB210901012242500020A7
:1075B0007047C0465C050000A80A0000F0B581B025
:1075C00004460020C343022C02D9184601B0F0BD86
:1075D00015460E461B4A62431B498F1879680129DC
:1075E00010D1002D28D01C460090B83738463146BF
:1075F000FCF7ECF9002821D1761C6D1EF6D100981D
:1076000001B0F0BD0090743738462946FCF7E8FD1C
:1076100000280CD00446006831462A46F8F7AAFD37
:1076200038462146FCF7ACFD009801B0F0BD07A03C
:107630002146FCF789FA009801B0F0BD204601B060
:10764000F0BDC0465405000074AE0102536F636B79
:1076500065745B25755D20526563762042756666AC
:1076600065722046756C6C0D0A000000F0B583B0A1
:10767000154607460022D043022F19D8002D17D0F7
:1076800000AB07C30F4878430F490E184436304605
:107690002946FCF7A5FD00280CD004460068019996
:1076A0002A46F8F767FD30462146FCF769FD029847
:1076B00003B0F0BD05A03946FCF746FA009803B0C8
:1076C000F0BDC0465405000074AE0102736F636BD9
:1076D00065745B25645D2073656E64206275662049
:1076E00066756C6C0D0A000002460020022A04DC5C
:1076F0000B4B53430B4AD1507047C0437047C046B1
:107700005405000074AE0102022801D90020704720
:107710000349414303484018034940587047C04655
:107720005405000074AE0102CC04000080B504488A
:107730000168491C01600069002800D0804780BDB5
:10774000F4DF0102014802490160704780900102A4
:107750000026B80310B5C34800244461103002214C
:10776000024A2346FFF7B2FD204610BD19780000FB
:1077700070B584B0FDF7D0F8012814D1FCF712FBE6
:107780001F4D6969022914D0002909D129780029DF
:107790001FD0A969411A062902D300212970A861C6
:1077A000002004B070BD164800214161002004B0E3
:1077B00070BDE969421A13490E2A02D80A78002AD4
:1077C000EED0E8610020087000F004F9002004B059
:1077D00070BD01266E61AB88E88829896A8900AC92
:1077E00007C4B102084C09A22046FCF747FC2869EF
:1077F000AA892146FFF746FD2E70002004B070BD17
:10780000709601024493010260C5010225752E2580
:10781000752E25752E257500F0B58DB0032909D874
:107820007944097949008F4401070F155948416986
:1078300001290AD00DB0F0BD564841690129F9D19E
:10784000022141610DB0F0BD52480021416101703B
:107850000DB0F0BD002500954E4C20694E494F4AB1
:107860006B46FFF739FE0028E4D103204CA2014605
:1078700008F078FB48484DA10A22F8F7B0FC002830
:1078800012D045484CA10F22F8F7A9FC0028D1D10D
:1078900041482C2101AA0C23FCF701FC0298FCF7BB
:1078A000D7FA60870DB0F0BD3B482C2101AA0C230C
:1078B000FCF7F5FB0498FCF7CBFA608780B2684EC2
:1078C000B1888142B6D10298FCF70BFCE0620398C4
:1078D00001794279120251188279C3791B029A18F0
:1078E000120451188278C378077840780002C019D2
:1078F0001B029A1812041018206261620598FCF7A6
:10790000A7FAA0870698FCF7ECFBE0870798FCF73E
:10791000E8FB4027E0530898FCF7E3FB4221605462
:10792000E16A491E062901D80122A270062926D83B
:107930007944097949008F440318111C221E15004F
:10794000E08FB082E05BF082A08FB18D814216D0D3
:107950001E4902220A60B0851D4800E01A48012134
:1079600001700CE00120B08709E018480560B5857A
:1079700005E0B58703E0C0B23C214143B18301205B
:10798000A07000F027F807F053F925626562A57032
:107990000DB0F0BD7096010260C50102FF0300004A
:1079A000CAD5B5BDCAFDBEDD0D0A000024696E73DF
:1079B00074727563742C0000246D65737361676560
:1079C0005F7265706C792C00B4960102B89901025F
:1079D00038900102F0B5C7B0214CA0881490214D19
:1079E00068781390FBF784FE1290A08D1190687850
:1079F00010901D4800780F90A08A0E90E08A0D909C
:107A00001A48C0C81A490A684968AB78194C2468F2
:107A10002035089209910A950B930C9412980090C6
:107A200011980190109802900F9803900E9804906E
:107A30000D9805A9C1C11398012801D00F4A00E093
:107A40000D4A15ADC8212846149B09F081FD024658
:107A5000044800692946FFF709FE47B0F0BDC0465B
:107A60004AA9010270960102A3990102B09801028D
:107A7000A8980102F89801024832010089320100F9
:107A800080B582B00E4908680022C2600192CA68BF
:107A9000002A02D0016801A8904702B080BDC0460C
:107AA00080B582B0064908690022C26001220192B5
:107AB000CA69002A02D0016801A8904702B080BDBF
:107AC0001C930102F0B583B01348007800281ED043
:107AD00000224024114B1146009003E0A41C521CCC
:107AE000824215D29F5C7E1C9E54092FF6D81D5BE6
:107AF0000295C8B2019141005D1819464023029FCA
:107B0000EF520B4601991E540098491CE6E70021EC
:107B10000148017003B0F0BDD0980102089A01023B
:107B2000F0B589B009F038FCEA4C607809F0DAF970
:107B3000E9498A8807A882800A884988090489183F
:107B4000079105F06BF96078052804D00222E3491B
:107B5000092804D104E00122E049092800D089184D
:107B600049792078621C09F081FA607A06F07EFC7F
:107B7000DB48DC4904F044FCDB4C2078002600287C
:107B800006960AD0D9491A31D94A034610CA0C8040
:107B9000891C5B1EFAD14600D34CD64DA872D6483C
:107BA00000886871D549097829706178E970000A00
:107BB000A871481C607028460B30CC4F39464C31B8
:107BC00003913246F8F7D6FA70190B3039461A315C
:107BD0003246F8F7CFFA2020687206982071E088C4
:107BE0006870000AA870C320840106F0AFF9031979
:107BF000BD48C362BC48007881000D31012228468F
:107C0000069209F047FCB8498862B748C46A06F092
:107C100033F90019B44C06F08BFD05460E46AD480D
:107C2000007B06F011FC81B2C90B401800B2C117ED
:107C300040102818A0657141E16506F087F9A06140
:107C400004F050FB0028FBD106F080F9E0617D20B4
:107C50000601002738463946324609F0CFFBA062BC
:107C6000677106F073F92178A54A4A438118A6483E
:107C70000818421C01D1A3480818206306F066F9D1
:107C80006063216B884204D3A04A8918884200D8D7
:107C900097E006F05BF9606306F058F9E06104F0E4
:107CA00021FB0028FBD106F051F9206260790228FF
:107CB0004FD001287DD100206071954D697A21292E
:107CC00071D16979AA79120251188B4A12889142AE
:107CD00069D18A4909782A788A4264D16978AA7870
:107CE00012025118A181E278002A40D02278002A9D
:107CF0000BD07E4B4C3300201C888C4204D09B1C44
:107D0000401C8242F8D11046774CC0B2E081236E0D
:107D1000A16BA26D7E4D2C4622340094724C0191D1
:107D2000029229461A311E352A46FFF73DFAE089AC
:107D3000E178884208D341006C4A5118A2894C234B
:107D4000CA522178491C21700521684A1154704893
:107D500024E0002060710146324609F04FFBA0622A
:107D600006F0F4F8206206F0F1F8A06121E04C2062
:107D70005E4A11520698207005201070236EA06B89
:107D8000A16D2A46223200920190029129461A31B1
:107D90002A461E320020FFF707FA28469621F8F7F8
:107DA00002FA0020208200200146324609F026FB1C
:107DB000A062226B606B55495118904200D365E771
:107DC00067E70126304601F02DFF304609F040FB01
:107DD000A06DE16DFBF78AFAA770207800282FD0FC
:107DE00043484C213D463C46404B05E0891C001D64
:107DF000FAB26D1C95421AD25E5D002EF6D0761E48
:107E00005E55A3000693F6B22246424CE650374B2D
:107E10005E5A5300404CE6527F1C334B9F70036800
:107E20003E4C069EA3511446304B541CDEE705928F
:107E30002D48C77007700497F8B2022806D228E0D0
:107E4000E77805970497F8B2022822D30598441ED4
:107E50000021069403E0491C069CA14219D02F4A38
:107E600010682D4B2B4F0FE0156050605D881E8809
:107E70005E801D8060CF083F3E607D60641E121DE5
:107E80009B1C3F1D002CE6D05568A842ECDC284620
:107E9000F4E704980006059C10D062001E49039880
:107EA000F8F768F9A20012481C49F8F763F90F4A7D
:107EB000184802C81170521C641EFAD10A488389FE
:107EC0000B4800680090032015A2014608F04AF80C
:107ED00009B0F0BDC690010218200100DCA001022B
:107EE0009D010100ADEB0000B89601020898010267
:107EF00038D20102E6E90102C49901029E99010209
:107F000080AA020001CF030000CF03000026B803BF
:107F100088D30102ECE80102B4E9010250E9010250
:107F2000BBF9D5BE4944A3BA25582CBEE0C0EB3AF4
:107F30002025640D0A00000080B5002008F08CFAAE
:107F400080BD80B5012008F087FA80BDF0B581B012
:107F500003F008FD164CE060A178002901D001B0C3
:107F6000F0BD21790029FAD10121217100281BD00F
:107F70008D02281AA168814216D0614E2F46A06852
:107F8000305C21698847A068401CA060681EA16819
:107F9000814201DD0020A060E168A068022F03D3C8
:107FA000691A7F1E8842EAD10020207101B0F0BD1D
:107FB000F0950102B0B5294C2368002B07D0022BA5
:107FC0000DD0012B39D109F0B3F900F00FFC09F005
:107FD0008DF92368022B1FD0012B18D02DE0204DE6
:107FE000287800282FD003201EA2014607F0BAFFF0
:107FF0000020287009F09CF900F034FD1C4D287019
:1080000009F074F928780028E3D00120206019488D
:108010000021C181012310E011480178002909D114
:108020001449CA89531CCB81152A03D3012202703B
:108030000020C88108F022FF2368032014A2014613
:1080400007F090FFB0BD0B48C08914210B1A032024
:1080500009A2014607F086FFBBE7C046B8990102B6
:1080600038900102BFAAC6F4CBD1CBF70D0A0000AD
:10807000A0990102D0980102B5C8B4FDBDF8C8EBC3
:10808000CBD1CBF7C4A3CABDA3BA25640D0A0000A7
:10809000555742D7B4CCACA3BA25640D0A000000F2
:1080A00080B505480068022805D809F041F9FFF7B6
:1080B00037FD09F01BF980BDB899010270B50E2596
:1080C00000242846214603F049FD0D20214603F0F7
:1080D00045FD0124204608F0C7F80426284631460D
:1080E00003F03CFD0920314603F038FD204601F045
:1080F0000FFBA2020249034B204608F0B3FB70BD00
:10810000F8CD01029D0A010080B5032810D800298E
:108110000ED07C224243BF488018C268012A07D192
:108120002030FBF77AFC002801D00020C04380BD3E
:108130000020C04380BDC046F0B589B00022D543C1
:10814000032800D9ABE00C46002900D1A7E0009538
:10815000216A0727534DA9420EDC574DA9421ADD6B
:10816000564A91422FDC4B22D501A9423ED0120241
:1081700091424BD1042246E04B4A914217DD4B4AD3
:1081800091422ADCE1221203914231D0494A9142C4
:108190003CD10C2237E04B252E01B14233D06A018D
:1081A000914227D0AA01914230D102222BE0E12254
:1081B0005502A94220D09502A9421FD0D202914275
:1081C00024D109221FE04B225202914218D0E12211
:1081D000120291421AD1062215E0E1225203914285
:1081E00010D0334A914211D10D220CE003220AE053
:1081F0000A2208E0012206E0072204E0082202E049
:10820000052200E00B22D1002D4A57587C21414322
:10821000804A505056182068B0606068F060A168CD
:108220003161E2687261002505950323049303958B
:10823000029501970695079501231B0208930128D3
:1082400007D000280AD18818009A8018B161F0611F
:1082500004E0304620300123FBF7D7FB2069706330
:108260006069B063E069B067A069F063706801A9F4
:1082700008F024FA2068012806D83046403023460A
:1082800010330ECBFBF7D6FF6068012807D1301DF5
:108290007036006801220B4B314608F0E3FA28469D
:1082A00009B0F0BDFFC10100FF0F0E00FF1F1C0051
:1082B00080841E0040420F007F250000FF950000D3
:1082C00048200100B50A0100B0B50C467C214843A6
:1082D000504A15182846FBF7B7FD6C600020B0BD6A
:1082E000F0B583B00024E743032800D98EE00E46A2
:1082F000002900D18AE01546002A00D186E07C21C1
:108300004143444841188868022832D001283AD0B5
:1083100000282BD1EFF31080C00702D1EFF31080BB
:1083200072B602910846403001902946FBF758FF8B
:10833000002863D0014601980F46FBF721FF3868FB
:1083400031462A46F7F716FF0198FBF72EFFEFF3A9
:108350001081C90703D1EFF3108172B662B602999A
:108360004D6806C82C4B284608F0BEFB204603B0DB
:10837000F0BD4868002431462A46234608F0B4FB85
:10838000204603B0F0BDEFF31080C00702D1EFF339
:10839000108072B602910846403001902946FBF7E2
:1083A0001FFF00281ED0014601980F46FBF7E8FE8C
:1083B000386831462A46F7F7DDFE0198FBF7F5FEEF
:1083C000EFF31081C90703D1EFF3108172B662B6E3
:1083D00002994D6806C8104B284608F085FB2046D8
:1083E00003B0F0BDEFF31080C0070FD1EFF31080A2
:1083F00072B662B63C46204603B0F0BDEFF3108083
:10840000C00703D1EFF3108072B662B63C46204637
:1084100003B0F0BD70BE0102B90D0100B0B582B06D
:10842000602833D0622843D0642854D101A82F4952
:108430000180EFF3108072B600242046214602F03E
:108440007BFA2B4D002805D101200203002029468C
:1084500002F0CCF9103501AA02232046294602F089
:10846000A3FE62B623A0FEF783FE64201B490C52D4
:1084700006F0DEFB1A4801F0D5FBBFF34F8F194819
:1084800019490160BFF34F8F00BFFDE7602013491A
:1084900000220A5206F0CCFB114801F0C3FBBFF3E7
:1084A0004F8F104810490160BFF34F8F00BFFDE7A9
:1084B00062200A4900220A520A8006F0B9FB0848E5
:1084C00001F0B0FBBFF34F8F064807490160BFF3CF
:1084D0004F8F00BFFDE702B0B0BDC0464AA9010200
:1084E000A08601000CED00E00400FA05AAAA000035
:1084F00000D00204BDF8C8EBC9FDBCB6C4A3CABD18
:108500000D0A0000F0B5D1B0A74EA8490A78002A9C
:1085100025D0F28B002A22D1A54FBA68082A00D9AB
:1085200090E0930001A4E3589F46C04651850000A7
:108530004586000045860000558600007F860000C5
:108540008986000093860000638600009D860000F7
:10855000552800D0BBE00120B86051B0F0BD49788B
:10856000002900D1B7E0924D6A7996498854A979DB
:10857000A871E971521C6A710A2800D0ABE00D297C
:1085800000D0A8E003A8019037A800902C46303412
:108590008C488D491DAB2246F7F73EFEE8608BA163
:1085A00005222046F7F71BFE00282AD1F08B002871
:1085B00005D0032087A2834B014607F0D3FC1DA8FA
:1085C0000024214609F08DFCA861E961824B224616
:1085D000F8F76EF9002814D1804800F0A1FF1DA81B
:1085E0000024214609F07DFC2862696237A82146F3
:1085F00009F077FCA862E96203A8F7F79FFE2861FB
:1086000000E0286900266E71002806D074480670C4
:10861000744801210170744806806A489621F7F772
:10862000C2FD1DA864242146F7F7BDFD37A82146E9
:10863000F7F7B9FD03A82146F7F7B5FD6E71EE8097
:1086400051B0F0BDAA2838D1012A36D10220B86035
:1086500051B0F0BD0421B9600021B970787051B0FB
:10866000F0BD3979534A5054481C38717978491F04
:10867000C0B281422FD10820B86051B0F0BD0522B0
:10868000BA60887051B0F0BD0621B960B87051B0C1
:10869000F0BD0721B960387051B0F0BD7A78062A74
:1086A00002921AD3531F0025424A2C46565DA41944
:1086B000A4B26D1C9D42F9DB10E0032807D1022A09
:1086C00005D10120F8700320B86051B0F0BD002042
:1086D000B870B860787051B0F0BD00242018029ACC
:1086E000821888781118BD7849193C780919FA78E8
:1086F000002A00D0C91C2C4EC9B2FF2935D101284F
:1087000009D0022831D11E2D36D1FFF7D7FC012028
:10871000F08351B0F0BD284A94710320107190701D
:10872000AA2050705520107068085071651DD570D2
:10873000400031181646D01D2246F7F71BFD301DAC
:10874000E11CEAB2D21C037892B2D218401C491E36
:10875000F9D1A019D143C171090A0172093401206C
:1087600000233146224608F0BFF90020B870B860F7
:108770003871787051B0F0BD70190E4E31462246F6
:10878000F7F7F8FC3078012802D12846FFF746FEBB
:1087900006F04EFABFF34F8F084809490160BFF356
:1087A0004F8F00BFFDE7C0464AA9010218900102A1
:1087B0008898010294CD0102F49A01020CED00E0C8
:1087C0000400FA05FCCC0102E5310100474E4747A1
:1087D00041000000257300000000F03FB1AD010230
:1087E0002C940102B7960102B2AD0102F0B585B03A
:1087F00008F0D2FD7E487F4903F002FE7E4C002542
:108800002571E57005F0A2FB2062042003F032F927
:108810007A4E726828460495294608F0EFFD60718B
:1088200005F094FB054660632720410170684843CA
:108830000A21F7F74FFCA0634119481C00D00846F5
:10884000E06305F083FB2064E16B6D4D884202D349
:108850004919884234D96B4E6B4F05F077FB206481
:1088600003F040FD00280AD0FCF714F805F06EFB79
:108870002064E16B8842F3D949198842F0D2E0784C
:1088800001280FD130783978814212D1707A2028AE
:108890000FD17079B179090208185C49898D884235
:1088A00007D134E0554842680020014608F0A6FD93
:1088B0006071E16B206C8842CFD349198842CCD8D3
:1088C0000125284601F0AEF9284608F0C1FD2079BF
:1088D000002816D14E4806F02FFA514E3378032067
:1088E00059A2014607F03EFB3078411C3170062842
:1088F00007D35B480221016004983070E0813F4853
:108900000570042003F0A6F8002005B0F0BD01209A
:1089100020713F48623006F00FFA05F017FBE06166
:10892000B27A0392A2707079B17909020818608155
:1089300031460B315500374F384602912A46F7F73A
:1089400019FCA9190B31384632302A46F7F712FCC8
:10895000039A002A049835D000262F4D03E0BF1C4F
:10896000761C964210D2388829688142F7D1788ED9
:108970002081264989890818788601B260890022F9
:10898000FEF79AFAA278EAE7002A10D029680020B8
:10899000029D16462A786B781B029A18914209D0DC
:1089A000AD1C401C32468642F3D1104608E0002040
:1089B000024605E0C5B22846FAF716FC2A46A0781A
:1089C000824202D1C0B2FAF70FFC14480B4948604A
:1089D000134800210170062020560C498B8DA16A96
:1089E0000091019003200FA2014607F0BBFA67E750
:1089F00075010100FDEA0000D098010238900102E3
:108A0000007C3125F0D201029E9901024AA901029F
:108A10001A3F00007C9A0102C499010288130000E9
:108A2000EED20102B1EAC7A94944A3BA25582CBE27
:108A3000E0C0EB3A20256420D0C5BAC5C7BFB6C890
:108A4000A3BA25642E0D0A00B2E2BEE0CAA7B0DCCC
:108A5000A3ACBCC6CAFDA3BA25640D0A0000000081
:108A6000B8990102F0B585B008F096FC794C607AAF
:108A700008F038FA78498A8803A882800A884988E9
:108A800009048918039104F0C9F9607A052804D013
:108A900002227249092804D104E001226F49092801
:108AA00000D089184979207A2246093208F0DEFA86
:108AB000607C05F0DBFC6A486A4903F0A1FC6A4F60
:108AC0000024FC7005F042FA3862042002F0D2FF64
:108AD000664D2046029421462A4608F08FFC7871A4
:108AE00005F034FA62497863B9634118481C00D034
:108AF0000846F86305F02AFA3864F96B5D4E88423F
:108B000002D38919884235D95B4C03F0EBFB00286E
:108B10000AD0FBF7BFFE05F019FA3864F96B8842FA
:108B2000F3D989198842F0D205F010FAF861F87883
:108B300001280FD120785149097881420AD1607A01
:108B4000202807D16079A179090208184C49898D3C
:108B500088421DD005F0FAF93862002001462A4605
:108B600008F04CFC7871F96B386C8842CDD38919C8
:108B70008842CAD80125284601F054F8284608F052
:108B800067FC029C042002F065FF204605B0F0BDA2
:108B90003C4806F0D1F83C482E49486005F0D6F92B
:108BA000F861A27A0292BA706079A1790902081874
:108BB000788121460B315600344D284601913246CA
:108BC000F7F7D8FA31190B31284632303246F7F729
:108BD000D1FA029A002A29D000242D4E03E0AD1CC0
:108BE000641C944210D2288831688142F7D1688E83
:108BF0003881234989890818688601B2788900225A
:108C0000FEF75AF9BA78EAE7002A11D03168002055
:108C1000019D14462A786B781B029A18914210D055
:108C2000AD1C401C22468442F3D102E0002203E046
:108C30000022144694420BD1D0B2FAF7D5FA01249F
:108C4000A0E7C4B22046FAF7CFFABA789442F3D03C
:108C5000012497E7389001021E200100DCA00102E8
:108C600075010100FDEA0000D098010280841E0019
:108C70000098E00E007C3125F0D201029E9901029D
:108C80004AA90102913D0000204E00007C9A010299
:108C9000C499010280B582B0002001900448C268E6
:108CA000002A02D001A80021904702B080BDC04632
:108CB0008C950102F0B583B000242046FEF700F841
:108CC000FEF723F8274EB060FEF71CF87060264FC1
:108CD0000BE001A8C1888088084319D101A8408809
:108CE00024180834B068844235D201AD08212846E2
:108CF0002246FDF7F1FF28880028EAD0B8422AD0A2
:108D000001AD0421284600F077FFA9888842E5D00C
:108D10003460B06884420CD201AD0221284622465C
:108D2000FDF7DAFF2888B84203D0A41CB06884425B
:108D3000F2D370682118491E4042084030600DD0BF
:108D40000024254601202946FDF79EFF03CE4D193C
:108D5000083E8542F6D3346003B0F0BD0024346091
:108D600003B0F0BD20970102FFFF000010B5054CD5
:108D70006070FEF72FFE6078022801D1002060703D
:108D800010BDC0467096010210B5032404A220460F
:108D9000214607F0E7F8BF4884730121417210BDF6
:108DA000344720525820BBBDD0D10D0A000000002E
:108DB000F0B585B01F4604920646C8170C1844400B
:108DC0000A2C039114D301250A212046F7F782F9D2
:108DD0006D1C632C0446F7D804998D4200D32946B4
:108DE0000A9C002F09D00398002808D4002207E02D
:108DF000012504998D42F2D2F2E7002205E001221A
:108E0000042323409B081343FA1A022323400498A7
:108E10000028029412D1002B10D0F468002C62D4E8
:108E20000398002825D40298400734D57068B568A7
:108E30006F1C87422FD830682B2423E0E407ECD145
:108E4000002A0AD1E9E7376820203855B560F06874
:108E5000441CF460521E002CDFD49142DDD27768AE
:108E6000B468651CBD42EED9F468521E002CF4D5DE
:108E7000D3E7404203907068B5686F1C87420AD8F8
:108E800030682D244455B760F068441CF460002518
:108E9000ED43A84227DB002B1CD00120029B184089
:108EA000049B184316D1002A03D113E0521E002C54
:108EB0000ED491420CD27068B3685D1C8542F5D81F
:108EC00030683024C454B560F068441CF460EDE7A9
:108ED000002C08D40092029801900A22304603998F
:108EE000049B00F003F805B0F0BD0000F0B587B0BA
:108EF0001F4615460290012406919142009407D323
:108F0000012406982946F7F7E5F8641CA842F9D22F
:108F10000D980C9ABC42039700D30394009901402A
:108F2000002A009109D00029029C25D12021800728
:108F300005D40846002F11D004E0029C1CE030202C
:108F4000002F0BD0084609E023685854A260E1685E
:108F5000491CE1603246721E00290DD403999142EA
:108F60000AD216466368A1684A1C9A42ECD9E168A5
:108F70003246721E0029F1D5E068002859D40590C8
:108F8000012401E07F1E6C43022FFBD2069821468C
:108F90001646F7F79FF83246A842F4D20298806846
:108FA0000490069F0195069738462146F7F792F8F8
:108FB000049D691C029F7A68914206D9069F059A12
:108FC000019D0592002A0ED516E01B4A125C3B68F3
:108FD0005A55B960FA68521CFA600491069F019DC7
:108FE0000592002A08D460433F1A20462946F7F725
:108FF00071F8AC420446D6D200980028029C059B2A
:10900000049D16D0002E14D0701C01E0002B10D44B
:10901000401E039981420CD2691C62689142F5D8C6
:10902000226820235355A160E268531CE3600D467B
:10903000ECE707B0F0BDC04624230100F0B583B0D3
:1090400001900291002923D00025124F2E460AE0FC
:1090500013480818410F4018C010F872761CB0B2BF
:109060000299884214D2019800884B24210100B251
:1090700000F018F8400061014018788301B20648FA
:1090800081422846E9DB05488142E1DD6420E4E7CE
:1090900003B0F0BD98990102E40C00000410000038
:1090A0001CF3FFFF074A904201DD054A801800B219
:1090B0004143C817400D0818C00A00B27047C046A7
:1090C00000F0FFFFFF07000010B50078012819D15C
:1090D000AC480269012A04D1614A13680124A34300
:1090E0001360032905D080214161C269002A05D19E
:1090F00007E001214161C269002A02D0018980692B
:10910000904710BDFF222E32024803A107A305F0AD
:10911000CDFEC046D82E01006164635F646D615F5F
:1091200063616C6C6261636B00000000556E657872
:1091300070656374656420646D61206368616E6E40
:10914000656C0D0A00000000F0B58DB00D460124DD
:10915000EFF31081214002D1EFF3108372B6894EF4
:1091600073690F2B06DD102B37D0402B2FD0802BAF
:109170002DD005E0002B2AD0012B01D110237361E3
:10918000B5813581B061F261002900D162B63179D3
:10919000002929D00294304C05A90A460495039071
:1091A000E8CCE8C2E8CCE8C2029C204600F0AAFD68
:1091B0002A4800902A4D294608312046039A049BEC
:1091C00000F010FE2C60002420460DB0F0BD0029F8
:1091D000FAD162B620460DB0F0BD02240029F3D1C9
:1091E00062B620460DB0F0BD3178002907D01C488A
:1091F000072181610460002420460DB0F0BD326972
:10920000B3891749002B15D0B5693089012A02D0DE
:10921000002A03D003E09FB2874200D10C604F6860
:10922000FF07FCD08F6880C55B1E1F04EED10023B2
:10923000B381B561012A02D10A68A2430A60746150
:10924000F2690024002ABFD0B36931898800181A56
:10925000904720460DB0F0BD64230100C990000086
:1092600008D00140F0B581B0002856D00446424EE7
:10927000F068800754D41325284600F0FBFB2846ED
:1092800005F0E0FA27686168012538462840CA07DA
:10929000920F1018227C1207120E8018627C12079F
:1092A000120D8018A27C1207120C8018627D130721
:1092B0001B0AC01812091206801830607D200602B1
:1092C0000029304600D12D48E3681A0A7D2A1A4643
:1092D00029D22B4EB3422AD200292BD0002A29466C
:1092E000254E00D01146F6F7F5FE401E80B27060A4
:1092F00024480761E27C0270237D0371224F3E689F
:109300006902A468012C1BD02C0226433E60002B6E
:109310001ED00121184A116329E0012001B0F0BDDF
:10932000022001B0F0BD3246154EB342D4D33346CD
:109330000029D3D11A46002A29460F4ED2D1D2E7AE
:109340003F242401A6437618F0363E60002BE0D17E
:10935000002A0CD0FF2212020C4B1C6894430122FD
:10936000D203A2181A60304A1160304A11600121FC
:109370004161002001B0F0BD00D001400026B803DB
:1093800080841E00A09501022C06004008E400E045
:1093900070B5002801D0012070BD0C461625284666
:1093A00000F068FB284605F04DFA002C05D01B485C
:1093B000183014222146F6F7DDFE28211748415CBB
:1093C000002915D04168002916D403220B46934387
:1093D000144A9C588D07ED0EFF26AE40B4439C50B6
:1093E0001F220A40012191400F4A11600F4A11606B
:1093F00001210161002070BD8A07D20EFF23934036
:109400000F220A40083A03218A43054954589C43D5
:10941000545001210161002070BDC04684900102BA
:109420001CED00E000E400E080E200E000E100E08C
:1094300080B568480021017061480078C001614929
:1094400009788901014360480078400108435F4979
:109450000978090101435E480078C00008435E496D
:109460000978490001435D4800780843C0B2FBF722
:109470004DF980BD80B557480121017051480078F1
:1094800080014F490978C90101434F4800784001E4
:1094900008434E490978090101434D480078C0004E
:1094A00008434D490978490001434C480078084376
:1094B00004210143C8B2FBF729F980BD5A21014AB2
:1094C0005052704774A00102F0B581B013490A7878
:1094D000002A13D0052A01D104220A709300CD1866
:1094E000561C00231C462F686F60F917DB194C418E
:1094F0002D1F761E012EF6DC084902E000221346DD
:1095000014464860521C0A70C11718186141D2B243
:109510000023F6F709FE01B0F0BDC046C095010278
:10952000F0B581B0044600784142414121702448A1
:109530000078C00123490978890101432248007855
:109540004001084321490978090101432048007876
:10955000C00008431F4F3978890001431E4D287809
:10956000400008431D4E31780143C8B2FBF7CEF8E6
:109570007D20C00000F056FB20784142414121701F
:109580000F480078C0010F490978890101430E484E
:109590000078400108430D490978090101430C484E
:1095A0000078C000084339788900014328784000DA
:1095B000084331780143C8B2FBF7A8F801B0F0BD09
:1095C000F89E0102B69601021D9001027CEA01029A
:1095D000B1AD0102F99E01023CA301023DA30102CB
:1095E00070B54F4EB060112400252046294602F088
:1095F000B5FA204629462A4602F044FA03222046BC
:10960000294602F0D3FAB2680221204602F0B2F9EC
:109610002046294604F0FAFE70BDC046B0B5094D9B
:1096200028600224002120460A4602F02BFA01217C
:109630000522204602F0BAFA2A680321204602F0E9
:1096400099F9B0BDF49E01025C219D48002242526E
:1096500082847A2141840284C2830283C28202828C
:10966000114941608260C2603D21490441834182C9
:10967000090C8183818270475C219148002242520B
:1096800082847A2141840284C2830283C28202825C
:10969000054941608260C2603D21490441834182A5
:1096A000090C8183818270474C37373770B5854804
:1096B0004C21016001252C02601C00F05BF9322076
:1096C00000F0B0FA00F044F9284600F04BF92846C3
:1096D00000F05AF800F036F90C4800F04BF900267B
:1096E0003046314600F056FA2846314600F052FA2C
:1096F000204600F03FF9022000F03CF948342046B3
:1097000005F04CFB05F0AAFB70BDC046010200004D
:1097100010B50446072106F083FA0148046010BD25
:109720006096010270B505200424214602F016FA65
:109730000620214602F012FA0A20214602F00EFA13
:109740000920214602F00AFA00240121204602F0F5
:1097500005FA022520462946224602F027FA0B2662
:1097600030462146224602F08DF9304629462246EF
:1097700002F01CFA70BD000002480168012291430A
:10978000016070475800004002490A680240824266
:10979000FBD1704704600040B0B5494D286881078F
:1097A000484C0ED528797F21084022688A4310183A
:1097B000206023680B4002200321434A06F0D2FBBD
:1097C000286880040ED55E20285C7F2108406268EE
:1097D0008A431018606063680B40022003213B4AF3
:1097E00006F0C0FB172000F045F939480168022255
:1097F0000A4301218A4302603648374901603748ED
:109800000021C17181791F2529408171817A427CB3
:10981000837C1B029A18C37C1B04D218037D1B0691
:10982000D2182F4B9A4218D1427B837B1B029A1885
:10983000C37B1B04D218037C1B06D218294B9A4207
:109840000BD1C27A037B491E122906D81902891846
:10985000254A914201D1202101720178CA0602D124
:109860001022114301701C3C206820218843206095
:109870001E481F49016041680029FCD503F032FAF7
:109880000446022003211BA2234606F06BFB0A209C
:10989000C441032C05D8022003211DA206F062FB5F
:1098A000FEE71848C1680F229143C1600168164A5B
:1098B0000A40026019200001144948600D60B0BDE3
:1098C000DCA0010248000040202F01000A2F010007
:1098D000040200400C060040AF6B100A6B00014010
:1098E0004D383650312E32360734000000600040CB
:1098F000FE1C0080436869702049443A20253038B6
:10990000780D0A00C8600040FEFFC3FF0C04004051
:109910004F6C642063686970206D6F64656C2069AA
:1099200073206E6F7420737570706F72746564202D
:10993000627920746869732053444B2121210D0AF8
:109940000000000080B5172000F08CF8002080BDDA
:1099500010B51724204600F08DF8204604F072FF61
:10996000002010BD0121C907014301480160704773
:109970000060004010B5C1B2000AC2B202290CD08A
:10998000012913D0002930D1911E7F4802291BD212
:109990000121032A2AD0490429E07B484168002A92
:1099A0001FD00246203A1143416010BD764801683D
:1099B000D31E022B10D3012A29D0002A41D1012223
:1099C00092079143016010BD002A16D10121490779
:1099D00002688A43026010BD0123042A1FD05A0482
:1099E0001EE0012292079143416010BD0904194A0B
:1099F0007F32C36A13405918C16217498A699207B6
:109A0000FCD50121490702680A43026010BD052206
:109A1000120791430246203A0A43026010BD1A041D
:109A2000836A0C4C1C40A21882620B4A131F00244C
:109A30001C600A4B0A4C1C600D235B0214681C431B
:109A40001460054A93695B06FCD505221207114391
:109A5000016010BD80FFFCFF1402004004010040C3
:109A6000FF0F000001218140474802688A430260DD
:109A70007047C04601218140434802680A430260A2
:109A80007047C04610B5052811D8C0467844007903
:109A900040008744020E192434393B490A6808689B
:109AA000C0003CD53A4820390A425DD03BE0002056
:109AB00010BD35490A680868C00035D534480B46E2
:109AC000203B1A4237D134E02F490A680868C000A9
:109AD00036D52F480B46203B1A424CD135E02A4957
:109AE0004C680120C0030A680B46203B1C421AD078
:109AF0000C68E4003BD5264C1A423CD03AE02248A0
:109B000000680120C00310BD1F490A680868C00032
:109B10001ED51F480B46203B1A4220D11DE01B4892
:109B200020390A4220D010BD18480B46203B1A426B
:109B300001D10120C00349688900890FC84010BDC8
:109B400012480B46203B1A4215D10120C00312E0F7
:109B50000E480B46203B1A4201D10120C003496840
:109B60000903890FC84010BD0120C00310BD074C78
:109B70001A4200D020464A689200920FD0404968AD
:109B80000901890FC84010BD20000040006CDC02B4
:109B90000026B80304282CD8164AC0467844007919
:109BA00040008744020A121A2100032000071368AC
:109BB00083438807800818181AE00320800613687A
:109BC000834388070009181812E0032080041368F3
:109BD00083438807000B18180AE0FF20000213686F
:109BE00083430802181803E01068FF2398434018C5
:109BF0001060704724000040B0B5002200290CD04E
:109C0000074B047895B22D0A65406C001C5B12026C
:109C10006240491E401C0029F3D190B2B0BDC0463D
:109C20002421010000280AD030B407252C02CD25BC
:109C30006419604340091238001FFDD830BC7047DA
:109C4000F0B583B01F4616460D460146E8680291FE
:109C5000F6F7DAFB04460F2E11D8082E04D320465F
:109C60002146F6F778FB09E0042E02D38120C105D6
:109C700001E0412001062046F6F7C6FB044609999B
:109C8000089E2B20C043874205DB20460F46214615
:109C9000F6F761FB0DE03F20C04387420BDA492015
:109CA000C04387420CDBFF200F4681052046F6F7B4
:109CB000ABFB39460446688A0880346003B0F0BDC7
:109CC00001915320C043874206DB20462146F6F728
:109CD00042FB0446688A10E0A8690299F6F7BEFDC7
:109CE000002801D1A88B00E0E88BF6F718FE0146AA
:109CF0002046F6F789FB044600200199088034606D
:109D000003B0F0BDF0B581B005460120072D66D83F
:109D10000C46002963D04A4F38680169C90736D11B
:109D200005263046FFF7A6FE304604F08BFD03CF34
:109D30000369012213430361002918D403200B4651
:109D400083438E481E588807C00EFF278740BE43B6
:109D500040278740374389481F501F2008408240D2
:109D60008748026087480260354800680FE08A072C
:109D7000D20EFF2696400F230B40083B03218B4356
:109D80007D495F58B743402696403E435E50690187
:109D90004018012109024218E369DB069B0CA56902
:109DA000ED00EDB2EB18536062685207520B236866
:109DB0005B075B099A18A3685B079B0CD218E368E2
:109DC0005B075B0DD21823695B01DBB2D2186369B4
:109DD0009B07DB0ED218802313434350002001B0B1
:109DE000F0BDC046F0B581B0002A23D00546083545
:109DF000134C2668F668EE40F50702D0022001B049
:109E0000F0BD069D8600A619B560400124682018A3
:109E1000009301231D02461977680724A743776042
:109E2000F16032610099B1604159194341510020FC
:109E300001B0F0BD03A00AA174220DA305F036F80D
:109E4000D4920102696E636C7564652F64726976E1
:109E50006572732F6D6B5F646D612E63000000008F
:109E6000646D615F7472616E7366657200000000FC
:109E7000496E76616C6964207472616E7366657296
:109E8000206473742061646472000000000158490A
:109E9000085840687047C046F0B581B005460120BB
:109EA000012D4CD80C46002949D0002D03D0012D9E
:109EB00004D10F2000E00E20FFF7DCFDA668012E84
:109EC00004D0002E4FD1E08900284CD12901294827
:109ED00043580020D860F507AD0F27686668B607BD
:109EE000360F76192569EA07920EB618022F04D0AC
:109EF000012F03D10122164300E040361D4F9E6022
:109F0000E2681A6079188D606269CA604968002940
:109F100017D403220B469343184A9C588D07ED0E25
:109F2000FF26AE40B4438026AE4026439E501F22FB
:109F30000A4001219140124A1160124A116001B099
:109F4000F0BD8A07D20EFF2494400F230B40083B3C
:109F500003218B4308495D58A543802494402C433A
:109F60005C5001B0F0BD08A00FA1492212A304F07B
:109F70009DFFC0461C9301021CED00E000E400E0E0
:109F800080E200E000E100E0696E636C7564652FBB
:109F9000647269766572732F6D6B5F6475616C5F57
:109FA00074696D65722E63006475616C5F74696DB0
:109FB00065725F6F70656E00636F6E6669672069BA
:109FC0007320696E76616C69640000000001084AC4
:109FD00010580160816880220A4382607047C04641
:109FE00000010349085881688022914381607047CD
:109FF0001C930102F0B58DB0019315460E460A90F0
:10A000001298002408900480149F3C8013980990B3
:10A010000460159804900480FF2081053046F6F70F
:10A02000F3F90290304603963146F6F794F92B4641
:10A030003D460690274607950B9311E0118018883E
:10A0400080002858099908600120079D2880052074
:10A05000049908807F1CBCB21888844200D9A0E013
:10A0600028880028F6D1A0000A9D2E58304606996F
:10A07000F6F7E6FB002817D030460399F6F7E0FB29
:10A0800000280B9B079DE5D1089A1780099D2E603B
:10A090001888011B012934D11080198889000A9A77
:10A0A00051582960059035E0089A17800998066094
:10A0B0000B9B1988081B0128C0D00C960198251805
:10A0C0007E1CB0B28542BFD389B2B2B28A420ED8EA
:10A0D00080000A990C5820460C99F6F7A3FB0B9BBD
:10A0E000002804D109980460089806800C94761C16
:10A0F000B0B28542A8D3198889B2B2B28A42E7D9F0
:10A10000F5E70C96019962187D1CA9B216468A42A1
:10A1100005972CD2059884B2A5000A9E7259002C8E
:10A12000104609D0A819001F016810460C92F6F7D6
:10A1300012F90C9A062C07D80446A8194168104653
:10A14000F6F709F90C902046079D0299F6F786FB71
:10A1500000280B9B07D10C980299F6F771FB0B9B1B
:10A16000002800D076E701202880032070E780B225
:10A17000AAB282420FD888000A990C5820460C993E
:10A18000F6F750FB0B9B002805D10998046008984E
:10A19000058005950C946D1CA9B28E42BAD318881F
:10A1A000E5E70DB0F0BD00000A490A680A48024020
:10A1B0000A60FD214900094A1268515C002908D053
:10A1C00007490A6C02400A64012000060A688243BB
:10A1D0000A60704700040040FFFFFF7F44940102C3
:10A1E0002000004000207047F0B583B00D460446C3
:10A1F0007C26464350488719F869396AF5F76AFFA3
:10A20000A84200D892E0019502940121EFF310805A
:10A21000084002D1EFF3108272B63C4610343B691D
:10A220000025062B0CD80A469A40D3065B0F06D1B0
:10A2300061231A4275D00D46002803D003E00225A1
:10A24000002800D162B6002D02D0284603B0F0BD30
:10A2500000943C462034384880591021C1613E4664
:10A26000143604F0F5FD05463868C069C00605D50A
:10A2700004F0EEFD401B31888842F5D90621029D8D
:10A28000284600F00BFF206801994143B86909187E
:10A2900038688160172179563C461734002909D562
:10A2A000C16920220A43C2610121F9668905026859
:10A2B0000A4302600521284600F0F0FE207840B2F3
:10A2C00000250028C1D42B4800687D24E100F5F763
:10A2D00001FF61014143029800F0B2FE04F0B8FDB5
:10A2E00004463868C069C00705D004F0B1FD001B02
:10A2F00031888842F5D904F0ABFD04463868C1695D
:10A30000890706D504F0A4FD001B31888842F5D9E1
:10A3100038680121009A116053498161284603B0D1
:10A32000F0BD0321216000288CD08CE7034804A1F4
:10A33000084A09A304F0BAFD48930102502F010016
:10A34000666C6173685F626C6F636B5F657261738B
:10A35000650000005D020000626C6F636B20696441
:10A3600078206973206F7665722072616E67650D63
:10A370000A00000008E00102F0B583B002907C21E1
:10A380004143934A5418E56EEAB2511E02291FD286
:10A3900029040126090E18D001960092022100F02E
:10A3A0007DFE2746143704F053FD06462068C16938
:10A3B000890606D404F04CFD801B39888842F5D903
:10A3C0002068007DC007019E08D0304603B0F0BD74
:10A3D000032A36D100922804000E36D020466C3075
:10A3E0002D0C0021019101602746143704F030FD47
:10A3F00006462068C069C00705D004F029FD801B0F
:10A4000039888842F5D904F023FD06462068C169E1
:10A41000890706D504F01CFD801B39888842F5D9D0
:10A42000206811498161E9B20120002911D0032976
:10A430000099019E00D006202061226F002A0ED1D3
:10A44000C3E70026304603B0F0BD0126304603B016
:10A45000F0BD0099019E2061226F002AB5D002A8AC
:10A460009047304603B0F0BD000093EB70B5002874
:10A4700001D0012070BD7825CD4E705D00280ED032
:10A4800000240921204600F009FE0F20FFF7CAFB37
:10A490001520FFF7E7FA74553461204670BD04209B
:10A4A00070BDC046F0B581B00C460078484EF168EA
:10A4B00081422CD1032C54D1706EB16E884261D987
:10A4C00000240621204600F0E9FD3068F16D81602E
:10A4D0002046214600F0E2FD354660352CCDF0687F
:10A4E0003168B48C414F00975B1BA34200D81C46D7
:10A4F000A3081431FFF776FCB06E0019B066306E19
:10A5000000193066F06D0019F06501B0F0BDB1685A
:10A51000814255D1032C45D1F08CF16D0918F165BC
:10A52000316E09183166B16E0818B066716E8142DD
:10A5300038D900240621204600F0B0FD3068F16DC6
:10A5400081600121204600F0A9FD316EB068F38CD6
:10A550003268264C009414329B08FFF743FC01B08C
:10A56000F0BD30681021C16104F072FC054630680E
:10A57000C069C00616D504F06BFC401BB18A884246
:10A58000F5D90FE030681021C16104F061FC054687
:10A590003068C069C00605D504F05AFC401BB18A7A
:10A5A0008842F5D90120C107326813688B431360D4
:10A5B000F16E22040A4300021043F06601B0F0BDC0
:10A5C0004D200201034804A1844B04F06FFCC046F7
:10A5D00048930102502F0100666C6173685F646DDF
:10A5E000615F63616C6C6261636B0000A5A4000035
:10A5F000F0B581B000786E4DAA68824200D0D0E0FC
:10A6000001263002032942D16A6DAA66AB6DAC6A9D
:10A61000A418EB652C66AB6C5B1CAB646B6E934251
:10A6200035D95E30FFF7FEFA686CA96C02293AD37F
:10A63000814238D1E88C696D0818686500200621D0
:10A6400000F02CFD2868E96D81602F6D04F000FC9E
:10A6500004462868C069C00705D004F0F9FB001B58
:10A66000A98A8842F5D904F0F3FB04462A68D06928
:10A67000800706D504F0ECFB001BA98A8842F5D9B7
:10A680002A687420285C012841D0F10440E0F207D8
:10A690002B681C6894431C60EA6E09041143014353
:10A6A000E96601B0F0BD0229FBD38142F9D2E88C02
:10A6B000696D09186965A96D0818A865002006214B
:10A6C00000F0ECFC2868E96D8160EF8C04F0C0FBC1
:10A6D00004462868C069C00705D004F0B9FB001B18
:10A6E000A98A8842F5D904F0B3FB04462A68D069E8
:10A6F000800706D504F0ACFB001BA98A8842F5D977
:10A700002A687420285C012822D0F10421E0310558
:10A71000334B3B405918012802D01920400601E074
:10A720000720C00608182F4940185060002F0DD090
:10A7300004F08EFB04462A68D069800706D404F032
:10A7400087FB001BA98A8842F5D92A682B6D1FE078
:10A750003105234B3B40C918012802D0192040067F
:10A7600001E00720C00608181E4940185060002F5D
:10A770000DD004F06DFB04462A68D069800706D42A
:10A7800004F066FB001BA98A8842F5D92A68EB8C85
:10A79000296EA868144C00941432FFF723FB01B013
:10A7A000F0BD044804A10C4A0C4B04F07FFBC046EA
:10A7B00048930102502F0100666C6173685F646DFD
:10A7C000615F77726974655F6E62797465735F63E8
:10A7D000616C6C6261636B0072040000372F0100D2
:10A7E000FF3F000000808000F1A50000F0B587B0B9
:10A7F00004460126880E14D01546002A11D00F46B3
:10A800008120C004401B88420BD37C206043F04968
:10A8100008180590818C38460691F5F75BFC0029F5
:10A8200002D0304607B0F0BD28460699F5F752FC35
:10A830000029F6D1059880693E1A30460699F5F749
:10A8400049FC0746039670190190069E3146F5F7BC
:10A8500041FC0546C01B04900598006A02903146F1
:10A86000F5F738FC049981420FD20026BD42D8D9B1
:10A870002046394600F018FB2046FFF77DFD0028F2
:10A88000FAD17F1CAF42F3D3CBE700900398029D2F
:10A890002946F5F71FFC0646284670430399081A17
:10A8A000019800D0761C2946009D7543F5F712FCEF
:10A8B0000590029941430198401A03900699F5F7D3
:10A8C00009FC0490AF420BD22046394600F0ECFA66
:10A8D0002046FFF751FD0028FAD17F1CAF42F3D389
:10A8E00005988642069D009F0CD220463146FFF710
:10A8F0007BFC2046FFF740FD0028FAD1761C059826
:10A900008642F2D30398A84203D20026304607B00D
:10A91000F0BD059847430025E919204600F0C4FA28
:10A920002046FFF729FD0028FAD16D1C0026049867
:10A930008542F1D375E7C046F0B585B0002803D055
:10A940000124204605B0F0BD7822A14FB85C002854
:10A9500003D00024204605B0F0BD0492002905D0A4
:10A96000384614300CC90CC01CC91CC00020F86645
:10A9700015242046FFF77EF8204603F063FF386871
:10A980001021C16104F064FA04463868C169C9063F
:10A9900007D504F05DFA001BB98A8842F5D93868FA
:10A9A00000E0B98ABA7D1207120B5218F97DCB0765
:10A9B000DB08D2188B07DB0F5B05D218CB06DB0F49
:10A9C000DB05D2184B07DB0FDB06D2188B06DB0F3B
:10A9D0005B07D2180907C90F8907114301600024DA
:10A9E0000A21204600F05AFB3220FFF71BF908210C
:10A9F000204600F053FB04F02BFA05463868C16985
:10AA0000890606D404F024FA401BB98A8842F5D995
:10AA10003868017D0A46C23A5342534174257B553A
:10AA20000904027D12025118007D0B180220032632
:10AA300068A2314605F096FA785D0128039619D18F
:10AA4000F87D029000260621304600F027FB072102
:10AA5000304600F023FB012102988143785D0128F4
:10AA600047D138688901017506757521795C01291E
:10AA700038D048E00020032100F010FB04F0E8F992
:10AA800006463868C169890606D404F0E1F9801BDE
:10AA9000B98A8842F5D93868007D46080122F87DD8
:10AAA000014631431640C90701D0304036D00295E7
:10AAB000002506212846019200F0F0FA07210095B2
:10AAC000284600F0EBFA019846400298385C0128CD
:10AAD00013D13868B1010175009901757521795C50
:10AAE000012910D114307621795C4A424A41510043
:10AAF00008E038680675490003E038680099017578
:10AB0000710014300170374800687D21C900F5F7E5
:10AB1000E1FA28214143002000F092FA7720385CC6
:10AB2000012803D102200021FFF734F804F090F946
:10AB300006463868C069C00705D004F089F9801B53
:10AB4000B98A8842F5D904F083F906463868C169A4
:10AB5000890706D504F07CF9801BB98A8842F5D9AB
:10AB60003868D049816117203856002829D578687F
:10AB7000002816D40146039A91431C4A8B58850736
:10AB8000ED0EFF26AE40B3438026AE401E438E50EE
:10AB90001F210140012088401549086015490860BF
:10ABA0000FE08107C90EFF228A400F230340083BB4
:10ABB000039883430C481D58954380228A402A43BA
:10ABC0001A500120049978543861204605B0F0BD30
:10ABD000489301026A656465635F69642025780DA6
:10ABE0000A00000008E001021CED00E000E400E0C3
:10ABF00080E200E000E100E0F0B593B07C270A902D
:10AC000047439348C619980704D0F07D4024044078
:10AC100000D017E10125880E2ED0002B2CD08120EA
:10AC2000C004C01A884227D309920122EFF310848E
:10AC3000144002D1EFF3108072B630461030059008
:10AC40003069002506280891069310D80794144609
:10AC50008440E106490F04D161210C4203D015461E
:10AC600004E0022502E00221059B1960079C002CEC
:10AC700000D162B6002D02D0284613B0F0BD344694
:10AC800017347348C05910210491C16137461437F5
:10AC900004F0DEF805463068C069C00605D504F04A
:10ACA000D7F8401B39888842F5D92078400665D40A
:10ACB0000297B78C069C20463946F5F70BFA0790A9
:10ACC00039464143601A039035462435A74200D8DF
:10ACD00094E0039800281CD006210A9C204600F02E
:10ACE000DDF9288807994843089940183168886039
:10ACF00000272046039C394600F0D0F9079B099AAB
:10AD000028885843C0193168097D11547F1CA74217
:10AD1000F6D330680499C16104F09AF80446029DA4
:10AD20003068C069C00605D504F092F8001B298878
:10AD30008842F5D904F08CF804463068C069C00731
:10AD400005D004F085F8001B29888842F5D904F065
:10AD50007FF804463068C169890706D504F078F8A1
:10AD6000001B29888842F5D930680121059A1160B5
:10AD7000B24981610025284613B0F0BD03200025AB
:10AD8000089FF7650999316606997166B566F066A0
:10AD90000120C00731680A6802430A6006210A9C44
:10ADA000204600F07BF9306887602046294600F095
:10ADB00075F93A4F0BAA0A921BCF1BC21BCF1BC2BD
:10ADC000B48CF0680A99FEF79DFFF0683168344A48
:10ADD0000092069A944200D31446A3081431099AAB
:10ADE000FFF700F8B06E0019B066306E00193066DB
:10ADF000F06D0019F065284613B0F0BD002404E0A2
:10AE0000641C0798844200D363E706210A9800F087
:10AE100045F9288860430899401831688860002700
:10AE20000A98394600F03AF928880028099AE7D0AC
:10AE3000604310183168097DC1557F1C28888742FE
:10AE4000F6D3DDE7034804A1064A07A304F02EF871
:10AE500048930102502F0100666C6173685F726550
:10AE600061640000C603000054686520444D412021
:10AE700072656164206C656E6774682073686F75B5
:10AE80006C6420626520746865206D756C746970EF
:10AE90006C65206F6620340D0A000000C423010099
:10AEA000A5A40000000093EBF0B583B00D46044666
:10AEB0007C26464351488719F869B98CF5F70AF999
:10AEC000A84200D894E0019502940121EFF310808C
:10AED000084002D1EFF3108272B63C4610343B6951
:10AEE0000025062B0CD80A469A40D3065B0F06D1E4
:10AEF00061231A4277D00D46002803D003E00225D3
:10AF0000002800D162B6002D02D0284603B0F0BD63
:10AF100000943C462434394880591021C1613E4692
:10AF2000143603F095FF05463868C069C00605D59C
:10AF300003F08EFF401B31888842F5D90621029D1F
:10AF4000284600F0ABF8208801994143B8690918F8
:10AF500038688160172179563C461734002909D595
:10AF6000C16920220A43C2610121F966890502688C
:10AF70000A4302600421284600F090F8207840B28D
:10AF80002C4600250028C0D42B4800687D21C9002C
:10AF9000F5F7A0F820492D314143204600F050F844
:10AFA00003F056FF04463868C069C00705D003F0B7
:10AFB0004FFF001B31888842F5D903F049FF044652
:10AFC0003868C169890706D503F042FF001B318844
:10AFD0008842F5D938680121009A116017498161CA
:10AFE000284603B0F0BD0321216000288AD08AE7FB
:10AFF000034804A1084A09A303F058FF489301023B
:10B00000502F0100666C6173685F736563746F72C3
:10B010005F657261736500002B02000073656374E5
:10B020006F7220696478206973206F766572207270
:10B03000616E67650D0A000008E00102000093EBF5
:10B04000F0B583B001917C220290424353498C18A1
:10B050002546143503F0FCFE06460221029800F056
:10B060001DF803F0F5FE07462068C169890606D47D
:10B0700003F0EEFEC01B29888842F5D92068007DC8
:10B08000C00708D06420FEF7CDFD03F0E1FE801B71
:10B0900001998842E1D903B0F0BDC046F0B585B052
:10B0A000049104467C2060433C490F183D4614350A
:10B0B00003F0CEFE06463868C069C00705D003F02D
:10B0C000C7FE801B29888842F5D903F0C1FE0646D9
:10B0D0003868C069800705D503F0BAFE801B29884F
:10B0E0008842F5D91421049B5943DC2060432C4A43
:10B0F0001018039002914018018A8268C47C74265B
:10B10000BE5D012E0DD10191012B02990CD0012BB6
:10B110000DD07526BE5D012E0ED0019E072B0ED1DF
:10B120000EE00E4602990BE00222012BF1D13824E9
:10B130007526BE5D012EF0D10326072B00D0019E9F
:10B14000184B334024069207D20A1219D218039BD7
:10B150005958C907490C52184168CB071B0CD21823
:10B16000837C5B075B0BD218C0684007000A10188D
:10B170003A685060002E0ED001290CD103F068FE11
:10B1800004463868C069800705D403F061FE001BDF
:10B1900029888842F5D905B0F0BDC0464893010220
:10B1A0000C250100FF3F0000F0B59DB00D460126C3
:10B1B000890E2FD0002B2DD011928121C90410931C
:10B1C000C91AA94226D30121EFF310840C4002D101
:10B1D000EFF3108272B67C220F904243E74814923C
:10B1E0008718384610303B690026062B0DD80A46D2
:10B1F0009A40D3065B0F07D161231A4200D16FE357
:10B200000E46002C03D003E00226002C00D162B6CB
:10B21000002E02D030461DB0F0BD0290BD65002169
:10B22000139179651098401E12904019B964B9695C
:10B230000D916E1A1199B962FD6238637E63F98CC3
:10B240000E913046F4F746FF0446B8631298301862
:10B250000E9E3146F4F73EFF109B011B4A1CF8631B
:10B2600039647A64139A0029194608D07043591931
:10B270000D9BC91A0A1A7443581B801901193846C4
:10B2800048300E90384644300D90384640300B9090
:10B29000384626300590384658301390384654309A
:10B2A0001290F9643A651498B44908581021C161A4
:10B2B0003846143014903846503004903D464C3592
:10B2C00003F0C6FD04463868C069C00606D503F021
:10B2D000BFFD001B149909888842F4D9F87D400607
:10B2E0000C9500D574E201230E9803600D98016857
:10B2F00000290F9800D1CDE23A4674320A92DA045E
:10B3000007921A0509921922520606920722D206BE
:10B31000089216E09A4800687D21C900F4F7DAFE29
:10B32000109941430F9C2046FFF78AFE20460C9D52
:10B330000E9A11684B1C13600D9909688B4200D955
:10B34000A8E20B9A1268012A55D0002A00D0A8E082
:10B350002E6812990C6813990D6806211091FFF759
:10B360009DFE386885601198051903F071FD04464B
:10B370003868C069C00706D003F06AFD001B149945
:10B3800009888842F4D903F063FD04463868C1692E
:10B39000890707D503F05CFD001B149909888842D2
:10B3A000F4D938680A990A78012A089900D00699D0
:10B3B000012A099A00D0079A3346724C234013435E
:10B3C0000B4371490B434360002EA3D003F040FDB3
:10B3D00004463868C069800706D403F039FD001BB5
:10B3E000149909888842F4D93868297801756D1C48
:10B3F000761EFAD18EE7012B00D0C7E02E68129995
:10B400000C6813990D6806211091FFF747FE386804
:10B4100085601198051903F01BFD04463868C06962
:10B42000C00706D003F014FD001B14990988884258
:10B43000F4D903F00DFD04463868C169890707D5C2
:10B4400003F006FD001B149909888842F4D9386876
:10B450000A990A78012A089900D00699012A099ABE
:10B4600000D0079A3346474C234013430B434649C9
:10B470000B434360002E69D003F0EAFC04463868B1
:10B48000C069800706D403F0E3FC001B1499098807
:10B490008842F4D93868297801756D1C761EFAD176
:10B4A00054E0012B00D0C9E02E6812990C68139962
:10B4B0000D6806211091FFF7F1FD3868856011983D
:10B4C000051903F0C5FC04463868C069C00706D0FA
:10B4D00003F0BEFC001B149909888842F4D903F0DC
:10B4E000B7FC04463868C169890707D503F0B0FC8A
:10B4F000001B149909888842F4D938680A990A7897
:10B50000012A089900D00699012A099A00D0079AC1
:10B5100033461C4C234013430B431B490B434360EE
:10B52000002E13D003F094FC04463868C0698007ED
:10B5300006D403F08DFC001B149909888842F4D9C5
:10B540003868297801756D1C761EFAD10C480068A0
:10B550007D21C900F4F7BEFD109941430F9C2046A0
:10B56000FFF76EFD20460C9D2A68139B1968891809
:10B570001960129B196889181960D9E6489301026D
:10B5800008E00102FF3F0000008080008B4200D0F5
:10B59000CEE604990E6812990C6813990D6806217D
:10B5A0001091FFF77BFD386885601198051903F04D
:10B5B0004FFC04463868C069C00706D003F048FC59
:10B5C000001B149909888842F4D903F041FC044611
:10B5D0003868C169890707D503F03AFC001B149944
:10B5E00009888842F4D938680A990A78012A0899A2
:10B5F00000D00699012A099A00D0079A3346D44C04
:10B60000234013430B43D3490B434360002E00D127
:10B6100080E603F01DFC04463868C069800706D444
:10B6200003F016FC001B149909888842F4D9386885
:10B63000297801756D1C761EFAD16BE6129A126894
:10B64000119CA618139A15688B425FD104990C6857
:10B6500006210391FFF722FD3868856003F0F8FBAF
:10B6600005463868C069C00706D003F0F1FB401BEF
:10B67000149909888842F4D903F0EAFB10900C9DD4
:10B680003868C169890708D503F0E2FB1099401AB0
:10B69000149909888842F3D938680A990A78012AE6
:10B6A000089900D006991091012A099A00D0079AAA
:10B6B0002346A7490B40134310990B43A5490B435D
:10B6C0004360002C14D003F0C3FB10903868C069AD
:10B6D000800707D403F0BCFB1099401A149909881D
:10B6E0008842F3D9386831780175761C641EFAD126
:10B6F0009A4800687D21C900F4F7ECFC03994143A6
:10B700000F9C2046FFF79CFC204611E605990C880B
:10B7100006210391FFF7C2FC3868856003F098FBAF
:10B7200005463868C069C00706D003F091FB401B8E
:10B73000149909888842F4D903F08AFB10900C9D73
:10B740003868C169890708D503F082FB1099401A4F
:10B75000149909888842F3D938680A990A78012A25
:10B76000089900D006991091012A099A00D0079AE9
:10B77000234677490B40134310990B4375490B43FC
:10B780004360002C14D003F063FB10903868C0694C
:10B79000800707D403F05CFB1099401A14990988BC
:10B7A0008842F3D9386831780175761C641EFAD165
:10B7B0006A4800687D21C900F4F78CFC0399414375
:10B7C0000F9C2046FFF73CFC204605990A88CCE6F2
:10B7D0005E4815A90A4678C878C278C878C201259B
:10B7E000E8073A68136803431360B868FEF78AFAFB
:10B7F00002200026139C2168BA6AF9653A661099FE
:10B800007966BE66F8660C980068129A1168091885
:10B8100011600E9B19684A1C1A602268101820607B
:10B82000002900D0F6E410953846603013903C466D
:10B830005C3438460830129006210F98FFF72EFC32
:10B840003868216881600C980068119003F000FB53
:10B8500004463868C069C00706D003F0F9FA001B37
:10B86000149909888842F4D903F0F2FA0446109D2D
:10B870003A68D069800707D503F0EAFA001B1499EB
:10B8800009888842F4D93A687420385C01282DD0A0
:10B89000E9042CE003F0DCFA04463868C069C0070C
:10B8A00006D003F0D5FA001B149909888842F4D910
:10B8B00003F0CEFA04463868C169890707D503F05A
:10B8C000C7FA001B149909888842F4D93868012105
:10B8D000029A116022498161002630461DB0F0BDF8
:10B8E00004210160002C00D191E491E42905119C10
:10B8F000174B2340591801280C9D02D019204006EF
:10B9000001E00720C0060818124940185060002CBA
:10B910000ED003F09DFA04463A68D069800707D438
:10B9200003F096FA001B149909888842F4D93A6802
:10B930002B681398016812980068074C0094143221
:10B94000FEF750FA30461DB0F0BDC046842301001A
:10B95000FF3F000000808000F1A5000008E0010228
:10B96000000093EB3920C00001490968085870476E
:10B97000D4920102F0B5032920D8C0467944097950
:10B9800049008F4401080F15012181404F4B1B686E
:10B990005963D96212E0012181404C4B1B68196345
:10B9A000D9620BE001218140484B1B68596304E0D8
:10B9B00001218140454B1B6819639962830043490B
:10B9C000CB18DA608A68002A29D14A68002A16D47E
:10B9D000032314469C43174BE5589607F60EFF27A2
:10B9E000B740BD438027B7402F43E7501F23134084
:10B9F00001229A40104B1A60104B1A600FE0930717
:10BA0000DB0EFF259D400F241440083C0322944385
:10BA1000074AA658AE4380259D403543A5500122D4
:10BA2000824008680262886810438860F0BDC046A2
:10BA30001CED00E000E400E080E200E000E100E056
:10BA400010B501242046FEF715F8204602F0FAFE54
:10BA5000002010BD012181401C48006842688A43D3
:10BA600042607047194909680968C14001200840CF
:10BA70007047C046012181401448006842680A436B
:10BA800042607047012907D0002910D1012181406F
:10BA90000F4802680A430FE0012181400B4800680B
:10BAA0004368002A0DD00B434360016170470121B8
:10BAB0008140074802688A43026004480068416187
:10BAC00070478B43436001617047C046D8930102C1
:10BAD0000801004080B5114A1170114A10708001B0
:10BAE000C90101430F480078400108430E49097815
:10BAF000090101430D480078C00008430C4909784A
:10BB0000890001430B480078400008430A4909783E
:10BB10000143C8B2F8F7FAFD80BDC046F89E0102A5
:10BB2000B69601021D9001027CEA0102B1AD01024C
:10BB3000F99E01023CA301023DA3010201228240C1
:10BB40000548002903D0016811430160704701686E
:10BB5000914301607047C04600010040124A072827
:10BB600009D880000F238340814019401068984312
:10BB70000843106070470F280AD8800020380F2330
:10BB80008340814019405068984308435060704793
:10BB9000800040380F2383408140194090689843CB
:10BBA000084390607047C04634000040F0B543073A
:10BBB000DC0E0726A640C3089D000E4BEF187D68DB
:10BBC000B5433E1D002908D035600122824001297D
:10BBD0000CD1186810431860F0BD0121814018682D
:10BBE00088431860A24015433560F0BD1868904343
:10BBF0001860F0BD0C01004010B582B014460A4632
:10BC000001460498009301900820234600F092F822
:10BC100002B010BDB0B584B014460A46014608987B
:10BC200002250095019302900720234600F052F967
:10BC300004B0B0BD70B500285BD031490A783149F5
:10BC4000002A03D14A68012313434B6042880388CA
:10BC50001B049A180B46183B1A60828883891B04C0
:10BC60009B180C460C3C23600B46083B84681C6008
:10BC7000446903232340057CAD00EB188569AD07BB
:10BC80002D0D5B19457C2D035B19C569AE07B60AFE
:10BC90009B19867CB6059B190E1F3360036A122B15
:10BCA00004D107240C60541EA2410AE0032C05D1E4
:10BCB000012D03D807220A60012202E006220A6051
:10BCC0000122114C002525700F2464012034C57C0D
:10BCD0006D0225401B069B0BD218C3791B07DB0E98
:10BCE000D21880790007C00D101840191439086067
:10BCF00070BD064806A1862209A303F0D7F8C04606
:10BD0000F4CC010218100050F6CC01022D3C0100C9
:10BD10006C73705F656E67696E655F72756E00004B
:10BD2000506172616D65746572206973206E756C07
:10BD30006C000000F0B58BB0109E34043ED00D4670
:10BD4000D64C2140012701977F06B9423CD11146CC
:10BD50002140B9423FD11C40BC4243D1119902ACB1
:10BD60000027E781E780668027802782A774E17437
:10BD70009908A181A908A1800A90099708970797B7
:10BD8000900880B204902046FFF754FFAA4800783C
:10BD9000002801D00BB0F0BDAB480168C90708D13D
:10BDA0000168C90705D10168C90702D10168C9073F
:10BDB000F3D07F48019901700BB0F0BDB8480D4930
:10BDC000AF22C14B03F072F80095B5480949B02283
:10BDD000754B03F06BF80092B1480649B122724BE3
:10BDE00003F064F80093AE480249B2226E4B03F0B0
:10BDF0005DF8C046033C0100F0B58DB00392139E80
:10BE0000340446D00A46A54C2140012502956F0610
:10BE1000B94244D103992140B94247D11C40BC42A8
:10BE20004CD11499129D04ACE17429492182002758
:10BE3000E781E780668027809908A1819108A18029
:10BE40000B95012D01D16121CF43A7740C900220E5
:10BE50000A9009900398800880B206902046FFF768
:10BE6000E9FE75480078002801D00DB0F0BD764895
:10BE70000168C90708D10168C90705D10168C90768
:10BE800002D10168C907F3D04948029901700DB089
:10BE9000F0BD83480D49FB228B4B03F007F800925D
:10BEA0007F480A49FC22404B03F000F803980090B9
:10BEB0007B480649FD223C4B02F0F8FF009378488E
:10BEC0000249FE22384B02F0F1FFC046103C01004F
:10BED0008E8E0000F0B58BB0119E340447D00D4615
:10BEE0006E4C2140012701977F06B94245D111468A
:10BEF0002140B94248D11C40BC424CD11299109FFC
:10BF000002ACE174294921820021E181E18066804F
:10BF100021809908A181A908A1800997012F01D04A
:10BF2000712100E06121C943A1740A9003200890A7
:10BF30000790900880B204902046FFF77BFE3E48B1
:10BF40000078002801D00BB0F0BD3F480168C90758
:10BF500008D10168C90705D10168C90702D1016884
:10BF6000C907F3D01248019901700BB0F0BD4C48DD
:10BF70000C49D522544B02F099FF009548480949D5
:10BF8000D622094B02F092FF009245480549D7227C
:10BF9000054B02F08BFF009341480249D822024B27
:10BFA00002F084FF1F3C01004D3C0100868600002A
:10BFB000F6CC010210B582B014460A4601460020B4
:10BFC0000093019004202346FFF7B4FE02B010BD99
:10BFD00010B584B014460A46014600200090019333
:10BFE000029004202346FFF707FF04B010BD0000B5
:10BFF00070B50D46064604242046FDF73BFD20465D
:10C0000002F020FC0B4805600B480670002E0ED095
:10C010000A48016880220A437F218A430260012086
:10C0200000030749086007490860074804600020CA
:10C0300070BDC046F8CC0102F4CC01020CE400E073
:10C0400080E200E000E100E01C100050B0B582B0DA
:10C05000144602461148204001256D06A8420DD124
:10C06000180413D0174801600020009301900620A7
:10C0700011462346FFF75EFE02B0B0BD0094FF22DA
:10C080008C320748074908A302F010FFFF208C30CC
:10C09000421C034803490C4B02F008FF0300FCFF5D
:10C0A0002D3C0100F53B010044737420616464720F
:10C0B00065737320257820697320696E76616C69D9
:10C0C00064000000081000506B3C010080B582B095
:10C0D0000B46014600200092019003200A46FFF71C
:10C0E00029FE02B080BD0000002801D0042100E03C
:10C0F0000221C54A5172411E8841800103490A68E4
:10C1000040239A43101808607047C04650A0005062
:10C11000F0B583B002912E49CD7A0E7B7719874214
:10C120004FD908990191182545434126F604BF00CF
:10C13000BE19745B34490C4057033C199B07D90C5A
:10C140006418324B1B681B7A745375196C8803266C
:10C15000B60326409B079B0C9B193F2404401819EB
:10C16000029CA3061B0DC0186880012A184E13D824
:10C17000707B14224243307B5023434324011B191C
:10C180009A18F37AC0181C234343D01880081E4A1B
:10C19000104007430F432F800198686001F0D6FEDE
:10C1A000A860E8681A4908403030E860286908400B
:10C1B0002721715C4018286100F056FE686103B0C9
:10C1C000F0BDFF228832034803A108A302F06EFEEF
:10C1D000FCD10102BC3C01006D61635F63735F636E
:10C1E0006F6E7374727563740000000043532069AE
:10C1F0006E646578206973206F7665722072616E57
:10C2000067650D0A00000000FF070000449401026A
:10C210000000F0FF2820D84900220A547047C04689
:10C22000F0B581B0009314460D4607460626304609
:10C23000FDF720FC304602F005FB26211D4847543F
:10C240000021017041708171017181704171C17073
:10C25000C17102224272C16201634163816304734E
:10C260004273C572009A561C134A1680017241200F
:10C27000C00401214903F3F796FF502060432901D0
:10C28000081861198A00801818224A438018B2B22F
:10C290004A438018094940180949884204D200F0ED
:10C2A000B5F8002001B0F0BD064807A19A2209A305
:10C2B00002F0FCFDFCD10102F8D1010228000802C5
:10C2C00001200802BC3C01006D61635F696E697406
:10C2D00000000000454D206F766572666C6F770D2B
:10C2E0000A000000A448C179002901D0012070474C
:10C2F000007A411E88417047F0B583B002912A4907
:10C300004B7B834248D9CB7A0C7BE31818245C43DF
:10C310009B00E3184124E4041A19142401900546F3
:10C3200065430026565100925519EE882E4F0B4654
:10C330007A1C3240F54E3688497A711A2B4E0E40DF
:10C34000B618EE803740997BEF80AA88284F1740B7
:10C350004A424A4191007918264A8918A980264FF5
:10C360000F402D1D029801280AD124490E400921B1
:10C37000C902711869800121C9037918298000E078
:10C380002F800198444300980019074A918C4182FC
:10C39000118C018203B0F0BD3520C200034804A116
:10C3A00009A302F083FDC046FCD10102BC3C0100A0
:10C3B0006D61635F6C696E6B5F646573635F636F10
:10C3C0006E737472756374004C696E6B2064657370
:10C3D0006320696E646578206973206F76657220CA
:10C3E00072616E67650D0A00FFFBFFFFFF0300002F
:10C3F00003D0FFFFE80F0000EF1F0000FF830000E5
:10C40000BE4A506391637047FCD10102F0B581B020
:10C410004348CC21016003214160B8490A7BD30421
:10C42000404C1B19CC7AA218541E1C4318235343AA
:10C4300092009A184B7B14255D43521992012243B6
:10C44000012463061343436100228262C2620263D5
:10C4500042638263C26342650267334B1A605A606B
:10C460009A60324B1A601A619A61DC61304C1C622E
:10C47000304C251D1D6325460C3D5D632546283D3A
:10C480009D632D4EDE631C645C642C4D2F461C376F
:10C490009F642746143FDF64103C1C65284C5C6594
:10C4A000284C9C650C369E67274CA5634035E56398
:10C4B000DA651A665A669A66DA661A67234DDD6788
:10C4C00002258561224DC561C325AD03CD620A6396
:10C4D000D2435A601F4A1368FF25AB4326254D5DA2
:10C4E000AD072D0EEB1813601B4A102313601B4A77
:10C4F0001360272260238B5419498160C160016158
:10C5000021607D210901016641661649C164164911
:10C5100041641649016400F097FC01B0F0BDC046CB
:10C5200004A000500000F8FF94A0005034A1005077
:10C53000FF185A0030040040041000401C20004046
:10C540005430004060400040B8A100501400140076
:10C55000FF3F3FFF04E400E080E200E000E100E094
:10C56000DC05DC053F0270020133D007D007D0079D
:10C570002921C64A50547047FCD10102F0B58BB056
:10C58000079208910146C14FB8780991FFF7B4FEB0
:10C5900078793A7B79790691824200D89FE0FB7ADC
:10C5A0009A181823534392004124E104049152182D
:10C5B000D2187B7B14214B43D2185024604315586A
:10C5C00001230A93DB022E469E4316504E4B2B400E
:10C5D00005937D7B03914D433E7B7443F97A0B01B8
:10C5E0001B195B1971181C24029461435918A84B3C
:10C5F0001B88069C5C430919C904490D059BC91891
:10C60000115010180799416038787979089A00928A
:10C610000322099BFFF77CFDF87A397B09183878EB
:10C62000814263D983000993049AD45C0894F7216A
:10C630002140D154D1184D788E7836027619CB78B6
:10C640001B04F31807900A9886051E43330CCB7021
:10C65000FB7A387BBC784D709F4D3540039E664316
:10C66000C018029B4343981940029C4B03405C193D
:10C67000200A8870200CC870F023089D2B401B1DD9
:10C680003D7B0895FE7A099D5355C8700620079A90
:10C6900050438019089A801848701F22D202224005
:10C6A0000243100A88707879401C7871387B797958
:10C6B000814201D3002179713978491C3970F97AA6
:10C6C00008183978884201D80020387028200A9943
:10C6D0003954387A401C3872387A0BB0F0BDA72034
:10C6E0004200D2480649074B02F0E0FBA720420077
:10C6F0007A32CE487349744B02F0D8FBFCD1010268
:10C70000DC3C0100853C010000F0FFFFF8D1010294
:10C710000320000605490A6882430A600A6802434A
:10C720000A600348012101607047C0461C000040B8
:10C730001CA0005080B50120FDF752FC80BD000018
:10C74000F0B587B006930646504C607A504B1B8874
:10C75000181A0C9DA84200DC89E00F460592012EB4
:10C7600006D156480021C1620169554A8918016005
:10C77000A0783146FFF7C0FDE078E178069A2B46B5
:10C7800000F0AEF82078E178009700220692334658
:10C79000FFF7BEFCE07A217B0818217888426ED929
:10C7A0004120C20404918800815C0391F7250D406B
:10C7B000029285544549455C4549465C36027619E6
:10C7C0004449475C3F04F6190127BF0537433E0C37
:10C7D0004654E67A217BA3783C4A85543E4D3D4041
:10C7E00014275F4389191C234B43D91949023B4B3A
:10C7F0000B405D19290A364BC1542E0C354946545D
:10C80000F02703990F400599002900D13F1D217B96
:10C81000E37A029A87542F4A86540622049E724372
:10C82000D2185118294A81541F22D20215400D43B3
:10C83000290A274A8154E078401CE070E07AE178C8
:10C84000814201D30699E1702178491C2170217B36
:10C8500008182178884201D806982070E079401C99
:10C86000E071A07A401CA072E07907B0F0BD3920D9
:10C87000C2001632074808A109A302F017FB3920AD
:10C88000C20004480F49104B02F010FBFCD101021A
:10C89000F8D10102BC3C01006D61635F7478000057
:10C8A0004D4143205458206C656E206973206F768B
:10C8B00065722072616E67650D0A00000804004011
:10C8C00090D00300F23C0100A33C010001000802EB
:10C8D0000200080203000802FF07C0FF00F83F0043
:10C8E000F0B589B00893019204914F4DEF7A8742D9
:10C8F00000D891E0297B502632464A434124E30484
:10C900000693D218CC19A10051181822059254434D
:10C910000A19697B142307935943531802900001A5
:10C92000195804460390504A0A40A97AC90251187E
:10C9300008988205D2088A181A514C4911402A7B5E
:10C9400000965643384CE57A2C0106982418A7190E
:10C95000354E5419A5007D19059844432819747B58
:10C96000079D6C430519049FD2194148048854431C
:10C970002A19089CD204520D51181D4603981950CB
:10C9800000F07CFA0146707A001902043E460CD091
:10C9900080B2C000002900D1801E029FA52149005D
:10C9A000F3F798FB1F21014001E00021029F3801AD
:10C9B0002818427983791B029A18C3791B04D2186C
:10C9C0002C4B1340437109045918090CC171002CF8
:10C9D00020D0154835460646007B009B4343F17A3C
:10C9E0000A01069F3A43D21841188B00D218059BC2
:10C9F0004B43D118727B079B5343C91840191C4AFB
:10CA00001288424388180199884203D0019922462E
:10CA1000F3F7B0FB09B0F0BDFF225C32034804A17C
:10CA200009A302F043FAC046FCD10102BC3C01005C
:10CA30006D61635F74785F646573635F636F6E736A
:10CA400074727563740000005458204445534320A9
:10CA5000696E646578206973206F766572207261F3
:10CA60006E67650D0A000000FF0700E000F8FFFF99
:10CA7000F8D10102EFFFE00082B0FCF717FE0520BD
:10CA800000252946FFF76AF806202946FFF766F8D1
:10CA90000A202946FFF762F809202946FFF75EF8C9
:10CAA0000124204603F0E0FB284603F0DDFBFCF701
:10CAB00039FE2046FCF72CFE01F044FE01F03CFE5E
:10CAC0006E4801686E480068890308D4032109078D
:10CAD00008402107884202D0FCF7B6FD06E0FCF7CB
:10CAE000E9F8FCF7C9FD0020FDF7C0FCFCF754FE97
:10CAF0000025284604F0F8FC032662A230463146A1
:10CB000003F030FA30462946FBF7DEFBF7F7FCFE70
:10CB1000FAF720FEFEF794FF604F381DFCF7A2FBEA
:10CB2000F7F7EAFBF6F726FBF7F77BFE042630461D
:10CB30002946FFF713F8304621462A46FEF7A2FFA2
:10CB4000052230462146FFF731F820462146FEF700
:10CB5000C1FF534E30462830524A01902146FCF71F
:10CB6000F3FAFAF7D5F8A2024F49504B204603F0EA
:10CB700079FE01F0C5FBF6F7EBFA4D4A2046214657
:10CB800002F0AAF84B4802F0D7F84B48FCF746FDF4
:10CB90004A48FCF725FD01E0FBF7D8F91120FEF724
:10CBA00061FF3063B878002803D1F7F7A5FE0028AD
:10CBB00017D0707A012808D1022070720320014634
:10CBC0003FA203F0CFF9FAF7D3FCFCF753FCF7F7D9
:10CBD000A7FEF6F7B9FEF7F7E9F8FAF7C9FDFCF793
:10CBE00027FCB07A002827D0B5723079411C31710A
:10CBF0003D2806D30020307101210198294AFCF715
:10CC0000A3FAFAF75FFF34480470F7F775FE0028BF
:10CC100002D0BD70757107E070791E28214600D3DF
:10CC20002946B970401C7071F7F7FCF87F20C105E8
:10CC3000F069F3F790FBF0610B20FEF713FF3978F2
:10CC400000280DD00029A7D1012024490870387090
:10CC500000202349087003F0E1FAFBF777F99DE71C
:10CC6000012999D1002038705749C8831B490870A1
:10CC700001201B49087003F0B1FA8DE7180000404D
:10CC8000300001405557422073696D706C65206516
:10CC900078616D706C650D0A000000001C90010247
:10CCA000989901023D900000F8CD01029D0A010013
:10CCB00079EC00007C3F00000DCD0000898D000064
:10CCC000D4CBD0D0536F636B65745F52656376418C
:10CCD0006C6C0D0A00000000B6960102189001026B
:10CCE00019900102014800687047C0460C000040DE
:10CCF00081B080B581B0039303AB009302F0ACFD2B
:10CD000001B080BC02BC01B008470000014800210E
:10CD1000C161704798990102F0B581B00026304694
:10CD20003146FDF709FE0125AC022649264F304663
:10CD30003A462346FDF760FF3988244881423ED0B9
:10CD400064217E5262217E5260217E524422BE5274
:10CD5000FD87BD8778227A8702223A874322FA86A6
:10CD6000BE83FE811A4ABA817E810A223A81C82294
:10CD7000FA80184ABA803880FE8306203885F98404
:10CD8000FF20123078848730B88450203E523A8396
:10CD9000EFF3108072B630463146FDF7CDFD002826
:10CDA0000CD12A0300263046064D2946FDF71EFD0C
:10CDB000054A304629462346FEF7F6F962B601B029
:10CDC000F0BDC04600E002044AA90102AA550000D5
:10CDD000E1FF0000341200000020704710B500246D
:10CDE000002809D0002905D003464A000348194607
:10CDF000F3F7C0F9204610BDE04310BD3C9301029B
:10CE0000014600200A2901DAC0437047014A118017
:10CE10007047C046C49301020020704780B5018866
:10CE2000064A11808178064A1170C178054A11704E
:10CE30000079FCF743FB002080BDC0462E94010220
:10CE400030940102ACD20102044805490160152169
:10CE500009044160034981607047C0469C3000402E
:10CE60004100080034000700074800684069704727
:10CE7000FD20400004490968085C704702480068CA
:10CE80006221405C7047C0464494010210B50648D8
:10CE90000468064800686421F3F732F90221C943A7
:10CEA0004143081910BDC046B0D20102B4D20102FC
:10CEB0000A491A220A600A4948704878FF21090283
:10CEC000084A13688B43800380B2C018106006487C
:10CED000202101600548016000207047702000405B
:10CEE0003494010204E400E080E200E000E100E0AC
:10CEF000F0B5A9B016460F460546C648002B0246B7
:10CF000000D01A463921CC003D21C9005118119199
:10CF10008242189206D001204202BE491898F3F7C7
:10CF200029F9189A6120111913910E21119C0A9167
:10CF3000A170002F0D9501D00A2100E0092159238D
:10CF400017938300E1707842784113990870307824
:10CF500010901070F17AE17471785170B778977011
:10CF6000F178D1703579157174795471B179917105
:10CF7000F179D171317A1172717A5172B17A9172FB
:10CF80007E1EF0B200210328169106D870B28000F0
:10CF9000A1A210586A00805A16901798820018981B
:10CFA000C0181490F81E022804D3012E084604D895
:10CFB0009D4800E09D48031918781290189DA81804
:10CFC00017902846303015902C4656346D2080003E
:10CFD0002950974A974B149E33627262B362F26291
:10CFE0003176F182139B597009229A70281841609A
:10CFF0008160C1600161109880008F490858F3F783
:10D0000047FD012F10900F9104D0022F05D17F21F1
:10D010007E2004E07C217B2001E05B215A20159DCD
:10D02000A984207003200C90A080012666701F2028
:10D030000B90A8821820A8740A46083A179BDA7643
:10D04000169B129AD2184A439100189A9163B7021C
:10D05000791E8B420E9109D978486080342068840B
:10D060007748288277481399088339E07F2B10DDB1
:10D07000802B18D031028B421BD071028B4227D1FA
:10D080006E49618068846F4813990883CF20C0007F
:10D0900025E0202B17D0402B1AD16848608004204F
:10D0A000688469481BE0654860800620688467489A
:10D0B00015E06248608010206884624813990883F4
:10D0C000C520C0000BE0624860800220688404E054
:10D0D00004206884812040006080FF200230288284
:10D0E000104600F0D7FE1298102806D0402808D12C
:10D0F00008201499C876072000E00420179988704A
:10D1000002E017980C9981701898169A8078C11EC1
:10D1100002290CD3022811D001280CD12672BA4260
:10D1200000D900266672BA4213D8F44812E00D20E6
:10D130000002119908800120800201E00C98000291
:10D140002081BA4201D8EE4800E0FA2017998860A1
:10D150000EE0FA201799886013980078002811993A
:10D1600001D0E8484880E848139A1083E7480880CF
:10D17000A88CF3F7EFFB0026E54B3246F3F772FA83
:10D1800002460B46E3493046F3F7D4FAE24B324607
:10D19000F3F768FAF3F730FC0746E080DF493046E2
:10D1A000109A0F9BF3F7C6FADD4B3246F3F75AFAA3
:10D1B000F3F722FC78434042800B608116990E9869
:10D1C000814208D90C20149FB872D64817998883D9
:10D1D0001220189A0EE0480A189A149F01D00D20C8
:10D1E00003E0080A00D1DBE20A98B872CE4817992A
:10D1F00088831220F872D078052844D878440079C2
:10D20000400087440227402C3339C848B881C848B9
:10D210002FE0C046D49001023423010034230100E2
:10D220004423010044230100242001002B2001009D
:10D230003075000010270000E42001000502000006
:10D24000FF060000040800000A0400003604000085
:10D2500003020000B748F881B748388013E0B748A8
:10D26000F881B7483882B74838600CE0B448B881D4
:10D27000B5481799C88306E0B4487882B448B880A6
:10D280000B9800069064AE483881A748F880B148F2
:10D2900002882A84B0480078E874B0480078119F6A
:10D2A0007875387D139000285ED0AD490A68102348
:10D2B000DA413A600A794B79CF8867801B029A1865
:10D2C0006A840A7A4B7A8F7AC87A0D7B65701B0262
:10D2D0009A183B04D21800061018179FF860487B74
:10D2E0008A7BCB7B3B77120210186081087C7877B1
:10D2F000487C149A9072887CD072C87C159B1874F4
:10D30000087D5874487D11909874C87D0A7E120279
:10D3100012181A84887DD87418464B7EC375887E8F
:10D32000CD7E2D022818B880087F4D7F2D02281849
:10D33000F880887FB877C87FF8772020085C149D34
:10D3400028732120085C68732A20085C2A314D78F4
:10D350002D0228188D782D044019C9780906401827
:10D3600018998864119801E0EB7DA87C7D498B7049
:10D370000A8080001F38C882C883139800281FD0F5
:10D3800022227748825C034622335B781B029A187C
:10D390000A842422825C034624335B781B029A1899
:10D3A000CA842622825C034626335B781B029A18C5
:10D3B0008A832822825C2830407800028018888482
:10D3C0006948032569A2294602F0CCFD189F3878E8
:10D3D00014907B78B8780F90FA78B8791390F87930
:10D3E0001190387A1090787AB97A08900991009360
:10D3F0000F98019002921698039012980490139837
:10D4000005901198069010980790FAA2F8482946BE
:10D41000149B02F0A7FD3D46643580212846F2F7B3
:10D42000C2FEB878C11E02290ED3012800D18FE1B7
:10D43000022800D0ABE11691149078787F225043F7
:10D44000F7494018F74907E01691149078785B2265
:10D450005043F1494018F14941182846F2F78AFE35
:10D460000D9D1898C6870E34324602E0641C0F2AC0
:10D470000ADA21780029F9D0491C8907C90F91409F
:10D480000E43C687521CF1E71699022907D3149957
:10D49000491E012900D97DE14279D24901E0427952
:10D4A000CF4989180C78002D00D177E1C1790E9110
:10D4B000032900D94AE14279062A00D979E14921B4
:10D4C000890041181191E43010900E98401E12907E
:10D4D00019A800190F9000231392149403E01898D0
:10D4E000290600D15AE1052A5AD8C0467A44127951
:10D4F00052009744455C728598ABC0468813000083
:10D50000E20400000C080000060A0000040F0000FE
:10D510000000104130C1BD41000070400000F040EB
:10D520000000D041120C0000140B00001212000089
:10D53000140E00000E160000130D0000121600005D
:10D540000E120000140B0E0A120800001016000044
:10D550000E0B00002E94010230940102ACD20102A5
:10D56000B8D201029C940102010800004361736576
:10D5700020706172616D65746572733A200D0A00E6
:10D580001693DFB2002F04D019A801223946F2F712
:10D5900003FE002C00D191E019A8C019BB498AE014
:10D5A000E8B2022867D00027022867D06BE00E9807
:10D5B000022872D1E8B2022800D103461693DFB2E6
:10D5C000002F04D019A801223946F2F7E5FD002CFE
:10D5D00074D019A8C019ACA16DE0E8B2022800D13E
:10D5E00004231693DFB2002F04D019A80122394674
:10D5F000F2F7D2FD002C61D019A8C0199FA15AE002
:10D60000E8B2022800D106231693DFB2002F04D01F
:10D6100019A801223946F2F7BFFD002C4ED019A8F7
:10D62000C01992A147E0E8B2022800D10C2316935A
:10D63000DFB2002F04D019A801223946F2F7ACFD61
:10D64000002C3BD019A8C019874934E0E8B2811EEC
:10D650004A424A419700022804D119A801223946BA
:10D66000F2F79AFD002C16D019A8C0197CA1224609
:10D67000F2F780FD0FE00627022804D119A8012245
:10D680003946F2F789FD002C05D019A8C019804948
:10D690002246F2F76FFD169710E01693DFB2002FC7
:10D6A00004D019A801223946F2F776FD002C05D0E6
:10D6B00019A8C01973492246F2F75CFD3C193F2CAA
:10D6C00005D80F98C0194021091BF2F76CFD12987C
:10D6D0000228189801D2002002E0C078411E88413B
:10D6E00015990870611E2E46E8B202280CD1179ACF
:10D6F000517019A9119AB8C9B8C2B8C9B8C2B8C985
:10D70000B8C2B8C9B8C20DE0179A117019A9109A19
:10D71000B8C9B8C2B8C9B8C2B8C9B8C2B8C9B8C21D
:10D72000C10709D180073546149C139A169B00D473
:10D73000D5E602208543D2E6FE20354605401898FE
:10D74000149C139A169B290628D0CCE637A231E008
:10D750001691149078780B994143334808181F3874
:10D760006F21C9430D9D7A180378D427D355437888
:10D77000D827D3558378DC27D355002900D170E60C
:10D78000C378E027D3551031001D189FEBE7012027
:10D79000404A10E00024002D00D087E629B0F0BDFB
:10D7A00080290ED30F20B872104817998883102053
:10D7B00020E525A20120014602F0D4FB189829B0EB
:10D7C000F0BD1020402904D3B8720849179B9983F3
:10D7D00010E5B87204481799888314200AE5C046FA
:10D7E0002B20010024200100150F0000140B000065
:10D7F000010800002564202564202564202564207C
:10D8000025642025642025642025642025642025A6
:10D81000642025640D0A0000784601001DF7FFFF13
:10D82000903D010089FBFFFF804501007472785F25
:10D830006D6F646520706172616D657465722065DD
:10D8400072726F720D0A00004E736664207061720E
:10D85000616D65746572206572726F720D0A0000E9
:10D86000FFFFFFFF01FF0000E4230100FFFFFFFFB8
:10D87000FF0101FFFF01FF01FFFF01FFFFFFFF01AC
:10D88000FFFF01FFD0290100FFFF01FF0424010079
:10D89000542301002E3D0100002800D10148064913
:10D8A00008607047D4900102F0B586B0002805D119
:10D8B0000148006802E0C046449401023121C900D9
:10D8C000049141188A791F231A40CD79ED06AD0DD8
:10D8D000AA180D7AED066D0C52194D7AED062D0B36
:10D8E00052198D7AED06ED095219CD7AED06AD0883
:10D8F00052194D7CED075219BD4C22600A7B1A402B
:10D900004E7BF606B60DB2188E7BF606760C921993
:10D91000CE7BF606360B92190E79F606F6099219A9
:10D920004E79F606B608921962604A6AB14D2A40ED
:10D93000A2608A6A2A40E2602D22D20087183A7ECD
:10D940001A4003937E7EF606B60DB218BE7EF6062A
:10D95000760C9219FE7EF606360B92193E7FF6067D
:10D96000F60992197E7FF606B60892190E7CF60724
:10D9700092192261BA7F1A400597FE7FF606B60D0E
:10D98000B218049BC35CDB065B0CD2184B78DB0639
:10D990001B0BD2188B78DB06DB09D218CB78DB06A1
:10D9A0009B08D2186261CA692A40A2610A6A2A40A9
:10D9B000E2618A7C01252A40CB7CDB079B0F9A1809
:10D9C0000B7DDB075B0FD2184B7D9B07DB0ED2185C
:10D9D0008B7DDB079B0ED218CB7D1B079B0D9A1806
:10D9E0000B7E1B079B0CD2184B7E5B06DB0A134396
:10D9F0008A7E520612091A43CB7E5B075B081343EB
:10DA00002362CA6A62620A6BA2624A6BE2628A6B32
:10DA100022633922D200835C1E462E4066635E423A
:10DA20005E41B304AE04744F3C68B443E3183B60FA
:10DA300083185A782A409C782407E40EA2188C8F09
:10DA40006401A2186D4C1440C98FC905490A09190F
:10DA5000DA78D207120A89181A7912071209891876
:10DA60005A79D207D2088918FB4EB1639968F163DD
:10DA7000997904952940DA79D207920F51181A7BC7
:10DA80005207D20E89185A7BD206920D51189A7BF2
:10DA90005207D20C8918DA7BD206920B89181A7CAD
:10DAA000D206520A89185A7C520792090A43997C75
:10DAB000C906490851183164D97C039A11401A7D6E
:10DAC000D206920D51185A7DD206520C89189A7DB1
:10DAD000D206120B8918DA7DD206D2098918716430
:10DAE000197E0F2421405A7E120151189A7E12038A
:10DAF0008918DA7E1207120A51181A7F12071209C2
:10DB000089185A7F12078918B164997F01942140BE
:10DB1000DA7F1207120E51183D22D200835C5B0798
:10DB20005B0D5918841862781207520C8918A27874
:10DB3000D206120B8918E278D206D2098918F1644C
:10DB4000217907220A406179C9008918A279520611
:10DB5000920B5118E2799207120B8918227AD20798
:10DB60008A18BF490A60627AA37A1B029A18E37A7C
:10DB70001B04D2184A60E289BA4B13400394228AEC
:10DB8000D2049209D2188A6003463033598CB64ABF
:10DB9000114002939A8CD205D20A51185622825C07
:10DBA00012068918B14D2960014656314A788C78A1
:10DBB0002402A2188C8864056409A218CC78240772
:10DBC00012196A60CA880C7AA407A40BA2184C7AAE
:10DBD0006407E40A1219AA604989E96049218900A9
:10DBE0004118FF226632821800921035002207E0A9
:10DBF00000300040FFFFFF0004040040FF3F000032
:10DC000084186427E65D03273E406523E35C9B0799
:10DC10001B0F9B196626A65DB607B60EF31867267E
:10DC2000A65DB601F318DBB26826A65DB607B60D91
:10DC3000F3186926A65DB607360DF3186A26A65DA9
:10DC4000B607B60CF3186B26A65DB607360CF318AC
:10DC50006C26A65DB607B60BF3186D26A65DB60753
:10DC6000360BF3186E26A65DB607B60AF3186F26B4
:10DC7000A65DB607360AF3187026A65DB607B60984
:10DC8000F3187126A65DB6073609F3187226A65D4D
:10DC9000B607B608F3187326A45DA407E31808C5F1
:10DCA0001032802AACD1019AD243704EB4180B784E
:10DCB0003B404D78AD072D0FEB188D78AD07AD0EBD
:10DCC000EB18CD78AD01EB18DBB20D79AD07AD0DDA
:10DCD000EB184D79AD072D0DEB188D79AD07AD0C17
:10DCE000EB18CD79AD072D0CEB180D7AAD07AD0B08
:10DCF000EB184D7AAD072D0BEB188D7AAD07AD0AF9
:10DD0000EB18CD7AAD072D0AEB180D7BAD07AD09E9
:10DD1000EB184D7BAD072D09EB188D7BAD07AD08DA
:10DD2000EB18CD7BAD07EB18A3641031121DBDD1EC
:10DD3000009B19785A785207520D51189A78D207D9
:10DD4000120D8918B164059B1968F164D97D5A6870
:10DD50001202511831659968454A0A40998A490565
:10DD600089187165D9683D4C2140B1651969214018
:10DD7000F165029E3178049D294082785207120F86
:10DD80005118C2799207920E8918427A9207920D21
:10DD90005118827A9207120D8918C27AD207920C12
:10DDA00089189A7DD207520C891872789207D20B83
:10DDB0008918B2781207D20A8918F2781207D209A4
:10DDC0008A182C490A60327C737C1B071B0D9A1839
:10DDD000B37C9B069B0BD218F37C1B079B0AD218C3
:10DDE000337DDB065B09D218737DDB071B09D21874
:10DDF0004A60B27D2A40C38F5B009A188A60826CA9
:10DE0000CA60C26C22400A61F27D7F231340328CCB
:10DE10005204520AD2184A6102698A614269CA618F
:10DE200082690A62C2694A62026A8A62426ACA6294
:10DE3000826A0A63C26A4A63039A927CD201121D03
:10DE40000A64027A3A40CA65808F074A1040086621
:10DE5000002006B0F0BDC04600300040FFFFFF00CC
:10DE60009C300040FF1F0000FF0300000040004006
:10DE7000FFFF1F000020004004480068806B8008FE
:10DE80000349096849004018093070474494010269
:10DE90001004004010B52D21C9004118027A032A50
:10DEA00004D10079002807D0082006E08378DA1E24
:10DEB000022A05D2032412E0142088601C203DE0D1
:10DEC000012B02D1C8228A6012E00479042C01D30C
:10DED000462404E0032C01D1322400E014248C6099
:10DEE0005B1E022B04D3022A10D24279154B01E0AB
:10DEF0004279154B9B181B78402B04D0102B06D170
:10DF00001423442405E02A233E2402E042793423EA
:10DF100048244B800C80022A06D0062A08D0052A05
:10DF200008D118224C2301E0142250230B8000E07A
:10DF30001C224A80C078042803D114204880642021
:10DF4000088010BD2B200100242001001348006828
:10DF50007047C04610B5104A107091700F490028E4
:10DF600013D050680861042048619078FF221202A3
:10DF70000B4B1C689443800380B200191860012089
:10DF80004007084A1060084A1060002008600749EE
:10DF900001220A6010BDC0463494010218040040FA
:10DFA0001CE400E080E200E000E100E070000040DE
:10DFB000F0B591B0002801D1C04800688778F91EFB
:10DFC000022913D3012F21D0022F3CD11021CA43A3
:10DFD00044782146193991423DD800970125B94A24
:10DFE00028462946234601F0BDFF53E10821CA43D4
:10DFF000447821462139914218D800970125B14A29
:10E0000028462946234601F0ADFF43E10821CA43D3
:10E01000447821460939914234D800970125A94A0C
:10E0200028462946234601F09DFF33E1032F3CD0CB
:10E03000042F43D1C3780125042B00D02DE10646DF
:10E040002A02042343E00125A6A2284629463B468E
:10E0500001F088FF1EE1C3780125052B0AD806468A
:10E060002A02284698401B21084230D10021052B66
:10E0700008462ED002200090914A2846294601F0F9
:10E0800071FF07E10646C3780021022B1ED3032B44
:10E090001CD0042B08460A461BD001250095884A4F
:10E0A0002846294601F05EFFF4E0C3780125032BE2
:10E0B00000D0FAE006462A02032308E0012583A2E5
:10E0C000284629463B4601F04DFFE3E00A46012180
:10E0D00048020F91592189007518FD2149007118D6
:10E0E0000291314662313F05D219641E1F27274035
:10E0F0005C013C191443044332795207D20C224389
:10E100002B789B065B0BD218B379DB071B0B1343F1
:10E110006D4D2B60F279032310931A40737A9B079D
:10E120009B0E9A18B37A5B07DB0D9A18F37ADB071C
:10E130009B0DD218337BDB075B0DD218737B1B075B
:10E140005B0CD218AA603269EA6072692A61B2690E
:10E150006A61F269AA61326AEA61726A2A62B26A23
:10E160006A620F980870F06AA8623F20C4432C3599
:10E170003046E4300F903046E5300E903046E630C1
:10E180000D903046E7300C903046E8300B9030462A
:10E19000E9300A903046EA3009903046EB3008907A
:10E1A0003046EC3007903046ED3006903046EE3089
:10E1B00005903046EF3004903046F03003903746FB
:10E1C000F1373046F230F3360F990A194021525C8C
:10E1D000109B1A400E9B1B195B5C9B071B0F9A1828
:10E1E0000D9B1B195B5C9B079B0E9A180C9B1B19C4
:10E1F0005B5C9B019A18D2B20B9B1B195B5C9B0763
:10E200009B0D9A180A9B1B195B5C9B071B0D9A18A8
:10E21000099B1B195B5C9B079B0C9A18089B1B199D
:10E220005B5C9B071B0C9A18079B1B195B5C9B078D
:10E230009B0B9A18069B1B195B5C9B071B0B9A1880
:10E24000059B1B195B5C9B079B0A9A18049B1B1977
:10E250005B5C9B071B0A9A18039B1B195B5C9B0763
:10E260009B099A183B195B5C9B071B099A180319B9
:10E270005B5C9B079B089A183319595C89078918BE
:10E2800002C51034A0D102980078042101430E4841
:10E29000C1630025284611B0F0BD04200090084A53
:10E2A0002846294601F05EFEF4E703200090044A68
:10E2B0002846294601F056FEECE7C0464494010288
:10E2C000033D0100493D010000100040556E6465AA
:10E2D00066696E6564206D65616E2050524620252A
:10E2E000640D0A00496E76616C6964206D65616E2B
:10E2F000205052462025640D0A00000070477047E8
:10E3000080B50E490E480246083A1268920000D4C1
:10E31000603142680A4342600A490A6808239A4306
:10E320000A60091F012252040A600321890402685D
:10E330008A430260FBF720FA80BDC04620000080BF
:10E340002800004004020040B0B5032000072D491A
:10E350000A688243012568071018086000242046D7
:10E36000FFF7CDFF2046FFF7C9FFEFF310802840ED
:10E3700002D1EFF3108172B68021C943224A53685B
:10E380000B40536093680B409360D3680B40D3609D
:10E3900013690B40136153690B405361002800D18E
:10E3A00062B6B0BD70B50C4603210907154A136863
:10E3B0000B4313600122EFF31081114002D1EFF300
:10E3C000108272B68025EA430F4B5E6816405E608D
:10E3D0009E682E439E60DD681540DD601D69154016
:10E3E0001D615D6915405D61002900D162B600289C
:10E3F00002D00120FFF783FF002C02D00120FFF79D
:10E400007DFF70BD00040040D89501020D4A00292F
:10E4100007D001290BD10121814010688843106089
:10E4200007E00121814010680843106001E00121EC
:10E430008140101F02680A430121C907114301608E
:10E440007047C04644000040032804D840000649F5
:10E45000085A00B27047002000B27047032802D863
:10E460004000014A11527047E6D201029E490870ED
:10E470007047C04670B58AB00C460546FF20FC3098
:10E48000A8490E68315C59208000335CB27830783E
:10E4900008AE069609AE05960C4E04962126760621
:10E4A00003960B4E0296012601960E2600965B1CE3
:10E4B000DBB2F7F7B3FB0998F2F770FA2870089807
:10E4C000F2F76CFA20700AB070BDC046000020411F
:10E4D00000000443F0B58BB00446457C82480078C8
:10E4E0008249002822D000200880814A1080814B78
:10E4F00001269E761E830A907F4800787F4E3678EC
:10E500006DB205957E4D04957E4D03950AAD02953D
:10E510007D4D01950096F7F7BFF80A9D1120205612
:10E520007A497B4A00F02AFC064626E000260E8047
:10E530006F4A16806F4B01209876188309966E48B3
:10E5400000786E4F3F786DB205956D4D04956D4D19
:10E55000039509AD02956C4D01950097F7F79CF86E
:10E56000099D112021567F20C00500900190029640
:10E57000664A674B3046F8F7E3F943200106284620
:10E58000F1F742FFF2F70AFA089062480078002893
:10E5900024D05120800060494A7D42438D185F4855
:10E5A0000068A8642F46403750480078B874504837
:10E5B0000078F874554800783875554800787875B3
:10E5C00057480078F87550480069F2F7E7F9B875D0
:10E5D00052484069E8644C4800686864FF20FE3097
:10E5E00050490968085C3922D2008918022812D3E0
:10E5F00003D04E48007801280DD14B4806604348AF
:10E6000000883A4A108042480088394A1080092020
:10E610000790089605E04448089A02603548C08B88
:10E6200007900B780022002B01D0114600E0D14367
:10E630000125002B01D0042300E0EB43A67AAD1B9B
:10E64000EE175B1971416568AE0F277AAD00ED19C1
:10E650005641677A3F1FF817ED1970414000EE0FE1
:10E6600080196D00EB1848418001990E41189801FE
:10E6700027239B02C31A91411D4805881B48008827
:10E68000854201D00798421B10202056C001194D29
:10E690002D8C032D07D1E468E5176D0A6419E41584
:10E6A0000519EC170FE0E468E5176D0A6519EC171A
:10E6B000ED15C6174519744197B2002F00D03446A6
:10E6C000002F00D00546581BA141130409D012B2F7
:10E6D000D2015242D31780185941089BDA17C01A49
:10E6E00091410BB0F0BDC046C693010254AD01028A
:10E6F00052AD01029C940102C5900102C490010236
:10E7000040A301023CA1010258AD0102A2AD0102E9
:10E71000A0AD01020CA7010244A401026420004044
:10E7200050AD0102449401024CAD0102B0AD0102B2
:10E73000C10D4002803070470120C0071B490860AE
:10E740007047C04610B519480068C10710D181074D
:10E7500011D4410712D4010713D4C10614D4810681
:10E7600015D4410616D48021084016D031A215E0F8
:10E7700001240FA213E0022411A210E0032414A22A
:10E780000DE0042416A20AE0052419A207E00624DD
:10E790001CA204E0072421A201E0254A040902206A
:10E7A000032101F0DFFB204610BDC0465C000040A5
:10E7B000526573657420627920504F520D0A000033
:10E7C000526573657420627920424F520D0A000031
:10E7D00052657365742062792050494E0D0A00001D
:10E7E0005265736574206279205744540D0A000005
:10E7F0005265736574206279204C4F434B55500D20
:10E800000A00000052657365742062792053572016
:10E810005265626F6F740D0A0000000052657365E7
:10E8200074206279205359535245510D0A0000005B
:10E83000AE2F0100526573657420627920445644FE
:10E84000440D0A0001218140044A1F2802D01068AB
:10E850008843106010680843106070471C00004037
:10E86000F0B583B0029104469949F1F733FC0546AF
:10E87000984901942046F1F72DFC9749461897498D
:10E88000714300956F189649441864212046F1F7AA
:10E8900021FC3818A108471A92492046F1F730FCAC
:10E8A000381891494518914F05D464213046F1F745
:10E8B00011FC0C4614E0A6B264213046F1F70AFCC4
:10E8C000B7204000A20701D1002907D1884B73432C
:10E8D0000422D341874A934200D3401E0C46451977
:10E8E0000098474302980680192001013046F1F74D
:10E8F000F1FB2A461F3A284600DB1046019BFF1811
:10E90000B30705D1002C03D01F2D05DA0120C5E087
:10E910001F2D0BDA0120C1E005461D3D034600DB3B
:10E920002B461C2808DC02201546B7E000290CD035
:10E930001C21451A0CD50CE019461F39184600DB7E
:10E9400008461F2B1DDA0320A8E01D21451A00D41C
:10E950002846002D08D401461F39024600DB0A462E
:10E960001F2804DA032099E00220154696E0154698
:10E970001E3D104600DB28461E2A0CDA04200D46F8
:10E980008CE005461E3D024600DB2A461E280BDAB7
:10E9900004200D4682E001461F39024600DB0A468C
:10E9A0001F280ADA052079E011461F39104600DBDE
:10E9B00008461F2A0BDA052070E015461E3D10465A
:10E9C00000DB28461E2A0CDA06200D4666E00546C6
:10E9D0001E3D024600DB2A461E280BDA06200D46A5
:10E9E0005CE001461F39024600DB0A461F280ADAAE
:10E9F000072053E011461F39104600DB08461F2A46
:10EA00000BDA07204AE015461F3D134600DB2B4674
:10EA10001F2A0CDA08200D4640E005461F3D02463D
:10EA200000DB2A461F280BDA08200D4636E019467F
:10EA30001E39184600DB08461E2B0ADA09202DE095
:10EA400011461E39104600DB08461E2A0BDA092043
:10EA500024E01F28054601DB05461F3D1F280CDA70
:10EA60000A200D461AE01F28054601DB05461F3D1A
:10EA70001F2806DA0A200D4610E01E2D05DB0C20AB
:10EA800004E01E2D06DB0C2005E00B201E2D05DB0F
:10EA90001E3D03E00B201E2D00DB1E3D029EB070CC
:10EAA000681CF070E12001013846F1F713FB30716A
:10EAB000C0B211494143CC193C212046F1F70AFB71
:10EAC00070713B21C94341430819B07103B0F0BDD7
:10EAD000805101008033E101B207000093FEFFFF87
:10EAE000B107000070FEFFFFA7FA0A0080AEFEFF2C
:10EAF000295C8FC20BD7A300F0F1FFFFF0B581B006
:10EB00000446FFF721FCA08A00280FD0FFF71EFA69
:10EB10002249486122481C302CCC2CC02CCC2CC063
:10EB20002CCC2CC00020088201B0F0BDE08A1B4F25
:10EB30003882A1693A8A1B48F1F71CFB184D1C3535
:10EB4000204629464CC84CC14CC84CC14CC84CC18D
:10EB5000FFF7FCF978611248066AFFF78DF9301A61
:10EB6000F8622846FFF7B6FC06460D460E48007DC3
:10EB7000FFF76AFC0121F970617CB971796C491C5D
:10EB8000796481B2C90B401800B2C1174010301A25
:10EB9000B8658D41FD6501B0F0BDC046D098010259
:10EBA000089A0102F0D201023890010270B50446C1
:10EBB000FFF7CAFBA08A1B4E7082718A002908D019
:10EBC000B0820220707100203082FFF7BFF9F0613F
:10EBD00070BDE08A3082A169328A1348F1F7CAFA1F
:10EBE0002046FFF777FC05460C461048007BFFF7F0
:10EBF0002BFC81B2C90B401800B2C1174010281A73
:10EC000030668C417466FFF7A1F9B061F06C401C6E
:10EC1000F064FEF73BF9F063FAF756FC306401202C
:10EC2000707170BDB896010288D30102C6900102CE
:10EC3000F0B581B0EFF3108072B600200146FBF70B
:10EC40007BFE0446002803D062B6204601B0F0BD2A
:10EC500001273A030025074E28463146FBF7C6FD3B
:10EC6000BB021C4A28463146FCF79EFA62B6204693
:10EC700001B0F0BD00E0020410B5F5F7D2FD134C71
:10EC8000E078002801D0F9F795F9F9F709FAF7F7D4
:10EC900017FF0F480121C173027C0B469343837217
:10ECA000521C02740B4A928F002A08D0427B837850
:10ECB000134304D0027B511C017301219143617005
:10ECC000817B002901D0491E817310BD1C90010277
:10ECD000989901024AA9010270B514460D460646EC
:10ECE0001120FAF7C7FE2248042101600C48046095
:10ECF0001E4805608660002E0DD0FF2000060949E1
:10ED00000A6882430120C0071018086006480821DD
:10ED10000160064801601A200221FFF777FB70BDF1
:10ED200088D4010200E400E080E200E000E100E0BD
:10ED30000C4908607047C04610B504460948006891
:10ED400060430949F1F7DCF90019084948600848AF
:10ED50000022026002460C3A4B68136009680160A9
:10ED600010BDC04684D4010240420F000C90010245
:10ED70002C10014000480047C100000080B582B05F
:10ED800013460A4600900348011D0348F7F784FD27
:10ED900002B080BDC4D4010274A0010210B50C49B8
:10EDA0008A1C90420DD2401E0D4A50600D480368E7
:10EDB0000B4003218C071B19036000209060116039
:10EDC00010BD04480449E622044B00F06FF8C04629
:10EDD000FFFFFF00852F01009F2F01006B2F010017
:10EDE00010E000E020ED00E0B0B50120EFF310816D
:10EDF000014002D1EFF3108272B6124A1368124C2E
:10EE0000226864688506114800682840850E5D19EF
:10EE10002923DB006B43002C1D4606D1002809D1B5
:10EE20001E20684300290AD0B0BD121BD218551C01
:10EE30000028F5D01D461E2068430029F4D162B693
:10EE4000B0BDC046F4DF010214E000E004ED00E0D4
:10EE500080B50020FBF71AF8404280BDB0B586B0FF
:10EE6000104869460A4638C838C238C838C2002433
:10EE70002046FBF711F803992046FBF7A7F8019805
:10EE8000012803D00824002804D102E0042400282B
:10EE900000D104460220FAF7F5FDE040024908607F
:10EEA00006B0B0BD3020010008E0010290B01C4661
:10EEB00005AB07C3EFF31080C00702D1EFF310805A
:10EEC00072B6EFF310800B9068460E907046089073
:10EED00010AB0F93CF4F3E1D01200490C50230466A
:10EEE0002946224600F0B8FC00213154EFF303809C
:10EEF0000990EFF308800C90EFF309800D90EFF389
:10EF000014800A9000F02CFC3868012833D80028BF
:10EF1000C14F00D0C14F2A20C1497A69920703D559
:10EF20000A783A60401E491C0028F6D1B948041DF1
:10EF30002046F1F74DF9002807D079698907FAD5FD
:10EF400021783960401E641CF5E70220B5497A69D2
:10EF5000920703D50A783A60401E491C0028F6D172
:10EF60002A20AF497A69920703D50A783A60401E91
:10EF7000491C0028F6D1FFF737FF0346AA4A30465E
:10EF80002946FDF7B5FE04463018291B089F3B1F94
:10EF9000049A9343A5A2FDF7ABFE9E490968012997
:10EFA00066D8001900299C4C00D09C4C00280AD03F
:10EFB0009849091D6269920703D50A782260401EAC
:10EFC000491C0028F6D10A209F496269920703D59F
:10EFD0000A782260401E491C0028F6D10598F1F7F6
:10EFE000F7F8002809D061698907FAD5059A1178E0
:10EFF0002160401E521C0592F3E702208949626994
:10F00000920703D50A782260401E491C0028F6D1D9
:10F010000A208EA16269920703D50A782260401EF9
:10F02000491C0028F6D10698F1F7D2F8002809D03B
:10F0300061698907FAD5069A11782160401E521C31
:10F040000692F3E7022077496269920703D50A78AE
:10F050002260401E491C0028F6D10A207EA1626968
:10F06000920703D50A782260401E491C0028F6D179
:10F070007CA230462946079BFDF73AFE65490968A0
:10F0800001290E9B1BD80029634900D06349002841
:10F090000AD0604A121D4C69A40703D514780C608D
:10F0A000401E521C0028F6D102205E4A4C69A4077B
:10F0B00003D514780C60401E521C0028F6D16AA2B9
:10F0C00030462946FDF714FE04463018291B694ACC
:10F0D0003B46FDF70DFE4F490968012911D800197B
:10F0E00000294D4900D04D4900280AD0494A121D37
:10F0F0004B699B0703D513780B60401E521C0028F8
:10F10000F6D15D4A30462946099F3B46FDF7F0FDA2
:10F110000446F800C00FB900C90F7A00D20F009260
:10F12000019102903019291BFB0F544AFDF7E0FDB5
:10F1300004193019291B3F233B40514AFDF7D8FDE4
:10F1400034490968012911D820180029324900D012
:10F15000324900280AD02F4A121D4B699B0703D55C
:10F1600013780B60401E521C0028F6D1454A3046E9
:10F1700029460B9BFDF7BCFD04463018291B424A6B
:10F180000A9BFDF7B5FD23490968012911D800192B
:10F190000029214900D0214900280AD01D4A121D0A
:10F1A0004B699B0703D513780B60401E521C002847
:10F1B000F6D1364A304629460C9BFDF799FD0446A8
:10F1C0003018291B324A0D9BFDF792FD1149096841
:10F1D0000129114A0DD80019002908D00F4A06E06C
:10F1E0005169890703D531781160401E761C0028CB
:10F1F000F6D128490E98091AA94200D32946890850
:10F2000000F03AFE24480068002800D0804700F053
:10F2100045F8C046D8E001020090014000A001403E
:10F22000DF2F01006D3D0100C82F01000D0A2323CF
:10F230002320415353455254204020307825303804
:10F2400058202323230D0A00A230010046554E43C7
:10F2500054494F4E3A2000004C494E452020202072
:10F260003A200000256400000D0A53503D25303837
:10F27000580D0A00673001007D300100893001001F
:10F2800071300100263001003530010044300100AA
:10F290004F30010000F80202D4E00102F748006894
:10F2A000012811D8002801D00B4800E0FC480C21AF
:10F2B0000A4A01E0002907D043699B07FAD5137871
:10F2C0000360491E521CF5E71E20FFF7BBFA00BF82
:10F2D00000BF00BF00BFFAE700A00140D22F01002D
:10F2E0008AB00646E448B06600F03AFAFFF77CFDC3
:10F2F0000346E248041D01200590C502E04A20466D
:10F300002946FDF7F5FC074608942018DB4C0995C3
:10F31000E91BF36C3F2206921340DAA2FDF7E8FCEA
:10F320002168012910D8C0190029DD4900D0DD4924
:10F33000002809D0221D4B699B0703D513780B6069
:10F34000401E521C0028F6D1F36BD7A2089C204621
:10F35000099D2946FDF7CCFC0746291A2018336C75
:10F36000069A134007D1D8A2FDF7C2FCC34C21680E
:10F37000012907D917E0CEA2FDF7BAFCBF4C2168DE
:10F38000012910D8C0190029C54900D0C549002855
:10F3900009D0221D4B699B0703D513780B60401ED3
:10F3A000521C0028F6D10027CBA5B8003058009099
:10F3B000089809992A463B46FDF79AFC21680129DD
:10F3C0000FD80029B64900D0B649002809D0221D1F
:10F3D0004B699B0703D513780B60401E521C002815
:10F3E000F6D17F1C0D2FE0D1736BBFA2089C204685
:10F3F000099D2946FDF77CFC074620189F4CE91B18
:10F40000B36BBC4AFDF774FC2168012910D8C01900
:10F410000029A34900D0A349002809D0221D4B6927
:10F420009B0703D513780B60401E521C0028F6D1B1
:10F43000336CB14A089C2046099D2946FDF758FCCB
:10F440000746326CD000C00F9100C90F5300DB0F8C
:10F45000009301910290E019E91BD30FA74AFDF731
:10F4600047FC3246C619A019A91B1546136C069A0B
:10F470001340A34AFDF73CFC80490968012911D8D3
:10F4800080190029864900D0864900280AD07B4A85
:10F49000121D4B699B0703D513780B60401E521C4D
:10F4A0000028F6D12E466B6C964A089C2046099D92
:10F4B0002946FDF71DFC07462018E91B0796B36C8B
:10F4C000914AFDF715FC6D4A1168012910D8C01941
:10F4D0000029734900D07349002809D0121D4B69D7
:10F4E0009B0703D513780B60401E521C0028F6D1F1
:10F4F0000798426E042360215C2004931A400B4657
:10F5000000D003460693002A00D00846079E3358D1
:10F510007E4A089C2046099D2946FDF7E9FB0746DF
:10F5200006983358E019E91B794AFDF7E1FBC61943
:10F53000A019A91B079A536E76A2FDF7D9FB4F4974
:10F540000968022911D280190029554900D055496E
:10F5500000280AD0494A121D4B699B0703D513782E
:10F560000B60401E521C0028F6D10798C36C06465B
:10F570006DA2089C2046099D2946FDF7B9FB074668
:10F580002018E91B336D6B4AFDF7B2FBC619A019B1
:10F59000A91B079F7B6D68A2FDF7AAFB8619A0191E
:10F5A000A91BBB6D67A2FDF7A3FB344909680129BC
:10F5B000059C11D880190029394900D03949002803
:10F5C0000AD02E4A121D4B699B0703D513780B6096
:10F5D000401E521C0028F6D10798476B5D4A97429F
:10F5E00037D2032087430026059CB00039580246D5
:10F5F000049B1A43BA5808230343FB580C250543C0
:10F600007D5900910192029303953B18089809993E
:10F61000514AFDF76DFB1949096801290FD80029E6
:10F620001F4900D01F49002809D0089A4B699B0741
:10F6300003D513780B60401E521C0028F6D11B2EF8
:10F64000444A06D80798406B361DB10040189042D6
:10F65000CBD30798406B111A099A914201D88908B7
:10F6600000E0610200F008FC3C480068002800D07F
:10F670008047FFF713FEC04622224B4DD8E001021F
:10F68000C82F01000D0A0D0A2323232045584345A6
:10F690005054494F4E202564202323230D0A000097
:10F6A0000090014000A0014050433D2530385800F3
:10F6B0002C20457863657074696F6E4E756D626558
:10F6C000723D25640D0A00002C2054687265616447
:10F6D0004D6F64650D0A000052252D32643D2530C2
:10F6E00038580D0A0000000053503D253038580DA1
:10F6F0000A000000673001007D3001008930010000
:10F700007130010026300100353001004430010025
:10F710004F3001004558435F52455455524E3D25E8
:10F720003038580D0A000000494353523D25303807
:10F73000580D0A005A3001005343523D25303858C5
:10F740000D0A00004343523D253038580D0A0D0A7A
:10F750000000000000F802020A300100D4E00102BB
:10F76000F0B583B0344D2C68012C06D8601E84415E
:10F77000204601F073FB0028FAD10120EFF310813D
:10F780000140019102D1EFF3108072B62B48285A44
:10F790002B49695A814245D02A68002A01D02A4E55
:10F7A00000E0284E1F23DB020293284C022A27D2B6
:10F7B00005E01046214AA85282B2914232D087B267
:10F7C000B9420A4600D8621C131A21482B52180469
:10F7D0000DD0E819001D9FB201E0002F07D073691A
:10F7E0009B07FAD5037833607F1E401CF5E7A242E1
:10F7F000DFD902981018DDE7304683B299420CD069
:10F80000024680B281420E4600D8661CA642F3D959
:10F810000298301883B29942F2D108496852B01A5E
:10F820000B4968520B48002129540198002800D147
:10F8300062B603B0F0BDC046D8E001020A0800007D
:10F84000080800000090014000A00140FF070000F0
:10F850000C0800000F080000F0B58DB007931746A4
:10F8600000240C9409AA13C215E006986849F0F721
:10F87000CBFDF1F793F8C117401848406549F0F700
:10F8800029FC009509A806223346F9F791FABDE054
:10F89000002C00D5BEE138787F1C25280DD000282B
:10F8A00000D1B7E10B9A511C0A9B9942F0D8099BF1
:10F8B0009854641C0C940B91EAE70894002539785D
:10F8C00023390D2914D801207944097949008F443E
:10F8D000090F0F0F0F0F0F0F0B0F060F0F0D054323
:10F8E0007F1CECE70820FAE70420F8E70220F6E79F
:10F8F0003878014630390024092902D9264639468C
:10F900000BE000260A2171430E18303E791C7878EE
:10F910000246303A0A2A0F46F4D32E2817D14A1C41
:10F92000487801463039092905D911464F1C253838
:10F93000532811D96AE000240A2161430C18303C95
:10F94000511C50780246303A0A2A0A46F4D34F1C1A
:10F950002538532800D959E04000C04678448088B3
:10F9600040008744A000530053005300530053004D
:10F9700053005300530053005300530053005300EF
:10F9800053005300530053005300530053005300DF
:10F9900053005300530053005300530053005300CF
:10F9A00053005300530060005300530053005300B2
:10F9B00053005300530053005300530053005300AF
:10F9C000530053005300530053009800530053005A
:10F9D000530053005300530053005300530053008F
:10F9E000AD00B600530060005300590053005300AF
:10F9F00053005900530053005300DE0053005300DE
:10FA0000BD005300D3005300530098000C9C3FE707
:10FA10000024744940420F00791C38780F4625387D
:10FA20005328F3D898E70799C91D07208143086830
:10FA300007914968F1F740F800210690F0F70EFFB2
:10FA400000280BD10B99481C0A9A904206D8099AB3
:10FA50002D2353540899491C0C910B90079808309A
:10FA600007900698F0F79AFF0095C2178118514049
:10FA700009A822463346F9F79BF90B98411C0A9ACC
:10FA8000914200D9F1E6099A2E2313540B910C9858
:10FA9000401C0C90E9E6079802C807900096019573
:10FAA00009A8102239E00B98411C0A9A9142ADD85E
:10FAB000099A252313540B910C98401C0C90A5E730
:10FAC0000B9A511C079C201D0A9B994239D907901B
:10FAD0009CE7079802C80790009509A82246D3E63C
:10FAE000079901C9079109990A9A089E02E0401CEA
:10FAF000002E8BD40378002B88D00B9D6C1C944275
:10FB0000F5D84B55761C0C960B94F0E7079802C875
:10FB100007900096019509A80A222346F9F7E6F90D
:10FB200074E7079B10CB102C079308D300202146C5
:10FB3000401C0A09FF291146FAD806280AD80820CD
:10FB400009E02368099CA354089A521C0C920B915B
:10FB500007905BE7401C069009230C980B9D0999C0
:10FB600005910A9E04940DE0202104463046059E2E
:10FB7000715506462046049C401C154601460891D6
:10FB800000290AD45B1E0699994206D26A1CB24229
:10FB9000EAD9089908910029F4D50C900B9508989A
:10FBA000002800D532E70126082501E06D1E360148
:10FBB000022DFBD220463146F0F78CFA0F28F6D8FA
:10FBC0000C980590099803900A9806900B9D204682
:10FBD0003146F0F77FFA691C069A914204D90899D8
:10FBE000089100290CD511E00C4A125C039B5A5570
:10FBF000089A521C0D46059211460891002905D419
:10FC00007043241A3009102E0646E0D205980C9055
:10FC10000B95FBE620460DB0F0BDC0462423010045
:10FC200070B588B00022032803D9D243104608B02B
:10FC300070BD7F4CC34D2A510F4B104EEE508123A7
:10FC40001E010123AB5528602C1962600128EDD8F4
:10FC500007930022069205920492032303930292D3
:10FC600001920091411E8841694600F027FD02463D
:10FC7000104608B070BDC04604080000FFC0FFC0B9
:10FC8000F0B583B00C460023D943012C56DB074660
:10FC900002910126EFF31085354002D1EFF3108079
:10FCA00072B65849584A505C002800D0A3E0565418
:10FCB0005E48115A5E48105A0196F202161A8142A5
:10FCC00040D832465218A24240DB00930295A64229
:10FCD000354600DB25464C490818001D39462A46A2
:10FCE000F0F748FAA642484E04DA7919621B301D33
:10FCF000F0F740FA4E48305A001981B24D4A91420D
:10FD000001D94D494018029D009B49497052304627
:10FD10004A4E805D002865D1EFF3108501980540BB
:10FD200002D1EFF3108072B6374A4048115A40486A
:10FD3000105A884232D1424813524FE00C462046B6
:10FD400003B0F0BD42425218A242BEDA3B4A2E4EE8
:10FD5000B25C002A0CD03A4AB25A51188AB2354CD9
:10FD6000A242284C029F01D9334A8918304A02E046
:10FD7000244C2F4A029F3355B152421A89B288420D
:10FD800002D22C488018421C93B22F4801212FA286
:10FD900000F0E8F83C46002DD1D128E0019F9755AE
:10FDA000884201D82348401C421A90B2800A01D0F0
:10FDB000019882022248144F3A52386801280DD81F
:10FDC000431E9841104B5918091D92B21D4B00F06B
:10FDD0008BFE009B002801D00B488355002D029D0F
:10FDE00000D162B6074808490B54002DA7D162B66E
:10FDF000204603B0F0BD21200201044804A108A35D
:10FE0000FFF754F80E080000D8E001021E3101008F
:10FE100074726163655F6F757470757400000000C3
:10FE20005452414345204255535900000A080000EE
:10FE300008080000FF07000000F8FFFF0F0800009F
:10FE40000C0800009100010002FF00000D0A54722E
:10FE500061636520627566666572206973206675E8
:10FE60006C6C2C2064697363617264732025752047
:10FE700062797465730D0A00F0B587B005460026F7
:10FE800006960596049603960296800701D007B061
:10FE9000F0BD019102A8142126A2FCF729FF2949EF
:10FEA0000968012911D80029274900D027490028CD
:10FEB0000BD002AA01E0002807D04B699B07FAD5B6
:10FEC00013780B60401E521CF5E701990029DED023
:10FED000204C3746B8002B58D80724D0581EA042D3
:10FEE00004D31B4818181C4A90421CD802A814219D
:10FEF0001AA2FCF7FDFE13490968012911D800294F
:10FF0000114900D0114900280BD002AA01E00028B5
:10FF100007D04B699B07FAD513780B60401E521C23
:10FF2000F5E7761C01997F1C8F42B0D2322ED1D3D7
:10FF3000ADE7C0460D0A4261636B74726163653A56
:10FF4000200D0A00D8E001020090014000A001400D
:10FF5000FFFFFFFCFFFF0200FEFF010025303858C5
:10FF60000D0A000081B0F0B5C4B00E4607464993B3
:10FF7000812000012F49085C002845D00292012011
:10FF8000050204A82946F0F70EF9FCB20021C84387
:10FF90000C2C3AD8721E032A37D82748005DB0428D
:10FFA000084632D3F80535D50021B8050DD404A88C
:10FFB00001904018691AA20022A39B582E4AFCF710
:10FFC00097FE0198F0F704F9014678050ED404AFC6
:10FFD0007818691AB20029A3D218121F1368264A8A
:10FFE000FCF786FE3846F0F7F3F80146029A04AEB5
:10FFF00070180C46691A49AB0393FFF72DFC0119E1
:020000040001F9
:100000003046FFF73DFE00E0002044B0F0BC02BCEB
:1000100001B00847FEF7E8FE034604A8019007A2D6
:100020002946FCF765FE0198F0F7D2F80146B805BD
:10003000BDD5CAE7D8E0010250490100253130752D
:10004000207C2000C2300100183101001231010073
:10005000F1300100BC300100DD3001000B31010046
:1000600004310100FF300100B5300100C83001004B
:10007000D8300100AD300100D1390100F730010066
:10008000E3300100EA300100CE3001000000000042
:10009000F0B581B00B460120EFF31084044002D18B
:1000A000EFF3108172B6990F07D0022001212DA223
:1000B000FFF758FF002C3DD141E02249224D002797
:1000C0006F54224AAB5A224AAE5AF3189EB2F60A2D
:1000D00001D0204E9B19AB52EFF31086064002D19F
:1000E000EFF3108372B6AA5A1C4BEB5A934202D11B
:1000F00016482F521AE06854934201D8164B5B1CE5
:100100009B1A99B2890A00D0830210482B522868A2
:1001100001280BD8411E8841A918091D9AB2104B1D
:1001200000F0E2FC002801D006482F54002E03D036
:10013000002C04D001B0F0BD62B6002CFAD162B63A
:1001400001B0F0BD0F080000D8E001020C0800006B
:100150000A08000000F8FFFFFF0700000808000081
:100160009100010055415254204572726F72202552
:10017000780D0A0010B50446FEF7E6F8A08A0028BC
:1001800000D010BDFDF7E2FE034948624861886C6B
:10019000401C886410BDC046D098010210B50446CA
:1001A000FEF7D2F8A08A002800D010BD0A4CA06C3F
:1001B000401CA064FDF7CAFE6062606C002805D098
:1001C000FDF7C4FE60650020606410BDA069206575
:1001D0000120606410BDC046B896010210B50A2027
:1001E00000242146FBF7BAFC09202146FBF7B6FCA8
:1001F0000124204600F038F80E200421FBF7AEFC65
:100200000549204600F05AFAA2021549154B20462E
:1002100000F028FB10BDC046DC940102B0B50E20F2
:1002200000242146FBF79AFC0D202146FBF796FCA3
:100230000124204600F018F80A2004252946FBF77F
:100240008DFC09202946FBF789FC2046F9F760FA66
:10025000A2020349034B204600F004FBB0BDC04698
:10026000F8CD01029D0A010070B5012801D90120D5
:1002700070BD48224243734B9C58A5691F218D4392
:10028000A5610625A5600F2525629C18A27C002A81
:1002900005D1627C002A02D1227C002A14D0636836
:1002A000002B11D4251D0B40012216469E400C4BFD
:1002B0001E60BFF34F8FBFF36F8F2B68002B03D4EB
:1002C0000B409A4007490A60002803D0012804D156
:1002D000092000E00820F9F7C5FB0020A06170BDEF
:1002E00080E100E080E200E0F0B585B00D460278E4
:1002F000E348C368934219D0446D944216D0836892
:10030000934203D0016D914200D07FE09B1A591EA9
:100310008B41049348215943032D46D14418E16988
:1003200000294ED01C34002020606DE09B1A5A1E1C
:1003300093410493032D1AD1039548225A438418FC
:10034000A26B0121EFF310850D4002D1EFF310876E
:1003500072B6A7691026B743A761A669002E01D11E
:1003600018342160002D00D162B6039D0CE04821B5
:100370005943421891691832302902D01168102966
:100380004CD180211160002248215943401800219E
:10039000816301628162243000210160002A33D030
:1003A00004A82946904705B0F0BD4218916918325B
:1003B000302902D01168202939D180211160002212
:1003C00016E00395E26B0126EFF31085354002D16C
:1003D000EFF3108172B6A1692027B943A161A16929
:1003E000002901D118342660002D00D162B6039D8A
:1003F0004821594340180021C163C1624163303034
:1004000000210160002ACBD105B0F0BD00920E4A58
:100410002E329C480D490E4BFEF748FD10680093A4
:10042000019098480949084A0A4BFEF73FFD1068B9
:1004300000930190044A243292480449054BFEF788
:1004400035FDC046FC940102B10200009A31010062
:100450006F31010053310100F0B585B0049048219F
:100460000A464243864B9C58E6690F2535409A1848
:10047000167C002E31D04F2040026169014200D12C
:1004800085E0A06904218843A06102202062012048
:1004900081076918D161D36BEFF31084044002D156
:1004A000EFF3108572B695692026B543956195697D
:1004B000002D00D173E010463C30002C00D162B614
:1004C00000240460D4625463303200201060002B9A
:1004D00063D004A8984705B0F0BD0C2D5DD8C04688
:1004E0007D442D796D00AF4467586B580658A16361
:1004F0005858585806009569202D04D015461835CF
:100500002D68302D49D1156B566B3432AE4217D25F
:100510006669360714D5646815686E1C1660484312
:100520001818C06A445504980C4644431A19156BB0
:10053000566B3432AE4203D21C5966693607EAD490
:100540001268AA4229D14143585882690524A2431E
:1005500082615A18D36B0121EFF31080084002D159
:10056000EFF3108472B694692025AC4394619469CA
:10057000002C02D114461834216014463C34002863
:1005800000D162B600212160D16251639CE70C2D3D
:1005900000D176E7012D00D173E705B0F0BD154617
:1005A0001835286010463C30002C00D187E787E7DB
:1005B0000420206205B0F0BD0120206205B0F0BD2E
:1005C00008252562164618369569102D02D0356823
:1005D000302D4BD10396566A15462835976AB74297
:1005E00028D1A06902218843A061936B0121EFF318
:1005F0001080084002D1EFF3108472B6039E346875
:100600001027BC4334603468002C00D1316014469C
:100610003834002800D162B60021216029601162BF
:10062000243200201060002BB7D052E70220206255
:1006300005B0F0BD2A68B242AFD262699207ACD56C
:100640002A68561C2E6048431818006A805C206097
:1006500004980A4642439D18AC6A6E6AB4429CD222
:1006600028359C5862699207EAD496E73168009071
:100670000191044804A1094A09A3FEF717FCC046EA
:10068000FC94010239310100756172745F69727105
:100690005F68616E646C6572000000003D030000DD
:1006A0005561727420256420737461746520676FCE
:1006B00065732077726F6E6720256400F0B585B092
:1006C0000E460546022804D3002E02D1012005B0B3
:1006D000F0BD002D03D0012D08D1092400E008242D
:1006E0002046F9F7C7F92046FEF7ACF848216943E0
:1006F000E74A505883691F240294A3438361062369
:1007000083600F230193036257180023BB62BB630E
:10071000FB633B627B62FB623B63317F3974727FB8
:100720007A74B27FBA7404937B637368B268F468B6
:10073000920022435B1E032B0ED8C0467B441B79DC
:100740005B009F4401050307082304E0282302E01F
:10075000182300E038231A43C260C907090F7269E1
:100760009201D2B28918B2699207920E8918491C77
:10077000816079613169012901D122210161012D55
:100780005CD831680E2959D23846123003900324C0
:10079000002D01D0204600E004204C432D490E19C5
:1007A000B178F9F7F7F93968CA6880251046284307
:1007B000C8602848005D73781B021818C862AA43F5
:1007C000CA60F9F72FFA03980078002809D1384653
:1007D00011300078002804D1384610300078002805
:1007E00027D07868002815D4032102468A431B4984
:1007F00053588407E40EFF26A640B343A5401D438B
:1008000055500299014001208840A24908601449CE
:1008100008600EE08107C90EFF228A40019C044057
:10082000083C032084430C48235893438D401D43C8
:1008300025500120B861049805B0F0BD0248034975
:10084000DA22034BFEF732FB39310100AC310100F3
:1008500089310100B82001001CED00E000E400E057
:1008600000E100E0F0B58FB00E900125002900D125
:100870004BE0039304910592002A00D145E0012149
:10088000EFF3108201910A4002D1EFF3108172B6AA
:100890004827029747437E49CE19B5690023302D7A
:1008A00023D831461831C0467D442D796D00AF44C0
:1008B00020242626262626262626262626262626E0
:1008C0005E26262626262626262626262626262690
:1008D00018262626262626262626262626262626C6
:1008E00018000223002A0CD00CE0402D01D0802DEE
:1008F00005D10123002A04D004E020240C60002A42
:1009000000D162B61D46002B02D028460FB0F0BDC4
:10091000002575630399F1630499F16205993163C8
:100920005B4CE35959691322D202114205D00621CA
:1009300099600F21196271699960317C00290CD08E
:10094000F56109950895079506950D950B9502217A
:100950000A91012810D017200FE0717C9A690029B4
:100960002CD0952002439A6128460FB0F0BD302468
:100970000C60002AC5D0C5E71920049F0C90706850
:10098000002805D41F210840019981404148016099
:1009900014209861B06806A9F9F7B4F90E98029985
:1009A00041436018806861583B4A0092091D3A46ED
:1009B000059BF9F717FA28460FB0F0BD343611063B
:1009C00002D580218A439A6131680025059A9142B7
:1009D0002DD205955D694F214A0215421BD1E905CB
:1009E00002D4029CF24F0AE0596833685C1C346000
:1009F000029C6043EE4F3818C06AC1540E982146DD
:100A000041437E18736B346BA34238D234367B5823
:100A10005D691542E3D002211962019EB1072943A5
:100A20003546E34CEFF31082324006D008E0294609
:100A3000019EEFF31082324002D1EFF3108372B6C1
:100A4000029B4343E01883692024A34383618369A5
:100A5000002B05D0002A08D0C26B002A0AD154E727
:100A6000034618331E60002AF6D162B6C26B002A14
:100A700000D14AE70EA8904728460FB0F0BD29469E
:100A8000059D019E3C46EFF310823240D5D0D7E75A
:100A9000FC94010280E200E0E902010080B501203F
:100AA00082020249024BFFF7DDFE80BDF8CD010254
:100AB0009D0A0100B0B582B079208400E54D285D23
:100AC00001A90870652080002818F2F77FFF2F2009
:100AD000C000285829190122024BFFF7C3FE02B0BB
:100AE000B0BDC046B50A0100F0B591B01090012626
:100AF000002900D19BE003930591002A00D196E0E4
:100B000007900121EFF310800291084002D1EFF32A
:100B1000108172B604924823069307994B43D64935
:100B2000C9188D690026302D6ED80C461834AD00DA
:100B3000374602A675593E46AF46C046110C010025
:100B4000190C01001D0C01001D0C01001D0C010001
:100B50001D0C01001D0C01001D0C01001D0C0100ED
:100B60001D0C01001D0C01001D0C01001D0C0100DD
:100B70001D0C01001D0C01001D0C0100010C0100E9
:100B80001D0C01001D0C01001D0C01001D0C0100BD
:100B90001D0C01001D0C01001D0C01001D0C0100AD
:100BA0001D0C01001D0C01001D0C01001D0C01009D
:100BB0001D0C01001D0C01001D0C0100AF0C0100FB
:100BC0001D0C01001D0C01001D0C01001D0C01007D
:100BD0001D0C01001D0C01001D0C01001D0C01006D
:100BE0001D0C01001D0C01001D0C01001D0C01005D
:100BF0001D0C01001D0C01001D0C0100010C010069
:100C0000022600280CD00CE0402D01D0802D05D10B
:100C10000126002804D004E010252560002800D11A
:100C200062B6002E069D944F049C079802D0304671
:100C300011B0F0BD00268E62039A8A63059A0A629B
:100C40004C620A7C002A0BD00C960B960A960996E9
:100C500008960E9602220D9201282DD018202CE025
:100C60008A7C2831002A3BD00A68A24216D22B4641
:100C70004343FA585469A40710D50868441C0C6013
:100C8000F918096A085C10601098294641437A18DF
:100C900011462831936A526A9342E8D34543785902
:100CA000816982220A438261304611B0F0BD30254D
:100CB00025600028B4D0B4E71A200F90C86808A9AE
:100CC000F9F720F8109845437A597819C0683949DE
:100CD000009105992346F9F785F8304611B0F0BD2B
:100CE000FB589A69140602D58024A2439A610A68C7
:100CF0000026049882422ED25D694F22520215428C
:100D000007980AD002211962029EB10729431FE009
:100D100028315D6915423E46F4D137465C69A40727
:100D200002D40699544E0AE00C68661C0E600699BF
:100D30004843514E3018006A005D186010984143D6
:100D4000735871188C6A4E6AB442E1D329463E4604
:100D5000069D494F01E0314607985A6A002AFCD1A6
:100D6000EFF31082029B1A4002D1EFF3108372B6A8
:100D70004543781983691024A34383618369002B59
:100D800005D0002A09D0826B002A0BD14FE7034619
:100D90001833029C1C60002AF5D162B6826B002ACF
:100DA00000D144E710A89047304611B0F0BDC046CE
:100DB000FC940102E9020100B0B5264900684A68C6
:100DC000824202D10D1D002016E080228A58824204
:100DD00003D10D46803501200EE0FC228A58824264
:100DE00003D10D46FC35022006E02F22D2008B589D
:100DF00083422ED18D1803207C2242438C18A06898
:100E0000012814D0002824D140342046F3F7CDF92E
:100E100001462046F3F79FF92046F3F7C6F900286C
:100E200017D006C828680C4BFFF75EFEB0BD4034F3
:100E30002046F3F7BAF901462046F3F78CF920462D
:100E4000F3F7B3F9002804D006C82868024BFFF76F
:100E50004BFEB0BD70BE0102B90D010048214143F7
:100E6000054842189269D20601D4002070474058C4
:100E70004169012008407047FC94010280B5114887
:100E80000078C00110490978890101430F480078B2
:100E9000400108430E490978090101430D480078D3
:100EA000C00008430C490978890001430B480078C9
:100EB000400008430A4909780143C8B2F3F726FC09
:100EC00080BDC046F89E0102B69601021D90010247
:100ED0007CEA0102B1AD0102F99E01023CA30102CC
:100EE0003DA30102F0B587B0014601270225052880
:100EF0003A4600D02A4600200929014600D0114672
:100F0000C900374A54180E210591615EFDF7A6FA13
:100F10001026A15F3846FDF7A1FA1227E15F2846A7
:100F2000FDF79CFA06951425615F03200490FDF7F8
:100F300095FA0598235EA05FE15F625F00AD07C58B
:100F400028A2069F3846049D2946FFF70BF8204645
:100F5000263004263146FBF741FF2620235E282059
:100F6000205E2A21615E2C22A25E009001910292F5
:100F700024A238462946FEF7F5FF27463E37384675
:100F80003146FBF749FF3E20235E06983C5EB95F81
:100F90000622BA5E00940191029221A207462E46D3
:100FA0002946FEF7DFFF56240D4D285FFBF728FF8B
:100FB0002B5F2C4621A2384631463546FEF7D2FF3C
:100FC000264658363046FBF707FF5820235EF05F71
:100FD00000901FA238462946FEF7C4FF07B0F0BDB7
:100FE000DCA00102546F4620616E742064656C6160
:100FF00079732025642025642025642025640D0A4A
:101000000000000050446F412064656C61797320DA
:1010100025642025642025642025640D0A00000035
:1010200050446F41206761696E73202564202564F8
:101030002025642025640D0A0000000050446F4103
:1010400020616E742073706163652025640D0A0051
:1010500050446F4120616E676C65206F66667365F2
:1010600074732025642025640D0A0000F0B587B054
:1010700015467A4B1A680F24A2432F783A431A6018
:10108000774C23462C3B774A1A600490034622464D
:10109000283A12681207FAD5734E092F029306D91F
:1010A000754A326072600C2F09D175480FE0042F29
:1010B00007D9704A3260704A7260092F06D37148AE
:1010C00005E06A4830607060694800E06B486E4A2D
:1010D0001060EB7AFF2B039102D10020B0620AE08E
:1010E00003210B406948C05C40220243B2620220E7
:1010F000674AFEF737FF029F0021384605952A46CA
:101100000B46FBF7F5FE06460225032161A22846A1
:1011100001913346FEF726FF06963046FCF7BCFBEE
:1011200001210498009108402CD13D4033D1604901
:1011300000283AD1002D1ED06548A062E0622063ED
:1011400060636448606264480860152085046E1C12
:101150008E608D60642420460F46F8F763FD3E6084
:101160003D602046F8F75EFD281D386003215BA234
:101170004E48FEF7F7FE0598007BFAF7B5FF069894
:1011800007B0F0BD2E4605460698FCF711FF28462D
:1011900035463D40CBD02E4605460698FCF784FBED
:1011A0002846354642490028C4D042480861424892
:1011B0004861424888611520C86141480168402261
:1011C0000A43026007210803274B5A6982430098AB
:1011D0004003101858610522039842432A480368C7
:1011E0009818334E766B47780F40995C0907490E83
:1011F000C919CA03334B33409A18C9015118324AEE
:1012000089182B4A51632A49896B38229143827885
:101210005207920E891804220A4325498A63124B09
:1012200019690279019E3240C0784007C00E8018CB
:101230001F2291430818186155204003411C21606A
:1012400020606420F8F7EEFC204A18483146039BE2
:10125000FEF788FE1649002D8DD06DE7040400408E
:101260002C60004000040080000600400F040F04C2
:10127000412B01000304030400040004722C01004C
:10128000102A0100A32D010048940102D42E010070
:10129000D831010050485920706172616D7320731C
:1012A00065747320253038780D0A000002080000AC
:1012B0009060004012A83E009DD79B5AD579BD4949
:1012C000340200403F0080FF40400000BA3101007E
:1012D0002008820002D50F00020255007577625F78
:1012E00072785F696E69740D0A00000080B522484B
:1012F0000021017022480078C00120490978890145
:10130000014320480078400108431F490978C9007B
:1013100001431E480078800008431D4909784900B0
:1013200001431C4800780843C0B2F3F7EFF980BDD1
:1013300080B51148012101701048007880011049E2
:101340000978C90101430F480078400108430E495C
:101350000978C90001430D480078800008430C4912
:101360000978490001430B480078084310210143E4
:10137000C8B2F3F7CBF980BD7CEA0102B696010250
:10138000F89E01021D900102B1AD0102F99E010219
:101390003CA301023DA30102F0B581B01820FDF786
:1013A00051FA1920FDF74EFA002420462146F7F79E
:1013B000EFFF20462146FAF71BFE012603257F2377
:1013C000304629462A46FAF72BFF3046FBF7D0F87D
:1013D00002273846FBF76CFD30463146FCF7BAFD74
:1013E00003A238462946FEF7BDFD204601B0F0BDF8
:1013F0007577625F6F70656E0D0A0000F0B581B0A1
:10140000164600910446002001273946FCF7CAFF22
:10141000EFF310853D4002D1EFF3108072B6272024
:10142000400170430A21EEF755FE0246002C02D01F
:101430000020009901E002200021FBF79FF80446FC
:10144000FBF766F9002D00D162B6204601B0F0BD71
:1014500070B504460E4D29680F2001400629FAD0C8
:1014600029680140072912D10120EFF310860640B8
:1014700002D1EFF3108072B6FCF768FDFA30A86075
:10148000002C01D0FAF7C6FE002E00D162B670BD66
:1014900000040040F0B581B01D460E460446022A05
:1014A00009D1012738463946FCF77CFF0096002217
:1014B000384629460FE0174601200021FCF772FF4D
:1014C000012F04D1009600202946024603E0009631
:1014D000022000210A462346FBF732F90446FBF7B7
:1014E00017F9204601B0F0BD70B5002801D00120E9
:1014F00070BD0325A9020F4802680F4B535000240A
:101500009460012253030D4E3360BFF34F8FBFF33E
:101510006F8F0B4E336003685A5084720481102021
:10152000F8F7A0FA022007A22946FEF71BFD204685
:1015300070BDC0468C95010251E5CC1A80E100E0F7
:1015400080E200E057445420636C6F73650D0A001D
:101550000FB47CB50C0009AD01D0611E00E0002184
:1015600001910090074B6A462946089800F012F94D
:10157000002C02D0009A002111707CBC08BC04B081
:1015800018470000CD1E01007CB51D4616460C0014
:1015900001D0611E00E0002101910090054B6A46D8
:1015A0002946304600F0F6F8002C02D0009A0021BF
:1015B00011707CBDCD1E01002021020C01D0102134
:1015C0001046020A01D010460839020901D010461F
:1015D000091F820801D01046891E420801D0881ECA
:1015E0007047081A704700000048704708900102D1
:1015F00002E008C8121F08C1002AFAD170477047DC
:10160000002001E001C1121F002AFBD17047000039
:10161000F0B51FB486B00998089A030D0021024363
:1016200014D05148514A18185043051411980128F4
:1016300010981AD0281A401C00264D4F4D4900968C
:1016400001910490002812DA444211E0119801241B
:1016500049A3012801D11098C1430698119A8460CA
:101660000360C26041600BB0F0BD4042E4E7044655
:10167000210500203F4A001C51410391029012E0D5
:10168000E00707D032463B4601990098EEF7EAFFA3
:101690000191009032463B4610461946EEF7E2FFB4
:1016A00006460F466410002CEAD10498039B0028DC
:1016B000029A0999089806DAEEF7D4FF019B009A7E
:1016C000EEF7D0FF05E0EFF735F8019B009AEFF752
:1016D00031F804460E460022284BEFF7F7FB03D8FB
:1016E0000020C043014607E00022254B204631463A
:1016F000EEF706FFEFF7CAFB102409E0002C0ADB27
:101700000A220023EFF7F4F9079B30321A55641EC2
:1017100002460A43F2D11122641C079B121B1C19BA
:10172000119B012B03D0012308430ED10AE008438B
:1017300004D0112010900020119077E71098151A0E
:101740006D1E0BE01098824202DD00236D1C03E049
:10175000824201DA00236D1E002BEED0069811990B
:101760008260C16030C07EE701FCFFFF104D0000C9
:10177000000014400000F03F300000000000F04383
:101780000000E03F30380A2801D2012070470020D5
:1017900070470000FFB597B00646002518E22528DF
:1017A00077D100242746FD49049400E00443761CC9
:1017B00032780120203A90400842F7D130782A2828
:1017C0000ED00222307801463039092916D8049902
:1017D0000A235943303940181443761C0490F1E72A
:1017E000189802C804911890002904DA01204003D7
:1017F00004434842049002200443761C30782E288B
:1018000014D1042004437078761C2A2809D1189832
:10181000761C80C8189009E00A214F43303FC71951
:10182000761C3078014630390929F5D930786C2892
:1018300010D006DC4C281AD068280ED06A2817D1A0
:1018400004E0742813D07A2812D110E0012040055A
:1018500004430CE00121090501E0032109050C43C3
:101860007178814203D1012000052418761C761C72
:101870003078119066280BD013DC58287DD009DC15
:1018800000287BD04528F6D04628F4D047281AD126
:10189000A5E118E0632835D0642870D0652812D1FE
:1018A0009DE170286CD008DC6728F1D069287BD0D6
:1018B0006E280DD06F2806D1BAE073282ED0752877
:1018C00071D0782859D01A9A199990476D1C7EE1E9
:1018D0006002400F022809D003280DD00428189870
:1018E00001680DD00D60001D189070E11898EA177E
:1018F00001680D604A60F6E7189801680D80F2E70C
:101900000D70F0E718986A4601781172001D189062
:101910000020507202A80090012005E0189802C82B
:10192000189000200091C04361070DD5002101E00F
:101930000199491C0191B94212DA8142F8DB009AFF
:10194000515C0029F4D10BE0002101E00199491C10
:1019500001918142FADB019A0099895C0029F5D155
:10196000019904981A9B471A21463846199A00F0A3
:1019700097FA0199401945180BE04FE02CE113E06C
:101980004EE0009800990078491C00911A9A199924
:1019900090470198401E0190401CF2D121463846E4
:1019A0001A9B199A10E137E00A200021009001915A
:1019B0006002410F022907D0189A01CA1892C21773
:1019C0009446032908D00AE01898C01DC108C90030
:1019D00005C91891944607E000B2C217944604293D
:1019E00002D140B2C1178C4600226146944506DA06
:1019F0000A460021404291418C462D2102E02105FA
:101A000004D52B216A461173012103E0E10701D0BF
:101A10002021F7E7029155E00A200AE0102008E0B3
:101A2000102000900021042004430191082703E0C6
:101A300008200021019100906002410F022907D087
:101A4000189A01CA189200229446032908D008E087
:101A50001898C01DC108C90005C91891944603E033
:101A600080B2042900D1C0B200210291210729D5FA
:101A70001199702906D0009A1021019B4A401A43FF
:101A800005D00EE040216A461173012108E061464D
:101A9000014306D030216A46117311995173022116
:101AA0000291009A0821019B4A401A430AD16146DB
:101AB000014301D1610705D530216A461173012127
:101AC0007F1E02911199582904D035A10E910DA9BC
:101AD0000D910DE037A1F9E76146019B009AEFF700
:101AE00007F80E9B8C469B5C0D9A521E0D9213704C
:101AF00061460143F0D10D9805A9081A20300190E4
:101B0000600703D501200004844300E00127019809
:101B1000874201DD381A00E0002001990090411849
:101B2000029809180498401A0490E00306D421464C
:101B30001A9B199A049800F0B3F94519002706E09A
:101B400003A81A9AC05D199990476D1C7F1C0298D2
:101B50008742F5DBE0030CD521461A9B199A0498BD
:101B600000F09EF9451904E01A9A3020199990471F
:101B70006D1C0099481E00900029F5DC08E00D98C6
:101B80000D990078491C0D911A9A199990476D1C6E
:101B90000199481E01900029F1DC63E10928010048
:101BA00030313233343536373839616263646566D3
:101BB0000000000030313233343536373839414295
:101BC000434445460000000000F05AF94519761CD0
:101BD0003078002800D0E2E528461BB0F0BD600751
:101BE00000D406271898C01DC108C90048680A68B3
:101BF0000831C30FDB071891190001D09CA108E040
